:020000040000FA
:107800005469616E59696E673130300000000000C4
:1078100054593230302E303830303030625F747925
:10782000424154333247313339474B3634464200B4
:1078300043414E5F5354440000000000000000002C
:1078400043414E5F43485F300000000000000000ED
:1078500043414E5F3530304B6270730000000000D2
:107860009407000014070000DF070000000000007C
:020000040000FA
:1080000090330020E9800000F1800000F380000040
:108010000000000000000000000000000000000060
:10802000000000000000000000000000FB800000D5
:108030000000000000000000FF80000009CD0100EA
:10804000C115010005160100351601006516010075
:1080500095160100C5160100F5160100251701004F
:108060005517010085170100B9170100CD17010050
:10807000DD1701001118010021180100311801005D
:1080800065180100A9180100F11801003919010053
:1080900081190100C9190100D91901000D1A010047
:1080A000411A0100711A0100A51A0100D91A010034
:1080B000E91A0100F91A01002D1B0100611B0100E2
:1080C000EF72E8FF03B40148019001BD897F0020F1
:1080D0000448854600F02CFA00480047B51102001C
:1080E000C046C046903300201648804716480047D7
:1080F000FEE7FEE7FEE7FEE7FEE7FEE7FEE7FEE758
:10810000FEE7FEE7FEE7FEE7FEE7FEE7FEE7FEE747
:10811000FEE7FEE7FEE7FEE7FEE7FEE7FEE7FEE737
:10812000FEE7FEE7FEE7FEE7FEE7FEE7FEE7FEE727
:10813000FEE7FEE7FEE7FEE7FEE7FEE7FEE7FEE717
:10814000FEE700000DD30100D180000030B50B46E2
:10815000014600202022012409E00D46D5409D4221
:1081600005D31D469540491B2546954040191546A7
:10817000521E002DF1DC30BD70B5002425460028CC
:1081800001DA01244042002901DA01254942FFF7C2
:10819000DDFFAC4200D04042002C00D0494270BD0F
:1081A000F0B51FB40646002082B005464024019178
:1081B00000901BE0019922460F46304600F066F918
:1081C000049A059B801A994110D3104619462246FD
:1081D00000F04CF9361A8F41019722460120002108
:1081E000009F00F043F938184D4100902046641E6E
:1081F0000028DFDC019B00982946324607B0F0BD1D
:10820000F0B51FB486B0002000900190029006984F
:10821000069980B204900798090C020400141143D7
:1082200007900027089D099806913E463C4603901A
:108230000398A9B20204000C039004982D0C154376
:1082400048430021224600F011F9C719714110344A
:108250000E46402CECDB3846029A00F007F9009AF3
:10826000019B8018009059410298019110300290B2
:108270004028CCDB00980BB0F0BD03460B439B07B6
:1082800003D009E008C9121F08C0042AFAD203E08B
:108290000B780370401C491C521EF9D27047D2B2B1
:1082A00001E00270401C491EFBD270470022F6E735
:1082B00010B513460A4604461946FFF7F0FF20465C
:1082C00010BD30B504460020034600E05B1C93421D
:1082D00003D2E05CCD5C401BF8D030BD0321001D13
:1082E000401E037812021A43491EF9D51046704702
:1082F000034603220870000A491C521EFAD518468C
:108300007047024670B54A40D30FDB0740002DD0BE
:108310004A002AD0010E140E000212020919400A66
:10832000520A8418E50104465443000A120A2E0436
:108330005043A4194219200CC543AA18120C012558
:10834000AD03521C521912047F39240400D0521C70
:10835000104301D44000491EC2B20C06C0092018C7
:10836000401C4008802A02D003E0002070BD400875
:108370004000002900DA0020184370BD70B50246A5
:108380004A40D50F40004A00ED0740085208002837
:1083900014D0002A12D0C40DD30D41020120C00513
:1083A0005202490A520AE41A091812187D349142FD
:1083B00001D3641C00E04900002C01DA002070BDEC
:1083C0000023914201D3891A034340084900002841
:1083D000F7D100290AD0914202D10121C90705E055
:1083E000914201D2012101E00121C943E005C018F9
:1083F000401900F05CF870BD10B5002296231146BC
:1084000000F05DF810BDC20FD207400040080BD04D
:10841000C10D0723DB01C91840020905400A1143B9
:10842000C208400711437047002001467047000012
:1084300010B5002904DB0124E40740428C412146A9
:10844000002B04DB1C460123DB075242A341994267
:1084500000D1904210BD00000122D207002800DBAD
:10846000101A002900DB511A8842704710B5202AE3
:1084700004DB0146203A9140002010BD91402023AA
:108480009C1A0346E3401943904010BD10B5202AC2
:1084900004DB0846203AD040002110BD0B46D340F3
:1084A000D0402024A21A91400843194610BD00294B
:1084B00004DA401C490001D140084000704770B404
:1084C0000024050C05D11024000402D1002921D07C
:1084D0001124050E01D100020834050F01D100015D
:1084E000241D850F01D18000A41C002801DB400061
:1084F000641C002908D020252E1B0D46F540A14004
:1085000000D001212943084301061B1B000ADB1D83
:1085100002D5002070BC7047DB05181880180029B0
:10852000F8DA401C4900F5D170BC400840007047A3
:10853000064C0125064E05E0E36807CC2B430C3CB6
:1085400098471034B442F7D3FFF7C6FD0C2602005B
:108550003C26020070B58C180578401C6B075B0F39
:1085600001D10378401C2A1106D10278401C03E097
:1085700006780E70401C491C5B1EF9D12B0705D4F0
:108580000023521E0DD40B70491CFAE70378401CDF
:10859000CB1A921C03E01D780D70491C5B1C521E07
:1085A000F9D5A142D8D3002070BD70B507F064F9A9
:1085B0000524204618F0B8FD0025284607F052F99A
:1085C000204618F0B1FD0126304607F029F9204673
:1085D00018F0AAFD284607F023F9204618F0A4FD5C
:1085E000304607F03FF9204618F09EFD70BDB0B54B
:1085F00007F042F90524204618F096FD012528468B
:1086000007F030F9204618F08FFD284607F008F9EA
:10861000204618F089FD002007F002F9204618F0E6
:1086200083FDB0BDF0B581B007F014F9052018F056
:108630007BFD08270026012007F0F2F805242046DC
:1086400018F072FD204618F06FFD07F0F9F80546A6
:10865000204618F069FD002007F0E2F8204618F0E7
:1086600063FD76002E437F1E3806E4D1F0B201B0E0
:10867000F0BD70B50446002007F0D2F807F0FCF812
:10868000052018F051FD0826E0B2C00907F0EAF80D
:108690000525284618F048FD012007F0C1F82846B6
:1086A00018F042FD002007F0BBF8284618F03CFD0A
:1086B000284618F039FD6400761E3006E4D1052006
:1086C00018F032FD012070BDF0B583B0019314465F
:1086D0000E460746012038430290032504E000F0CF
:1086E0008EF86D1E280631D000F067F83846FFF787
:1086F000C0FF00F0A7F80028F1D13046FFF7B9FF1E
:1087000000F0A0F80028EAD100F057F80298FFF72F
:10871000B0FF00F097F80028E1D1019802280BD3B0
:10872000451E0026FFF77EFF2070FFF73EFF641C0A
:10873000761CF0B28542F5DCFFF774FF2070FFF77E
:1087400056FF00F05CF8202003B0F0BD102003B00D
:10875000F0BDF0B583B01C46009201910290032554
:1087600004E000F04CF86D1E280623D000F025F838
:108770000298FFF77EFF00F065F80028F1D101981C
:10878000FFF777FF00F05EF80028EAD1002C0CD04C
:108790000026009F3878FFF76CFF00F053F80028A0
:1087A000DFD1761C7F1CA642F4D300F028F8082005
:1087B00003B0F0BD102003B0F0BDB0B507F05CF819
:1087C0000524204618F0B0FC0125284607F028F8BB
:1087D000204618F0A9FC284607F044F8204618F077
:1087E000A3FC0025284607F03DF8204618F09CFC25
:1087F000284607F015F8642018F096FCB0BDB0B517
:1088000007F03AF80524204618F08EFC002528468B
:1088100007F006F8204618F087FC284607F022F8F3
:10882000204618F081FC0125284606F0F9FF204675
:1088300018F07AFC284607F015F8642018F074FC4C
:10884000B0BD0000B0B507F005F80524204618F0CB
:108850006BFC012006F0E4FF204618F065FC0B4D90
:1088600006F0EEFF044606F0D5FF002C02D06D1E88
:108870002804F5D10525284618F056FC002006F0FE
:10888000CFFF284618F050FC2046B0BD3321000031
:10889000034801780B2901D8491C01707047C04674
:1088A0007B2F002070B584B00025039502950195BB
:1088B000009506F0AFFF0F20C6430E4C1036F1B204
:1088C000A0206A461023FFF744FF204618F02CFC36
:1088D000204618F029FC912EF0D3A020B0216A4642
:1088E0001023FFF736FF204618F01EFC02480580D3
:1088F00004B070BD581B00006E2F002070B5022917
:1089000002D2EB24E0B270BD891EEB250022134693
:1089100005E0401C5B1CDDB2A94225460EDB047855
:108920006C40154604E034466E1C072D3546F0D2E7
:108930006608E407F7D09A246640F4E7E0B270BD19
:10894000F0B591B00C91417810AA117083781B0298
:108950005918C37804792402E3181B0459180B0E24
:10896000D3700C0C94700D0A55700B910895691812
:10897000099409190A93C9180278D24389184279CF
:1089800083791B029A18C379047A2402E3181B0422
:108990009A188918130A0693C918130C0593C91855
:1089A0000792120E04928918827AC37A1B029A18CF
:1089B000037B0F90447B2402E3181B0498180918CA
:1089C000020A02928918020C019289180D910390F3
:1089D000000E0E9000200346014606E032409A4009
:1089E000D2B211435B1C082B0ED0012635469D40A8
:1089F0000746024602E07F1C042FEFD010ACE45D76
:108A00002542F8D0521CF6E70E9C0D980019C3B20F
:108A10000F98827B934205D0427A914202D1002086
:108A200011B0F0BD1021FFF769FF0C99CC72019ACB
:108A30008A72029A4A72039A0A72049ACA71059A51
:108A40008A71069A4A71079A0A710A9ACA70099A33
:108A50008A70089A4A700B9A0A7011B0F0BDF0B58E
:108A60008DB055220270002747720B784370CA7987
:108A7000059202728A790492C2714A7903928271D4
:108A80000A7902924271CA7A089242738A7A0192F2
:108A900002734E7AC6720C7A84720CAA13704D78E7
:108AA0002D02EB188D78C978090249190904CB18F1
:108AB000190E01711D0CC57009931B0A0B90837070
:108AC00038460A91D170079595700693537031021C
:108AD0000919089A1202019BD21812045118089120
:108AE00003990902029A8918059A1202049BD21866
:108AF0001204511805913D463A4605E02640AE4025
:108B000032436D1C082D0ED001242146A940034696
:108B1000064602E05B1C042BF0D00CAFFF5C394230
:108B2000F8D0761CF6E70B9B5A7209980699401804
:108B3000079940180A994018059A8018110A401898
:108B4000110C4018110E4018089A8018110A40188C
:108B5000110C4018110E4018563898731021184601
:108B6000FFF7CCFE0DB0F0BDF0B58FB00446FF208E
:108B7000E070A07060700F20C04302900F30207032
:108B8000704818F0D1FA70490868632801D8642049
:108B900008606E4F002038806D4E0190308008E0F4
:108BA0000B99814222D338881030388080B2A128B6
:108BB0006DD206F02FFE3978A02003AA1023FFF70C
:108BC00083FD30802028EED103AD0BA92846FFF7A6
:108BD000B7FEE97B8842E6D128785528E3D15D4885
:108BE000017800290298DBD10846D9E73888A02807
:108BF0004DD8C0B20021019105E006F00BFE398886
:108C0000C8B2A12943D2C1B2A02003AA1023FFF702
:108C10005BFD3080398810313980202837D103AD91
:108C200007A92846FFF78CFEE97B8842E5D1287822
:108C30005528E2D1474800780028029900D1014622
:108C400007988842D9D240490A68962151430B9A25
:108C5000824208D90818904219D30BA90E22204647
:108C6000FFF70BFBC9E78918814210D307A90E2231
:108C70002046FFF702FB0BA80A99818107980B9009
:108C800008980C9009980D9038880190B5E72078E5
:108C9000617809020818A178E278120251180904D3
:108CA0000818401C24D1002001903880A020B02159
:108CB00003AA1023FFF708FD3080202818D103AD48
:108CC0000BA92846FFF73CFEE97B884210D12878A3
:108CD00055280DD11F480078002800D102900B982C
:108CE0000299884204D20BA90E222046FFF7C5FA4A
:108CF0002078617809020818A178E27812025118E8
:108D000009040818401C0CD10020E072A0726072A7
:108D10002072E071A07160712071E070A0706070CD
:108D20002070019838802078617809020818A178AD
:108D3000E2781202511809040818074908603088BF
:108D40000FB0F0BD70110100682F00206E2F0020C1
:108D5000642F0020672F0020742F0020F0B581B011
:108D600000910646214800250570002A2ED01446A1
:108D7000C036631B71190F2008401022101A83425D
:108D800000D303461A480278102A01D0042A1AD1C7
:108D9000C809FE2707405F2F13D80127B843603862
:108DA000C0B29E3282420CD3009A5219C9B2DFB2CD
:108DB0003B46FFF789FC0F490880ED19A542D8D33F
:108DC00004E0082000E004200A49088009480188DE
:108DD0000020042902D0082900D00120034908708E
:108DE000411E8841400001B0F0BDC0467A2F0020EE
:108DF000662F0020782F00200A4A012313700A4AA8
:108E000010700A4A11600A4A00211160042801D139
:108E100005218901102801D11D208101054801800B
:108E20007047C046672F0020662F0020682F002063
:108E3000742F00206C2F0020F0B587B0994D0026CC
:108E40002E80994B1B688B4224D1994C2188202974
:108E500025D1029000920196964C00272760964DEE
:108E6000964E2878062809D806F0D4FC2068401CC5
:108E70002060B042F5D38D48042101802F70904CC2
:108E800020880107029B31D0884820210180854D30
:108E9000019E0BE0012040028449088006E003A8FF
:108EA000FFF762FE20808148802101807F48008892
:108EB0003F2807DD874988420BDC402812D08028F4
:108EC00010D010E004280DD008280AD0202809D09E
:108ED00009E001214A02904204D0C902884201D02F
:108EE00001E002262E80288807B0F0BDA128019E4F
:108EF00000D32780009A012A6A4D1ED1187B0128D1
:108F000056D1DF719F715F711F711F73587B0128EC
:108F100004D1DF729F725F721F725F7303AF3846B6
:108F20001946FFF79CFDF8732088002846D01038BA
:108F3000C1B2A02003AA102344E0002AB6D16148A0
:108F400001780029B2D002701878597809020818FF
:108F50009978DA7812025118090408185A490978E0
:108F6000002901D00F21C943884233D2274603ACE0
:108F700020461946FFF773FDE0733978A0201023CF
:108F80002246FFF7E6FB029A4849088008288DD15F
:108F90003888103038801078517809020818917894
:108FA000D2781202511809040818484908607DE770
:108FB000597B012911D10128A3D0A7E7A02003AA3A
:108FC00010230146FFF7C5FB384908803D4800994A
:108FD00001706BE70120C0025EE73D480078012880
:108FE00012D103AC20461946FFF739FDE073A020EB
:108FF000B02110232246FFF7ACFB2C49088008283B
:10900000E4D133480770E1E7187859780902081865
:109010009978DA7812025118090408182B4909685E
:10902000214A12685118884203D220484021018009
:10903000CCE725490978002901D00F21C94388428E
:109040002DD203AF384619461C46FFF708FDF873CA
:109050001B480178A02010233A46FFF77AFB1349FA
:1090600008800828B2D11649088810300880207876
:10907000617809020818A178E278120251180904EF
:1090800008181249086008490A6815215143FFF77A
:109090005DF800299AD101200D49087096E701205A
:1090A000C00291E7802F0020682F00207E2F002033
:1090B000642F0020842F00207B2F0020818D5B00F7
:1090C0006E2F0020702F0020672F0020742F0020AB
:1090D0007C2F0020FF010000F0B585B00646434C10
:1090E0000027278004921018414A1288904241D2EA
:1090F00001910397404F0020029038603F4C404D53
:109100002078052809D806F085FB3868401C3860AF
:10911000A842F5D3374804210180029820703948CD
:10912000018839480278102A01D0042A32D18819DE
:109130000346C033049C651A0F2404401020001B12
:10914000854200DB0546DC09603C01263002E7B2BF
:109150007F09052F12D3B443E6B29E32B242234CAC
:10916000039F0DD301984218D9B2EBB23046FFF7F6
:10917000F0FA05E01F482021018011E01B4C039FFD
:109180001C49088008280BD1E8B21E4A118808182B
:10919000108005E00120800216490880134C039FCF
:1091A000144800881F2809DD202813D001210A0255
:1091B00090420FD0890288420CD00CE0042809D0DC
:1091C000082808D10F4800880499884201D3022753
:1091D00000E001272780208802210143022902D1D3
:1091E000084900220A8005B0F0BDC046802F00204B
:1091F0006C2F00207E2F0020842F00207B2F00204A
:10920000818D5B00882F0020662F0020F0B585B08F
:10921000044600200190042C6FD20CF0B5F9002810
:1092200001D10CF031FA0020009000BF0098401CE2
:1092300000900CF0A9F903900398002803D0484946
:1092400000988842F2D30398002856D1042145485B
:109250000CF07CF94448454908802101444A515C9E
:109260004900404A505A41490A880121090300F047
:1092700055F902900120049020013D4940184078A2
:10928000002801D100264BE02001394940184078E0
:10929000012802D13548068842E0200134494018AF
:1092A000407802282AD12001401805792901304A46
:1092B000515C49002B4A505A2C490A880121090364
:1092C00000F02CF9064628012A49431828012849AC
:1092D00040180289280140180021C7683046B84765
:1092E00006462801224BC018C2882801C018817880
:1092F000304600F087F8064612E02DE020011C49B8
:1093000040184078032804D02001401840781328E2
:1093100004D1200116494018868801E000200490FD
:109320000498002818D02001124943182001104940
:1093300040180289200140183146C7680298B84792
:10934000019020010A4BC018C2882001C018817802
:10935000019800F057F80190019805B0F0BD0000A9
:1093600050C30000FA00002088130000F400002021
:10937000A81C0200E81C0200F8B505460E4614467B
:109380000020009001211C4801751C48007888438A
:109390001A490870084680780821084317498870E0
:1093A000002088710846007801210843134908709D
:1093B00008460572002717E010480078802108430E
:1093C0000E49087000BF0E48007D0028FBD0002029
:1093D0000B4908750948C0892080A41C0748C18929
:1093E0000098081800907F1CB742E5D331460098DA
:1093F000FEF7ACFE80B2F8BD406100400050044072
:109400004060004010B50346012908D1094CA41A58
:109410009C4202D99C18A0B20BE0064809E0022940
:1094200006D1934202DD9C1AA0B202E0002000E0C7
:10943000184610BDFFFF000010B504460121202092
:1094400001F0FEFF0020324908700121314801750A
:10945000002031490875152017F04EFB2C48807804
:10946000E17808432A4988700846807821780843C3
:10947000274988702078802806D108460079E1794C
:10948000490008432249087121488078E17A08435D
:109490001F498870A078002803D108460079087118
:1094A0000FE0A078012806D119480079602108430F
:1094B0001749087105E016480079802108431449CE
:1094C0000871134880792179084311498871084649
:1094D0008079617908430E498871207AC872607A70
:1094E0008872084600783821884309490870084680
:1094F00000786178C900084305490870A07A0873AC
:1095000008460078012108430149087010BD000099
:10951000005004404061004040600040F8B50446FF
:109520000E461746002E01D100250FE0A64201DCB1
:109530003D460BE00094009C204678430090314665
:109540000098FEF703FE0090009885B22846F8BD0B
:109550000146042904D28A00024BD218508800E048
:1095600000207047342900200146042903D28A00D4
:10957000024B985C00E00020704700003429002076
:10958000FFB587B004460898844203DA0A988068D9
:10959000002802D12448019042E00898001B82B2C2
:1095A0000292002625460A98806800212F463A46F6
:1095B0003346049605910690FEF722FE05460E46B8
:1095C000002328463146029AFEF7EAFD05460E467C
:1095D000304600210A4649405040014302D012481B
:1095E00001901DE003950A98C068039DA84202D32C
:1095F0000020019014E00A98C1680398401A039073
:1096000009990398FEF7A2FD03900398000C00044B
:10961000002802D00448019002E0039880B2019033
:1096200001980BB0F0BD0000FFFF000010B5084826
:10963000007880218843064908700121054801759A
:10964000002005490875152017F056FA10BD0000D6
:10965000005004404061004040600040F8B50546BD
:109660000E4614461F4621462846FEF785FD80B269
:10967000F8BD0000FFB587B006460A98406800288C
:1096800001D1029035E00A980168406808180390FB
:10969000002534460021274603980695049105903D
:1096A00038462946049B059AFEF7AAFD04460D4656
:1096B0000A98406802460023019020462946FEF79A
:1096C0006FFD04460D46002320462946099AFEF701
:1096D00067FD04460D4628460749214000235940AE
:1096E0005840014303D00448C043029001E0A0B2B7
:1096F000029002980BB0F0BD0000FFFF10B5FE48CD
:1097000000688079030017F0DDF907059ED8F5F4AD
:10971000F3F2F100F84800684079030017F0D2F93D
:109720000805138A2A8A468A638A13F025FA0020DC
:10973000F1490968C873F04800684079401CEE4957
:10974000096848717DE0ED494969EB4A1268D27AAF
:10975000885C13F089FAE84800684079401CE649C3
:1097600009684871E44800684079401CE24909688A
:10977000487166E00AF06EF9002810D113F074FA0F
:10978000DD4800684079401CDB4909684871DA48C7
:1097900000684079401CD8490968487105E013F019
:1097A00015FA0020D449096848714AE00AF052F9D4
:1097B000002811D1112013F057FACF4800684079E2
:1097C000401CCD4909684871CB4800684079401C6D
:1097D000C9490968487105E013F0F8F90020C64945
:1097E000096848712DE00AF035F900281BD1C248FC
:1097F0000068C07A401CC0490968C872BE48006849
:10980000C07ABE49097888420DDB0020BA49096850
:10981000C872B94909684862B74800688079401C35
:10982000B5490968887113F0D1F90020B249096877
:10983000487106E013F0CAF90020AF490968487181
:1098400000BF00BF32E3AC480068407C002817D05E
:10985000AA48C068002803D0A848C16819208847D2
:109860000020A54909684862A34800688079401C27
:10987000A1490968887100209F49096848711BE067
:109880009D480068406A282807D29B480068406AC3
:10989000401C9949096848620EE000209649096811
:1098A0004862954800688079401C9349096888712E
:1098B0000020914909684871F8E28F4800684079B2
:1098C000030017F0FFF8080518A42FA44CA480A4E7
:1098D00013F052F9002088490968C8738648006867
:1098E0004079401C84490968487197E0D4E2C7E296
:1098F00030E25DE194E0814949697F4A1268D27A99
:10990000885C13F0B1F97C4800684079401C7A49C2
:1099100009684871784800684079401C76490968B0
:1099200048717BE00AF096F8002811D1012013F06D
:109930009BF9714800684079401C6F49096848717B
:109940006D4800684079401C6B490968487105E022
:1099500013F03CF900206849096848715EE00AF09C
:1099600079F8002828D164490968C97A242251432A
:10997000634A12688918604A1268D27B885C13F0C7
:1099800073F95D480068C07B401C5B490968C87377
:1099900059480068C07B242814D357480068407990
:1099A000401C554909684871534800684079401C7B
:1099B00051490968487105E013F008F900204E4943
:1099C000096848712AE00AF045F8002818D14A4889
:1099D0000068C07A401C48490968C8724648006857
:1099E000C07A4649097888420ADB00204249096862
:1099F000C872414800688079401C3F4909688871F5
:109A000013F0E4F800203C490968487106E013F0BF
:109A1000DDF8002038490968487100BF00BF45E201
:109A2000354800684079030017F04CF80A0614B96D
:109A30002BB948B978B995B913F09EF800202E4992
:109A40000968C8732C4800684079401C2A49096895
:109A50004871ABE029494969274A1268D27A885C83
:109A600013F002F9244800684079401C2249096833
:109A70004871214800684079401C1F4909684871B5
:109A800094E009F0E7FF002811D14A2013F0ECF828
:109A9000194800684079401C174909684871164800
:109AA00000684079401C14490968487105E013F0CA
:109AB0008DF8002010490968487177E009F0CAFF65
:109AC000002824D1FF2013F0CFF80B480068C07B9A
:109AD000401C09490968C87307480068C07B2428EE
:109AE0001BD3054800684079401C03490968487148
:109AF00001480068407905E0E00700204C2F002075
:109B0000DC070020401CEA490968487105E013F0B1
:109B10005DF80020E6490968487147E009F09AFFBE
:109B2000002811D1FF2013F09FF8E1480068407928
:109B3000401CDF4909684871DD4800684079401CD5
:109B4000DB490968487105E013F040F80020D84966
:109B5000096848712AE009F07DFF002818D1D4482F
:109B60000068C07A401CD2490968C872D0480068B1
:109B7000C07AD049097888420ADB0020CC490968BC
:109B8000C872CB4800688079401CC949096888714F
:109B900013F01CF80020C6490968487106E013F06C
:109BA00015F80020C2490968487100BF00BF7DE177
:109BB000BF4800684079030016F084FF0C0715C306
:109BC0002CC349C366C382C39FC312F0D5FF0020D4
:109BD000B7490968C873B64800684079401CB44961
:109BE00009684871B4E0B3494969B14A1268D27A48
:109BF000885C13F039F8AE4800684079401CAC49E5
:109C000009684871AA4800684079401CA849096859
:109C100048719DE009F01EFF002811D1772013F054
:109C200023F8A34800684079401CA149096848719D
:109C30009F4800684079401C9D490968487105E0CB
:109C400012F0C4FF00209A490968487180E009F0C9
:109C500001FF002811D10C2013F006F89448006889
:109C60004079401C924909684871914800684079E0
:109C7000401C8F490968487105E012F0A7FF0020D9
:109C80008B490968487163E009F0E4FE002810D1AF
:109C900012F0EAFF864800684079401C8449096850
:109CA0004871834800684079401C814909684871BF
:109CB00005E012F08BFF00207D490968487147E0FC
:109CC00009F0C8FE002811D1132012F0CDFF78480A
:109CD00000684079401C76490968487174480068FA
:109CE0004079401C72490968487105E012F06EFF26
:109CF00000206F49096848712AE009F0ABFE00288E
:109D000018D16B480068C07A401C69490968C8725C
:109D100067480068C07A6749097888420ADB0020F2
:109D200063490968C872624800688079401C6049CC
:109D30000968887112F04AFF00205D49096848717E
:109D400006E012F043FF002059490968487100BF3E
:109D500000BFABE0564800684079030016F0B2FE41
:109D6000080513872A874787638712F005FF0020BD
:109D70004F490968C8734E4800684079401C4C49F7
:109D8000096848717AE04B494969494A1268D27AB0
:109D9000885C12F069FF464800684079401C4449DD
:109DA00009684871424800684079401C4049096888
:109DB000487163E009F04EFE002811D1492012F0ED
:109DC00053FF3B4800684079401C39490968487195
:109DD000374800684079401C35490968487105E0FA
:109DE00012F0F4FE002032490968487146E009F09B
:109DF00031FE002810D112F037FF2D48006840795D
:109E0000401C2B4909684871294800684079401C6A
:109E100027490968487105E012F0D8FE002024495E
:109E2000096848712AE009F015FE002818D1204879
:109E30000068C07A401C1E490968C8721C48006846
:109E4000C07A1C49097888420ADB00201849096851
:109E5000C872174800688079401C154909688871E4
:109E600012F0B4FE002012490968487106E012F0B1
:109E7000ADFE00200E490968487100BF00BF15E023
:109E800000200B4909688871094909684871062052
:109E900007490968C87009E012F098FE00200449DB
:109EA0000968487102490968887100BF00BF10BD88
:109EB000E00700204C2F002010B56A480068407968
:109EC000030016F0FFFD090610C627C644C6608EC3
:109ED000C60012F051FE634800684079401C614999
:109EE00009684871BCE0604949695E4A1268D27AE3
:109EF000885C12F0B9FE5B4800684079401C594903
:109F000009684871574800684079401C55490968FC
:109F10004871A5E009F09EFD002811D17F2012F0C4
:109F2000A3FE504800684079401C4E4909684871BA
:109F30004C4800684079401C4A490968487105E06E
:109F400012F044FE002047490968487188E009F092
:109F500081FD002810D112F087FE42480068407948
:109F6000401C4049096848713E4800684079401CDF
:109F70003C490968487105E012F028FE0020394983
:109F8000096848716CE009F065FD002822D1354868
:109F90000068C07A401C33490968C87231480068BB
:109FA000C07A3149097888420FDB00202D490968C1
:109FB000C8722C4800684079401C2A4909684871D9
:109FC000002028490968486208E0002025490968FE
:109FD000487103E0002023490968487112F0F6FD3A
:109FE0003EE020480068407C002816D01E48C0682B
:109FF000002803D01C48C16819208847002019494F
:10A0000009684862174909684871164909688871E2
:10A01000052014490968C8701AE012480068406AAF
:10A02000282807D20F480068406A401C0D4909687B
:10A0300048620DE000200B49096848620949096837
:10A040004871084909688871052006490968C8707F
:10A0500006E012F0BBFD002002490968487100BF0C
:10A0600000BF10BDE00700204C2F002010B50024D9
:10A07000F7480068807A01287ED1F5480068C079E9
:10A0800000287AD0F24800688079002804D001289E
:10A0900074D0022873D191E1ED480068007B242838
:10A0A0006ED2EB480068C07901287AD1002475E0AF
:10A0B000E7480068C07A24214843E6490968401807
:10A0C000E3490968097B415CE1480068C07A2422C1
:10A0D0005043E14A12688018DD4A1268127B805CA6
:10A0E000814229D0DA480068C07A24214843DA49FD
:10A0F00009684018D6490968097B415CD448006862
:10A10000C07A24225043D34A12688018D04A126879
:10A11000127B8154CE480068407B242805D3CC486C
:10A120000068007BCA4909684873C9480068007B19
:10A13000C7490968887308E0C5480068407B24283F
:10A1400003D20120C24909688871C1480068007BB8
:10A15000401CBF4909680873BD480068007B24287B
:10A1600008D3BB480068407B242803D20120B849AB
:10A1700009688871B64805E0D3E1CDE169E0BAE14C
:10A1800038E00EE00068007B242804D2B048006864
:10A190008079012800D103E0601CC4B2242C87D34D
:10A1A00056E0002413E0AA480068C07A24214843FE
:10A1B000A94909684018015DA5480068C07A2422B1
:10A1C0005043A44A126880180155601CC4B2242C64
:10A1D000E9D300209E490968487323209C490968F7
:10A1E000887301209A490968887124209849096870
:10A1F00008732DE0002096490968087394480068A8
:10A20000C07A401C92490968C87291480068C07AB7
:10A2100092490978884217DB8D480068007C012844
:10A2200004D102208A490968887106E00020884923
:10A230000968887186490968C871002084490968DD
:10A24000C872834909680874002081490968487107
:10A2500061E17F4800684079030016F033FC08058F
:10A2600013A62AA651A68EA601207949096808746A
:10A2700012F082FC764800684079401C74490968F5
:10A28000487199E075494969714A1268D27A885CC7
:10A2900012F0EAFC6E4800684079401C6C4909687D
:10A2A00048716B4800684079401C694909684871E9
:10A2B00082E009F0CFFB00281BD165490968497B82
:10A2C000491CC8B212F0D0FC61480068407B60496C
:10A2D0000968C8735E4800684079401C5C49096899
:10A2E00048715B4800684079401C594909684871C9
:10A2F00005E012F06BFC00205549096848715BE0ED
:10A3000009F0A8FB00282BD151490968C97A2422F9
:10A310005143504A126889184D4A1268D27B885CB2
:10A3200012F0A2FC4A480068C07B401C48490968FA
:10A33000C87347480068C07B45490968897B8842E3
:10A340001ADD434800684079401C4149096848715A
:10A350003F4800684079401C3D49096848710BE05E
:10A3600012F034FC3A480068407B39490968C873E8
:10A3700000203749096848711EE009F06BFB00288E
:10A380000CD1334909688871242031490968C873A0
:10A390002F49096848732E490968887312F016FC22
:10A3A00000202B490968487106E012F00FFC0020DC
:10A3B00027490968487100BF00BFACE02448006825
:10A3C0004079030016F07EFB08050F8E268E4C8E1A
:10A3D000688E12F0D1FB1E4800684079401C1C4971
:10A3E0000968487185E01D494969194A1268D27A9D
:10A3F000885C12F039FC164800684079401C14490A
:10A4000009684871124800684079401C1049096881
:10A4100048716EE009F01EFB002811D1492012F0AE
:10A4200023FC0B4800684079401C094909684871C1
:10A43000074800684079401C05490968487105E0F3
:10A4400012F0C4FB002002490968487151E0000085
:10A45000E0070020DC070020D80700204C2F002058
:10A4600009F0F8FA002810D112F0FEFB9C480068B1
:10A470004079401C9A4909684871994800684079B8
:10A48000401C97490968487105E012F09FFB0020C5
:10A490009349096848712CE009F0DCFA00281AD1C8
:10A4A0008F480068C07A401C8D490968C8728C4882
:10A4B0000068C07A8B49097888420CDB0020884903
:10A4C0000968C872864909688871854909684871B0
:10A4D00083490968C87112F079FB00208049096836
:10A4E000487106E012F072FB00207D49096848714E
:10A4F00000BF00BF0FE012F069FB00207849096837
:10A500004871774909688871754909680873744901
:10A510000968C87200BFE2E00020714909688872CA
:10A52000DDE06F480068807A0228F4D16C4800684A
:10A53000007A002879D06A4800684079030016F054
:10A54000C1FA0B0711BB25BB41545EBB7590BB0024
:10A5500012F012FB624800684079401C60490968AB
:10A560004871B7E05F494969087812F07DFB5C48A3
:10A5700000684079401C5A49096848715848006889
:10A580004079401C564909684871A3E009F062FA15
:10A59000002810D112F068FB514800684079401C37
:10A5A0004F49096848714E4800684079401C4C4941
:10A5B0000968487105E012F009FB00204849096864
:10A5C000487187E009F046FA002807D1444800683E
:10A5D0004079401C42490968487103E00020404925
:10A5E0000968487112F0F2FA74E012F0C5FA3C48BA
:10A5F00000684079401C3A49096848716AE0394965
:10A6000049690978491CC8B212F02EFB3448006829
:10A610004079401C324909684871314800684079E6
:10A62000401C2F490968487154E054E009F012FABF
:10A6300000280FD112F072FA2949096888700120A8
:10A6400012F0E6FA264800684079401C244909685F
:10A65000487105E012F0BAFA0020214909684871F2
:10A6600038E01F480068807811280CD100201C4970
:10A6700009680872AA201A490968887000201849D8
:10A680000968487011E0164800684078401C144979
:10A6900009684870124800684078032805D309F01B
:10A6A00079FA00200E490968487012F08FFA0020EC
:10A6B0000B49096848710DE012F088FA002008493A
:10A6C00009684871064909684870AA200449096860
:10A6D000887000BF03E0002001490968887210BD3E
:10A6E000E00700204C2F0020F0B505460C4616462A
:10A6F0001F462088482806DA3A462946304605F0A3
:10A70000C3F8012800D0F0BD2088C0002E5020885A
:10A71000401C208000BFF6E710B502469000074BB2
:10A72000C018405C002802D00320C04310BD0120A7
:10A730009300024C1B1958540020F7E7C82A002048
:10A7400070B5002508E06D1C1B48854202D20AF056
:10A75000C7FF01E0002503E00AF016FF0028F2D150
:10A7600000BF022100200AF01DFF032100200AF093
:10A7700019FF052100200AF015FF072100200AF02B
:10A7800011FF002408E00020A1000C4A5054A10051
:10A7900089184880601CC4B2042CF4D301200849F5
:10A7A000087000204870052088700020C870054897
:10A7B0000549088070BD000050C300003429002006
:10A7C000F600002088130000F4000020F8B58D4842
:10A7D0000078030016F076F9060405163D5EFDFCD0
:10A7E0000EE10AF051FF00208649C8704870084603
:10A7F0008078002802D10320087002E002208149FD
:10A800000870FDE07F488078002804D07D4880787B
:10A81000401E7C4988700AF0B7FE00280BD10AF070
:10A8200033FF00207749C8700846807800280FD190
:10A83000032008700CE07348C078401C7149C87050
:10A840000846C078052803D3052008700AF048FFA1
:10A85000D6E00AF099FE00280ED104216A480AF0D9
:10A8600075FE00206749C8704870684868490880CC
:10A870000420644908700CE06248C078401C6149BB
:10A88000C8700846C078052803D3052008700AF070
:10A8900027FFB5E05B49497809015E4A515C4900F0
:10A8A000594A505A5A490A8801210903FEF736FECF
:10A8B00000900125534840780001564940184078DF
:10A8C000002801D100243CE04E4840780001514965
:10A8D00040184078012802D14D48048831E04948A9
:10A8E000407800014B4940184078022812D1454970
:10A8F00049780901474A89180879FEF729FE044674
:10A90000404949780901434A89180879FEF72CFE25
:10A91000054616E03B48407800013E494018407823
:10A92000032806D0374840780001401840781328A3
:10A9300006D134484078000136494018848800E048
:10A940000025002D2FD02F484078000132494318B0
:10A950002C48407800012F49401802892948407846
:10A96000000140182146C7680098B84706462548A8
:10A9700040780001274BC018C28822484078000167
:10A98000C01881783046FEF73DFD06461D484078E8
:10A99000800022494018468001201A4949788900E0
:10A9A0001E4A50540AE000201649497889001B4A83
:10A9B00089184880134949788900505411484078D3
:10A9C000401C1049487008464078042809D301E02B
:10A9D00013E007E00AF058FE00200A4948700320FF
:10A9E00008700DE00AF0D0FD002803D101200549D0
:10A9F000087001E00AF074FE02E0FFF7A1FE00BF5C
:10AA000000BFF8BDF6000020FA0000208813000007
:10AA1000F4000020A81C0200E81C020034290020D9
:10AA200010B50AF07BFD002405E00020A100074AD4
:10AA30005054601CC4B2042CF7D3002004490870A1
:10AA40000520887003480449088010BD342900207F
:10AA5000F600002088130000F400002070B50446C2
:10AA6000002000F0AFF8002000F0DAF8002000F03D
:10AA70009BF8002000F0C4F8002000F087F80020C8
:10AA800000F0AEF800BF012000F08EF8012000F0C9
:10AA9000B7F8002521E0002000F086F8002000F043
:10AAA000AFF880202040002806D0012000F08AF86E
:10AAB000012000F0B5F805E0002000F083F8002048
:10AAC00000F0AEF800BF012000F06EF8012000F0A9
:10AAD00097F86006040E681CC5B2082DDBDB012068
:10AAE00000F054F8012000F07BF870BD70B504460A
:10AAF0000D46012000F066F8012000F091F80020DA
:10AB000000F052F8002000F07BF8002000F03EF842
:10AB1000002000F065F800BF012000F045F801209A
:10AB200000F06EF8002628E0002000F03DF800203C
:10AB300000F066F880202040002803D0012000F0BB
:10AB400041F802E0002000F03DF880202840002875
:10AB500003D0012000F064F802E0002000F060F86B
:10AB600000BF012000F020F8012000F049F8600645
:10AB7000040E6806050E701CC6B2082ED4DB012038
:10AB800000F004F8012000F02BF870BD10B5044669
:10AB9000002C04D0012103200AF0A0FE03E00021D4
:10ABA00003200AF09BFE10BD10B50446002C04D013
:10ABB000012104200AF092FE03E0002104200AF0A3
:10ABC0008DFE10BD10B50446002C04D001210220DA
:10ABD0000AF084FE03E0002102200AF07FFE10BD8F
:10ABE00010B50446002C04D0012104480AF076FE7A
:10ABF00003E0002101480AF071FE10BD01070000CA
:10AC000010B50446002C05D00121072000020AF0EF
:10AC100065FE04E00021072000020AF05FFE10BD7F
:10AC200010B50446002C04D0012104480AF056FE59
:10AC300003E0002101480AF051FE10BD02070000A8
:10AC400010B5F920FFF70AFF3221424805F05EFEF9
:10AC50008820FFF703FF9020FFF700FF9820FFF701
:10AC6000FDFE08210846FFF741FFE820FFF7F6FE4A
:10AC700012210846FFF73AFFA020FFF7EFFE7021F0
:10AC80000846FFF733FFA820FFF7E8FE70210846CB
:10AC9000FFF72CFFB020FFF7E1FE70210846FFF719
:10ACA00025FFB820FFF7DAFE00210846FFF71EFF58
:10ACB000C020FFF7D3FE00210846FFF717FFC8208A
:10ACC000FFF7CCFE00210846FFF710FFD020FFF76A
:10ACD000C5FE2F210846FFF709FFD820FFF7BEFE6B
:10ACE0002F210846FFF702FFE020FFF7B7FE2F21D4
:10ACF0000846FFF7FBFE4020FFF7B0FE00210846A4
:10AD0000FFF7F4FE0A20FFF7A9FE002405E000216A
:10AD10000846FFF7EBFE601CC4B25A2CF7DB002498
:10AD20000AE000200C4908550C4908550C49085503
:10AD30000C490855601CC4B25A2CF2DB8120FFF785
:10AD40008DFE0020084908708870C870087148702E
:10AD500010BD0000204E00005C260020B62600201A
:10AD6000102700206A270020CC00002010B580208A
:10AD7000FFF774FE10BD0000002004490870012098
:10AD8000034908700020487070470000D10000207F
:10AD9000CC00002010B54848007800287AD04648FA
:10ADA0008078030015F08EFE0604434A535A687EED
:10ADB000414800794149085C3F490979404A515C62
:10ADC000884209D13C4800793E49085C3A490979F2
:10ADD0003D4A515C88421BD0374800793749085CAE
:10ADE00035490979364A5054334800793549085C69
:10ADF00031490979344A50542F48C078002803D08B
:10AE000004202D49887011E001202B4988700DE045
:10AE100000202949C87008460079401C087108467E
:10AE200000795A2802DB00200871087041E04020B8
:10AE3000FFF714FE0220204988703AE01E4A11797B
:10AE40001079FFF753FE03201B49887031E00A2078
:10AE5000FFF704FE0420184988702AE0164A127988
:10AE6000194B995C144A1279154B985CFFF73EFE1A
:10AE70000520114988701CE00F480079401C0E49DC
:10AE80000871084600795A2805DB0020087108700F
:10AE9000C87003E00EE001200749C8700020064991
:10AEA000887006E00020044908708870C870087136
:10AEB00000BF00BF10BD0000CC0000205C260020B9
:10AEC000B6260020102700206A27002010B512F0B7
:10AED0008BFA01281ED101F08DFD1149884212D351
:10AEE000072009F0E1FB002806D04B22D200002108
:10AEF000012013F0A7FF12E07D22D20000210120E3
:10AF000013F0A0FF0BE07D22D2000021012013F0FE
:10AF100099FF04E000221146012013F093FF10BDB9
:10AF2000B80B000000200349087248708870486020
:10AF300070470000600A002058221152704710B577
:10AF400004460121022000F07BFA0021022000F0DB
:10AF500077FA10BD014600205322525C10231A409C
:10AF6000002A08D05322525C0C231A409210032A64
:10AF700018D1032016E05422525A0123DB031A4051
:10AF8000002A0ED05322525C0C231A409210032A3E
:10AF900005D05322525C9207920F032A01D102205E
:10AFA00000E0012070470246002058239B5A0B40C6
:10AFB000002B01D0012000E0002070470146002254
:10AFC0006020405AFF231B0218400005020F1001A9
:10AFD000014BC018704700000055044010B5002A0E
:10AFE0000AD056231B5A0C022343562423525623BD
:10AFF0001B5A8B43235209E056231B5A0C02A343CE
:10B000005624235256231B5A0B43235210BD0000D3
:10B01000F8B504460D46012700263448844203D182
:10B020000121022000F00CFA2878401EA070208830
:10B03000FF21013108432080208840084000208003
:10B04000A878401EC1B25A20015568790007000C4B
:10B05000E97909020843A97908435C210853288942
:10B0600081B240200153A868C000C10C42200153A6
:10B07000A88981B244200153E868C000C10C462071
:10B080000153288A81B2482001532869C000C10CAD
:10B090004A200153A88A81B24C2001536869C0003C
:10B0A000C10C4E2001535020005B2979090208434E
:10B0B000502108535020005B2979884350210853C0
:10B0C00000E0761C5020005B4007400F2979884241
:10B0D00002D007488642F4D15020005B4007400F61
:10B0E0002979884200D000273846F8BD0054044032
:10B0F000FFFF000030B5034600201C898C4209DDAB
:10B10000082A05D218244C431D682C19A05C02E0C3
:10B11000002000E0002030BD10B5024613898B42AC
:10B1200005DD18234B431468E318987C00E00020E9
:10B1300010BD0146FF22C889C007C00F00280AD0F1
:10B140000120C88100E0521EC889C007C00F002836
:10B1500001D0002AF7D1C889C007C00F00280FD13D
:10B160000220C8810420C881487A40084000487203
:10B17000487A38239843487200204872012070476B
:10B180000020FCE70246507A012318435072507A9F
:10B190000B78DB0018435072087A012808D18888A0
:10B1A00050814868000C0123DB031843908108E0BC
:10B1B000087A002805D15081486880001A4B184051
:10B1C0009081487A012804D1507A40231843507264
:10B1D00006E0487A002803D1507A40239843507201
:10B1E0000878002811D1C87A1072087B1070487B4B
:10B1F0005070887B9070CB7BD370087C10714B7C37
:10B200005371887C9071CB7CD371887A002803D0ED
:10B210000120C002D08101E00820D081FF20013050
:10B22000D081012070470000FC1F0000002904D0DD
:10B23000427A80231A43427203E0427A80239A437F
:10B240004272704730B5024600200F4B5024A45A7A
:10B250000D022C435025AC525024A45A8C43AC52BE
:10B2600000E05B1E5024A45A6407640F8C4201D096
:10B27000002BF6D15024A45A6407640F002C01D08F
:10B28000002000E0012030BDFFFF0000827A802313
:10B290001A40802A00D081727047000070B50446C1
:10B2A00000250023002D02D0012660200653042033
:10B2B000C88188890126F6033040002808D0012083
:10B2C00010728889C004C0084E893043506006E07F
:10B2D0000020107288890F4E304080105060087A2C
:10B2E000D072002304E0CE5C10460C30C6545B1CC8
:10B2F000D07A9842F7DCC88904263040002804D16F
:10B30000C889F6023040002801D0002070BDD07AF4
:10B31000FCE70000FC1F00000020024908800249F1
:10B3200008807047780000207A000020027C80238B
:10B330001A40802A00D00174704710B50246FF23DE
:10B34000D089C007C00F002802D00120D0815B1E29
:10B35000D089C007C00F002801D0002010BD507A4E
:10B36000012420435072507A3824A0435072C87A86
:10B370001072487A00280FD1087B1070487B5070FB
:10B38000887B9070CC7BD470087C10714C7C54719D
:10B39000887C9071CC7CD471FF200130D08140003A
:10B3A000D081107ADAE70000FFB581B004460D467F
:10B3B0000020012C03D140262E43304306E0002C10
:10B3C00000D103E0022C01D1C0263043012A06D16E
:10B3D000049E760010273E430643F0B206E0002AA2
:10B3E00000D103E0022A01D130263043134E3070E1
:10B3F00076788027BE43114F7E70012C08D1FF2143
:10B4000000BF0E4EB3781E460E4033468B42F8D135
:10B410000A4E76784027BE43084F7E70012A0BD132
:10B420000026009603E000BF009E761C0096FF27D2
:10B430006937009EBE42F6D905B0F0BD0004024057
:10B44000002905D0054A12780243044B1A7004E023
:10B45000024A12788243014B1A707047200402405E
:10B46000002905D0054A927E0243044B9A7604E0F7
:10B47000024A927E8243014B9A767047000802404E
:10B4800070B5034614460020002B01D1C0B202E083
:10B4900005468035E8B2012902D1051DE8B206E073
:10B4A000022903D105460835E8B200E0C0B2012CFC
:10B4B00002D1851CE8B200E0C0B2084DA870AD789A
:10B4C00001263543054EB570002201E000BF521C35
:10B4D0007D252D01AA42F9D970BD0000000C024063
:10B4E00070B500242448007920210840002801D0AC
:10B4F000224D3FE000F046F80546214800788021C3
:10B500000840002836D01E4880780840002801D026
:10B510001A4D02E000F036F8054619488078000719
:10B52000840F022C01DBAD0804E0012C01D16D0871
:10B5300000E000BF124880788007C00F002801D0CB
:10B540002D0101E00C2045430D4800784007840F91
:10B55000002C02D1601CC4B207E0032C03D1601C94
:10B560004006040E01E06006040E21462846FCF762
:10B57000EDFD0546284670BD0004024000127A0029
:10B58000000C024000B5C0229178F82211401C4AFC
:10B5900012781143EA2923D00ADC0A46E03A130064
:10B5A00015F090FA0A181C20242A2A2A2A161A2A88
:10B5B000ED291FD004DCEB2916D0EC291CD117E0B3
:10B5C000F02903D0F82917D10E4817E00E4815E0EE
:10B5D0000E4813E00E4811E00E480FE00E480DE053
:10B5E0000E480BE00E4809E00E4807E00E4805E063
:10B5F0000E4803E00E4801E00D4800BF00BF00BD4B
:10B60000201C02400090D003006CDC020048E801DE
:10B6100000366E010024F400001BB70000127A000F
:10B62000808D5B0000093D00C0C62D0080841E0097
:10B6300040420F0070B586B0044600250026206801
:10B640000290A1796846C173617941730021017349
:10B65000017100BF05E020460830415D04A8415556
:10B660006D1C6846C07BA842F5D80B22D201029916
:10B67000881A914237D007DC2C48081A1FD02321A2
:10B680000901401A48D113E0FF386F38002802D072
:10B69000012841D105E001A92548FFF74EFE0646E5
:10B6A0003BE001A922484030FFF747FE064634E060
:10B6B00001A91F485030FFF740FE06462DE001A9C2
:10B6C0001B482030FFF739FE06461A480088072835
:10B6D00005DA18480088401C1649088002E000205E
:10B6E0001449088019E005F09BFD002813D012488A
:10B6F00001780078401C104A1070022906DC01A96C
:10B700000B486030FFF719FE064604E000200A49A6
:10B7100008700A49087000E000BF00BF002E02D187
:10B72000012006B070BD0020FBE7000020020000F1
:10B73000805504407A00002076000020E8000020B8
:10B7400010B5A8211348FCF7B1FD12481249086052
:10B7500012484860072008810020887207220F499C
:10B760000D4800F0A9FA00210B48FFF78FFDA0213A
:10B770000B48FCF79BFD0A480A4948600A4B052222
:10B780000A49084800F015FC00210648FFF7CEFDE5
:10B7900010BD00008008002060080020C4180200CE
:10B7A000280900206C08002035B600003818020077
:10B7B0000C4A127812060B4B5B781B041A43094B98
:10B7C0009B781B021A43074BDB781A43104642084A
:10B7D0004240D20083085A401146034A5140034A6E
:10B7E0001160704723070020010200002807002095
:10B7F000F8B504460F46A07A4006400E002874D1E2
:10B800000025ACE01820684321680818407C012816
:10B810003CD10121182068432268101801740026C9
:10B820000CE018206843216808180830815D182052
:10B830006843226810188155701CC6B2082EF0D3D8
:10B8400000211820684322681018017418206843EA
:10B85000226810184174182068432268101841614A
:10B86000182068432268101881742C20684361688E
:10B870000818406A002809D018236B432268D018A2
:10B880002C236B436268D218516A8847182068439A
:10B89000216808184069FF21C94388425DD81820F3
:10B8A0006843216808184069C11918206843226854
:10B8B00010184161182068432168081841692C203C
:10B8C0006843626810188069814246D31820684333
:10B8D00021680818807C55283FD0552118206843DE
:10B8E000226810188174002624E03CE01820684388
:10B8F00021680818805D2C21694362685118103155
:10B90000895D08401821694322685118885518201C
:10B91000684321680818805D2C21694362685118CA
:10B920000831895D084318216943226851188855F8
:10B93000701CC6B2082ED9D32C2068436168081841
:10B94000806A002809D018236B432268D0182C2362
:10B950006B436268D218916A8847681C85B2208957
:10B96000A84200DD4EE7F8BD01200149087070478C
:10B970008C00002010B50446002015F007FC0228BA
:10B980004DD1FFF7C9FC2D480078002802D10120D5
:10B990002A49087029480078012823D1274840788F
:10B9A000401C2649487021465A20FCF7CFFB23490A
:10B9B0004978884241D8002020494870084680785C
:10B9C000401C8870084680780A2803D300208870BD
:10B9D00002200870FFF7A0FC00F068F8002015F0C6
:10B9E00005FC2AE015480078022826D11348407843
:10B9F000401C1249487021467D20C000FCF7A6FB80
:10BA00000E494978884218D800200C494870FFF741
:10BA100083FC00F04BF8002015F0E8FB0DE0074830
:10BA2000C078401C0549C8700846C078042804DB6B
:10BA30000020C87008704870887010BD7200002027
:10BA400000B587B0002168460171042141710C489E
:10BA50000290411003910B49049105910A48069008
:10BA6000FFF76EFE01A815F025FC00F059FB00F071
:10BA700033F80021054809F031FF07B000BD000090
:10BA8000FFFF1F00FFFFFF1F41BD00000205000078
:10BA900030B5034600201C898C4204D94D015C68F6
:10BAA0006419626000E0022030BD000010B500247F
:10BAB00000BF09E01C206043054940182146826808
:10BAC0000448FFF7E5FF641C052CF3D310BD00000C
:10BAD000381802006C08002010B5FF2002307249AF
:10BAE0004860002008720120087000204872012080
:10BAF00088726E48FFF71DFB6B496C48FFF742FBED
:10BB000001216A48FFF792FB6948674948600020B5
:10BB10000872012008700020487201208872634872
:10BB20001030FFF706FB604960481030FFF72AFB32
:10BB300001215E481030FFF779FB5D48401E5A49ED
:10BB4000486000200872012008700020487201201F
:10BB5000887256485030FFF7ECFA5349534850303A
:10BB6000FFF710FB012151485030FFF75FFB5048B1
:10BB7000C1384D494860002008720120087000203B
:10BB800048720120887249484030FFF7D2FA46498E
:10BB900046484030FFF7F6FA012144484030FFF7AD
:10BBA00045FBFF2012304049486000200872012008
:10BBB000087000204872012088723C486030FFF70E
:10BBC000B8FA394939486030FFF7DCFA01213748C3
:10BBD0006030FFF72BFBFF20213033494860002005
:10BBE00008720120087000204872012088722F48D6
:10BBF000A030FFF79EFA2C492C48A030FFF7C2FA7C
:10BC000001212A48A030FFF711FB29488F38264927
:10BC1000486000200872012008700020487201204E
:10BC200088722248E030FFF784FA1F491F48E0304D
:10BC3000FFF7A8FA01211D48E030FFF7F7FA1D4889
:10BC400019494860002008720120087000204872DD
:10BC50000120887215482030FFF76BFA124913480B
:10BC60002030FFF78FFA012110482030FFF7DEFA6D
:10BC70001048CB300C494860002008720120087041
:10BC8000002048720120887208483030FFF751FACE
:10BC9000054906483030FFF775FA01210348303076
:10BCA000FFF7C4FA10BD00008C2A00201055044094
:10BCB0000204000014070000F0B50B461446436070
:10BCC0000481002136E0002216E02C254D43466811
:10BCD0007519AD5C18274F430668F619B5542C2525
:10BCE0004D4346687519AD5C18274F430668F61931
:10BCF0000836B554551CEAB2082AE6D300251827A1
:10BD00004F430668F619357418274F430668F6192D
:10BD1000757418274F430668F619B57418274F43F2
:10BD20000668F619F57418274F430668F619756109
:10BD30004D1CA9B205898D42C5DC00258572F0BD78
:10BD400070B50446606800F0F1FD0546E27A2346CE
:10BD50000C332946094800F0B1FD09496068884262
:10BD600004D00749CB396068884206D1E17AA288BD
:10BD700090B222460C3203F0C7F870BD6008002074
:10BD8000DF070000F8B5054600262C46002C29D018
:10BD900000BF03E00020A055701CC6B2082EF9D3E6
:10BDA00004F0ECFFC00008210840074620788843D3
:10BDB00038432070E079E02188430B490988490124
:10BDC000E02211400843E07104F0D8FF012801D1BE
:10BDD000082000E00020C706FF0EE079400940017E
:10BDE0003843E071F8BD00007A000020F8B5054640
:10BDF00000260027002000902C46002C5BD000BFBE
:10BE000003E00020A055701CC6B2082EF9D305F03F
:10BE1000B3F800280DD005F0F7F9022809D1062162
:10BE20002548FFF779F9552803D005F09FF8002839
:10BE300003D100202070607011E005F0B3F892305B
:10BE40007D21C900884204D805F0ACF8923087B251
:10BE500001E07D27FF003804000E2070677005F0B8
:10BE60008FF900280DD005F0D5F9022809D1062157
:10BE70001148FFF751F9552803D005F07BF9002848
:10BE800003D10020A070E07015E005F08FF992302A
:10BE90007D21C900884205D805F088F9923080B22A
:10BEA000009002E07D20C000009000980004000E89
:10BEB000A0700098E070F8BD6008002070B50546DD
:10BEC00000262C46002C24D000BF03E00020A05503
:10BED000701CC6B2082EF9D305F0A2F901280AD1C8
:10BEE00031202070012060705920A0700820E0707F
:10BEF000002020710DE005F093F9022809D13120CE
:10BF00002070012060705920A0700820E07001208E
:10BF1000207170BDFEB5054600260020019001F09D
:10BF20004DFD074604F05AFF0A210090FCF724F962
:10BF300080B201902C46002C18D000BF03E00020F6
:10BF4000A055701CC6B2082EF9D33802000E6071DD
:10BF50003804000EA071E77105F03AF8FF2802DD01
:10BF6000FF20A07002E005F033F8A070FEBDFEB522
:10BF70000546002600200190002704F025FD6421DD
:10BF80000090FCF7F9F880B20190002001F038FD34
:10BF900087B22C46002C0BD000BF03E00020A05538
:10BFA000701CC6B2082EF9D33804000EA070E770DA
:10BFB000FEBDFFB581B004460F46002500260020D7
:10BFC00000902760039820810498E060002020748E
:10BFD00000BF9DE01C206843216808586A01616821
:10BFE00088501C2068432168081880686A016168CD
:10BFF000891848601C2068432168081840686A0155
:10C000006168891888601C20684321680818C06826
:10C010006A0161688918C8601C2068432168081893
:10C02000007C6A016168891808741C2068432168D3
:10C030000818407C6A016168891848741C206843AC
:10C0400021680818807C6A016168891888831C202F
:10C05000684321680818C07C6A016168891888747F
:10C0600000206A0161688918C8741C20684321682F
:10C0700008184068002813D01C206843216808185D
:10C08000C07C002805D1401E6A0161688918C883F8
:10C090001AE00020C0436A0161688918C88313E070
:10C0A0001C20684321680818C07C002805D00020A7
:10C0B0006A0161688918C88306E000206A01616826
:10C0C0008918C88301200090002607E000216A013A
:10C0D0006068801814308155701CC6B269016068B0
:10C0E0004018808BB042F1DC1C206843216808189E
:10C0F000406900280AD06B016268D21810461430DB
:10C100001C236B432268D21851698847681CC5B24A
:10C110002089A84200DD5DE7009805B0F0BD000071
:10C1200000B58BB068480790002108A801706846E8
:10C13000017608A84170002064498872082108A887
:10C14000C170002004E0002209A90A54411CC8B2B1
:10C1500008A9C9788142F6DC5D48FEF7EAFF06A926
:10C160005B48FFF70FF85848401C0790002108A8CB
:10C1700001706846017608A8417000205349887212
:10C18000082108A8C170002004E0002209A90A546F
:10C19000411CC8B208A9C9788142F6DC4C4840303D
:10C1A000FEF7C7FF06A94A484030FEF7EBFF4520DF
:10C1B00000010790002108A801706846017608A8D0
:10C1C0004170002041498872082108A8C1700020F0
:10C1D00004E0002209A90A54411CC8B208A9C97880
:10C1E0008142F6DC3A485030FEF7A3FF06A93848F2
:10C1F0005030FEF7C7FF112040010790002108A82A
:10C2000001706846017608A8417000202F498872A5
:10C21000082108A8C170002004E0002209A90A54DE
:10C22000411CC8B208A9C9788142F6DC28482030F0
:10C23000FEF77FFF06A926482030FEF7A3FF0B205C
:10C24000C0010790002108A801706846017608A87F
:10C25000417000201D498872082108A8C170002083
:10C2600004E0002209A90A54411CC8B208A9C978EF
:10C270008142F6DC16486030FEF75BFF06A91448E1
:10C280006030FEF77FFF1048A6300290002168461C
:10C2900001730171417381730821C173002004E0AF
:10C2A000002204A90A54411CC8B26946C97B8142D4
:10C2B000F6DC07481030FEF73CFF01A904481030B7
:10C2C000FEF760FF0BB000BDEE0600008C2A0020D8
:10C2D00080550440F0B585B004460F460025002681
:10C2E000207C4006400E55287ED100BF76E16901D2
:10C2F00060684018807C002877D169016068401828
:10C3000040686A01616889188968884209D26901B0
:10C31000606840184068C0196A01616889184860FF
:10C320005AE1690160684018C068AF49884208D87E
:10C33000690160684018C068401C6A01616889181A
:10C34000C860690160684018C07C002821D10026BF
:10C3500007E000216A016068801814308155701C64
:10C36000C6B2690160684018808BB042F1DC1C20C5
:10C37000684321680818406900280AD06B01626888
:10C38000D218104614301C236B432268D21851690E
:10C3900088476901606840580090690160684018EA
:10C3A000017C684601710021417169016068401893
:10C3B000017F68468171690160684018417C684668
:10C3C000C171002608E06901606840181430815D81
:10C3D00002A88155701CC6B2690160684018808B44
:10C3E000B042F0DCE06801E0FCE01DE0002806D08F
:10C3F0006846E16888476A0161688918C8746901FC
:10C4000060684018C07C002804D16A0161688918FE
:10C410004860E1E06901606840184068C01B6A013B
:10C42000616889184860D7E06901606840188068D1
:10C430000028EED0690160684018C08B0028E8D061
:10C44000690160684018C08B6A0161688918C96811
:10C45000884207D1690160684018C08B6249C943AE
:10C4600088427DD169016068401840686A0161684E
:10C4700089188968884209D2690160684018406853
:10C48000C0196A01616889184860A5E000206A0146
:10C49000616889184860690160684018C06852493D
:10C4A000884208D8690160684018C068401C6A0169
:10C4B00061688918C860002607E000216A01606889
:10C4C000801814308155701CC6B26901606840182C
:10C4D000808BB042F1DC1C20684321680818406959
:10C4E00000280AD06B016268D218104614301C2351
:10C4F0006B432268D21851698847690160684058C7
:10C500000090690160684018017C68460171002153
:10C510004171690160684018017F68468171690155
:10C5200060684018417C6846C171002608E06901D6
:10C53000606840181430815D02A88155701CC6B235
:10C54000690160684018808BB042F0DCE068002828
:10C5500008D06846E16888476A016168891800E088
:10C5600015E0C874690160684018C07C002804D1D7
:10C570006A016168891848602EE0690160684018A6
:10C580004068C01B6A0161688918486024E01C206B
:10C59000684321680818406800280FD00020C04375
:10C5A0006A0161688918C8831C20684321680818DB
:10C5B00040686A0161688918886008E000206A01A3
:10C5C00061688918C8836A016168891888600020D9
:10C5D0006A0161688918C860681CC5B22089A842D0
:10C5E00000DD84E605B0F0BD0000FFFF7CB500BFB4
:10C5F00019212C480078FBF7A9FD04462A4860431E
:10C600002A4A8118002201200DF0C6F920460A228C
:10C6100050436430001981B2002201200FF02EFA3D
:10C6200001200A2262431219D1B20A22624312196E
:10C630000090D0B201231A4609F064FCFF220721C2
:10C64000002007F09FF80120009001900B2060432C
:10C6500082B20B20604381B2002301200EF02AFF3A
:10C660006F20604381B201200FF0AEFC10486043A0
:10C670000246032101200BF009FF002505E00121FE
:10C6800028460BF03DFE681CC5B20F2DF7DB214696
:10C690000B2251436431C8B20FF000FF0FF0E8FEE7
:10C6A0007CBD00006F000020672B0000A086010009
:10C6B000FCB10100002005490870054908700549D2
:10C6C000087005490870054908707047700000201F
:10C6D000710000206F0000206E0000206D0000201F
:10C6E000F0B589B000BF00BF00BF00BF00BF00BFF2
:10C6F00000BF00BF00BF00BF5D4800783C2805DADE
:10C700005B480078401C5A49087002E03C205849B8
:10C710000870574800781D2805DC56480078401CF2
:10C72000544908700BE053480078002802D1514961
:10C73000087004E04F480078401E4E4908700321FD
:10C740004C480078FBF718FD4B49484303900521FE
:10C7500048480078FBF7FAFC044603214548007876
:10C76000FBF70AFD0B214843643080B20690414933
:10C7700009788A0088180621FBF7FEFCFF21F531B5
:10C78000484380B2079003213A480078FBF7F4FC55
:10C790000B214843643080B208900321354800786B
:10C7A000FBF7EAFC3549484335494018049003211A
:10C7B00030480078FBF7E0FC0B2106464E4303218E
:10C7C0002C480078FBF7D8FC0B2107464F43032188
:10C7D00028480078FBF7D0FC6F21484380B20590D1
:10C7E00003210120039A0BF051FEE1B201200BF06E
:10C7F00019FCE1B201231846069A09F05DFEFF21FB
:10C80000F5310798FBF7B8FCC0B201460290012051
:10C810000AF034FB0022012008990FF02FF90022C2
:10C82000012004990DF0B8F8012005990FF0CCFB18
:10C830000120F9B20090F0B201231A46029009F0EB
:10C8400061FBFF220721002006F09CFF032109481D
:10C850000078FBF791FC0B21484385B20120009042
:10C8600000232A46294601900EF024FE09B0F0BDAF
:10C870007100002070000020FCB10100672B000057
:10C88000A0860100002000BF06E00021044A1154E8
:10C89000044A1154411CC8B25A28F6DB7047000004
:10C8A0005C260020102700200348007A002801D1D0
:10C8B0000149487070470000600A0020FFB581B050
:10C8C00004460F463D462089A8422DDD18206843C6
:10C8D00021680818007C002826D1002609E0049869
:10C8E000815D182068432268101808308155701C3B
:10C8F000C6B2082EF3D3012118206843226810180D
:10C9000041742C20684361680818006A00280BD025
:10C9100018236B432268D218104608302C236B432F
:10C920006268D218116A884705B0F0BD0146072039
:10C93000124BCA1A994211D008DCCA1FFA3A002ACF
:10C9400014D0102A0CD01F2A14D10DE0322A0FD097
:10C95000C02A07D0C12A0DD100200DE001200BE034
:10C96000022009E0032007E0042005E0052003E0A1
:10C97000062001E0072000BF00BF70474103000010
:10C9800010B504467D21C90061430846322103F0F9
:10C99000BDFF10BDFF200B4908700020C0430A49AD
:10C9A00008800A490880FF20094908700949087071
:10C9B00009490870002009490860094908600949C7
:10C9C00008607047540000205600002058000020E6
:10C9D0005A0000205B0000205C000020480000207E
:10C9E0004C00002050000020014800687047000003
:10C9F0004C000020014800687047000048000020FB
:10CA000010B5054909886522514308466421FBF7A2
:10CA1000B3FB80B210BD0000560000200148007832
:10CA2000704700005B00002001480078704700005C
:10CA30005400002010B510F0D7FC01282CD100F0D4
:10CA400063F8012000F066F803F0C4FF044600F02C
:10CA500043F804F0A1F9044600F04AF804F002FC9F
:10CA6000012805D100F03EF8012000F047F805E06C
:10CA7000002000F037F8002000F040F800201349B3
:10CA8000086013480068134988421ED210480068A5
:10CA9000801C0F49086018E000200D4908600B4811
:10CAA00000680C49884204D208480068801C074985
:10CAB0000860002000F028F8012000F02BF800208A
:10CAC00000F00AF8002000F013F810BD4C00002020
:10CAD00048000020FFFFFF7F0149088070470000E9
:10CAE0005600002001490870704700005B000020DC
:10CAF0000149088070470000580000200149087073
:10CB0000704700005C000020014908707047000079
:10CB10005400002001490870704700005A000020AE
:10CB20000021014A11717047006000400022014954
:10CB30004A75704700600040002201494A767047FC
:10CB4000006000400021014A1172704700600040FF
:10CB50000021014A11737047006000400021014A22
:10CB600011747047006000400021014A1175704740
:10CB7000006000400021014A1176704700600040CB
:10CB8000002201494A7370470060004000220149B9
:10CB90004A7470470060004010B51C4C1C49206866
:10CBA00088421ED106221B49201DFBF78AFB002864
:10CBB00017D11222184920460A30FBF782FB0028C1
:10CBC0000FD10622154920461C30FBF77AFB0028BE
:10CBD00007D10622124920462230FBF772FB0028BB
:10CBE0000DD000F031FF0A480E490860074814F0E4
:10CBF0002EFC0C4A2C21054814F054FC04E02C2295
:10CC000021460848FBF739FB10BD00000002500028
:10CC10007AA7A55A390700203F07002033070020D4
:10CC20002D070020982E0020002008490870084990
:10CC3000087001200749087000200749087007485C
:10CC40000749086000200749087070471B0700204B
:10CC50001A0700201D0700202207002025060000DB
:10CC6000540700202C07002070B5044600BF912017
:10CC7000604305460A212846FBF768FA0546284620
:10CC800070BD000070B5A8B0054600240026A021A4
:10CC90006846FBF70BFB00F047FD1E490A681421AC
:10CCA0006943505000211B48026814206843101843
:10CCB00041601848026814206843101881601548C4
:10CCC0004068002824D000BF17E06006060E282E1A
:10CCD00000D316E00F480168142060430858B100E3
:10CCE0006A4650500B480168142060430818416898
:10CCF000701C80001150601CC4B20648007AA0422B
:10CD0000E3DC00BF6200034869464368022098479D
:10CD100028B070BD142F002030B5A9B00024002524
:10CD2000A02101A8FBF7C2FA00BF25E06006050EAE
:10CD300000F0FAFC1F490A68142161435050002199
:10CD40001C480268142060431018416019480268AA
:10CD50001420604310188160282D0BD215480168FB
:10CD6000142060430858A90001AA50500021681CF3
:10CD700080001150601CC4B20E48007AA042D5DC7D
:10CD80000C484068002813D00A48007A4000282840
:10CD900006D30848282201A943680220984707E0E3
:10CDA0000448007A4200034801A9436802209847DA
:10CDB00029B030BD142F0020FFB585B005460E46C2
:10CDC0001F460020049003900024029001900097D9
:10CDD000681C80004149085A0490002D05D0681E47
:10CDE000800040184088039003E0A8003B49085A9F
:10CDF000039003990E98884205D304990E988842AF
:10CE000001D80E9C08E0012E01D1049C04E0002E04
:10CE100001D1039C00E00E9C31480068052805D232
:10CE20002F480068401C2E49086053E000202C4920
:10CE3000086005210798FBF789F9029002980028FD
:10CE400044D028480068A04215D226480068201A1D
:10CE5000019002990198FBF779F901902148016846
:10CE6000019808181F49086008460068A04217D9B1
:10CE70000846046014E01B480068001B01900299FA
:10CE80000198FBF763F90190164801680198081AA8
:10CE90001449086008460068A04201D208460460B0
:10CEA000104800680090002E14D10E4800686330CE
:10CEB000B84201D300970DE064210A48006863304E
:10CEC000FBF744F964214843009003E005480460FF
:10CED00000680090009809B0F0BD0000161C020028
:10CEE000C0000020C800002008B510F07DFA01281D
:10CEF0007ED1FFF77FFD7949884216D20F2078490D
:10CF00008871C87108468078002801D105204870D2
:10CF100073488078052802D10020714948700020AC
:10CF20006F4948728872087035E0FA206C49887140
:10CF3000C8716C49088803F075FE6A48807800283B
:10CF40000CD16749087008468079C8700846C079D6
:10CF5000487100208870487088721CE00120604988
:10CF600008700846807A022805D1012088720020C6
:10CF7000C87048710FE05A48807A00280BD102200F
:10CF80005749887208464078887008468079C8708A
:10CF90000846C0794871524880785149497888429A
:10CFA00029DD50480088642148434D490090C979E3
:10CFB0004B4B5B79CA1A4A4988784B490B68002168
:10CFC000FFF7FAFE4849086000204549C87008711B
:10CFD00008464079401C487108464079C979884222
:10CFE00057DB00203E49487108468078401E00E02B
:10CFF00067E088704DE03A4880783949497888423E
:10D0000027DA3848008864214843354900908979F7
:10D01000334BDB78CA1A3249887833490B680121CF
:10D02000FFF7CAFE3049086000202D494871087199
:10D030000846C078401CC8700846C0788979884284
:10D0400027DB00202649C87008468078401C88707D
:10D050001FE0002022494871C87008460079401C32
:10D06000087108460079FA2801DBFA2008711D488A
:10D070000088642148431A4900900979FA235A1A12
:10D080001749887818490B680221FFF795FE164961
:10D09000086014488078002803D1012010494872A4
:10D0A0001BE003F0B7F8732803DB02200C49487239
:10D0B00013E003F0AFF870280FDC00200849487235
:10D0C0000BE000200649087008468079C8700846C1
:10D0D000C079487100204872887208BDB80B000002
:10D0E00050260020BC000020C4000020002004497D
:10D0F00088704870C8704871487288727047000024
:10D100005026002000200649088088700549887054
:10D110004870FA20C87048710020487288727047C1
:10D12000BC00002050260020F8B500240025002671
:10D13000002703F07FFC044603F08EFC054610F048
:10D1400053F901282ED105211A48FDF7E5FF55288E
:10D1500004D1002018498870088027E0012D04D1EF
:10D16000002015498870088020E00120124988704D
:10D170001248844202DB201A84B200E000240A2113
:10D180002046FAF7F9FF052901DB601D84B20C483F
:10D19000844200DD04460A212046FAF7EDFF0649E5
:10D1A000088003E00020044988700880FFF79CFE97
:10D1B000F8BD000060080020BC000020AA0A0000A2
:10D1C000C60700001CB500200090019000F0ACFAEA
:10D1D0000B49086000200B49096808600A4800688C
:10D1E00000280CD00749096808680A21FAF7AEFF41
:10D1F0000090012269460520034B1B6898471CBD1F
:10D20000F0070020E4070020EC0700200020084978
:10D21000488008490880084908800849087008497A
:10D220008872084908804880012008717047000012
:10D230002C0000201C0000201E00002020000020E8
:10D240004408002024000020F8B503F0D5FB074671
:10D2500003F0E4FB0090FFF7E7FB012860D1052114
:10D26000C548FDF759FF552802D00098012807D17D
:10D270000020C2490870C2490880C249887256E03D
:10D28000BE480078002810D10120BC4908703D46F6
:10D290002846E917890F091889030D0CBA488542F9
:10D2A00000DD0546B648058041E0B648807A40007A
:10D2B000B4490F520846867A0EE07000B1490D5A03
:10D2C000701E4000085A7100AE4A5052701E400055
:10D2D00011460D52701EC6B2002E08DD7000A9491D
:10D2E000095A701E4000A74A105A8142E5DBA54842
:10D2F000807A401CA34988720846807A052816DB8C
:10D30000002088720846C5882846E917890F091841
:10D310008D109D48854200DD05469948058006E050
:10D32000002096490870964908809649887294486A
:10D33000058896480088A84257DA94480088281A39
:10D3400084B292480079012827D190484088A042B1
:10D350000BDA8E4840880A308C494880084640885D
:10D36000A04204DD0846448001E0884844808748A4
:10D37000448803212046FAF7FFFE84B2192C00DA14
:10D3800019248248008800198049088008460088CE
:10D39000A84201DD08460580CDE07C48408814287D
:10D3A00005DD7A48408814387849488002E000203A
:10D3B000764948807548448803212046FAF7DCFE08
:10D3C00084B2192C03DA012070490871B3E06F4868
:10D3D0000088A04205DD6D480088001B6B4908806D
:10D3E000A9E0002069490880A5E068480088A842B3
:10D3F00059DD66480088401B84B2644800790128E2
:10D4000027D162484088142805DD604840881438D8
:10D410005E49488002E000205C4948805B484488BF
:10D4200003212046FAF7A8FE84B2192C03DA022061
:10D43000564908717FE05548008800195349088013
:10D44000084600885049884275DD08464F490880E3
:10D4500071E04E484088A0420BDA4C4840880A30C0
:10D460004A49488008464088A04204DD0846448076
:10D4700001E0464844804548448803212046FAF7A5
:10D480007BFE84B2192C00DA19244048008829193F
:10D49000884202DA3D4805804DE03C480088001B88
:10D4A0003A49088047E03948448803212046FAF782
:10D4B00063FE84B2192C3EDD34484088142805DD13
:10D4C0003248408814383149488002E000202F4912
:10D4D00048802E48448803212046FAF74DFE84B246
:10D4E0002A480079012813D1192C03DA0220274990
:10D4F000087120E025480088001924490880084662
:10D5000000882149884216DD08462049088012E03B
:10D51000192C03DA01201D4908710CE01B48008812
:10D52000A04205DD19480088001B1849088002E068
:10D5300000201649088016480088502804DC13484B
:10D5400000881349088016E01048008810490988AF
:10D55000884204DD0D4800880D4908800BE00B4827
:10D5600000880B490988081A84B2502C03DB07484D
:10D57000008807490880F8BD6008002020000020CE
:10D580001C00002044080020E02E000024000020A1
:10D590001E00002010B5044664204443A12120460B
:10D5A000FAF7D4FD0446204610BD000010B5012056
:10D5B0000F49087000200F49096808600D49096883
:10D5C00048600C490968886000F07EF9FFF7FAFDB1
:10D5D000FFF7A2FB08480068002807D00122054891
:10D5E000016808310020044B1B68984710BD0000FB
:10D5F000BD070020B8070020B407002010B5184868
:10D6000000681849884229D117480068002804D0CA
:10D6100015480068804715490870154800680028BB
:10D6200004D0134800688047124908701248006807
:10D63000002804D01048006880471049088010482E
:10D640000068002805D00E48006880470D49088012
:10D6500002E00D480B49088000F078F810BD00008A
:10D66000C807002078563412A4070020BC07002009
:10D67000A8070020BE070020AC070020C00700203C
:10D68000B0070020C20700201027000010B50023BB
:10D69000174C2360174C2370174C2370174C2370C2
:10D6A000174C2380174C2380174C2370174C13689A
:10D6B0002360174C53682360164C93682360164C04
:10D6C000D3682360154C1369236000280CD0144BD9
:10D6D0001860134C0B682468A3600023104C246866
:10D6E00023600F4C246863600E4B014C236010BD17
:10D6F000C8070020C4070020BC070020BE07002088
:10D70000C0070020C2070020BD070020A40700209A
:10D71000A8070020AC070020B0070020B4070020B5
:10D72000B807002078563412054800680549884239
:10D7300003D105480068806870470020C043FBE7BC
:10D74000C807002078563412B807002070B50024AE
:10D75000002500263048007801285CD12F48007849
:10D76000002858D12E480078012854D12D4805882A
:10D770002D490988694308462C49FAF7E7FC85B228
:10D78000E1200001854207D8192169430846092193
:10D79000FAF7DCFC044600E0244C254800680068E9
:10D7A0000019234909680860214800680068204979
:10D7B00009684968884207D31D48006800681C4909
:10D7C00009684968461A0AE019480068406800215B
:10D7D000C943081A1649096809684018461C1548C3
:10D7E000864218D3344601462046FAF7AFFC044679
:10D7F0000F48006841680F48604308180C490968E1
:10D80000486001200C4908700948006880680019C8
:10D8100007490968886070BDBC070020BD0700206B
:10D82000BE070020C0070020C2070020102700000C
:10D83000B8070020A0860100C407002000220C4B7E
:10D840001A600C4B0A681A600B4B4A681A600B4B43
:10D850008A681A600A4BCA681A600A4B0A691A6019
:10D86000002801D0084A1060084A014B1A6070472E
:10D87000C8070020A4070020A8070020AC0700204C
:10D88000B0070020B4070020B807002078563412F3
:10D8900010B50A48006800280ED009480078012811
:10D8A0000AD10020064908700122064801680831A3
:10D8B0000020024B1B68984710BD0000B4070020F1
:10D8C000C4070020B80700201CB50020009001907C
:10D8D0000024FFF729FF04460E480068046000207A
:10D8E0000C49096848600B49096888600A48006863
:10D8F00000280DD0074800680068009005480068BF
:10D9000040680190022269460120034B1B6898473A
:10D910001CBD0000CC070020D0070020F8B505464C
:10D920000C4616460027002D17D00E480560FFF75D
:10D93000FBFE07462068B84203D90A480068076022
:10D9400003E00849206809680860064960680968BA
:10D9500048600449A0680968C8600348066000F090
:10D9600005F8F8BDCC070020D007002070B50024D2
:10D970000025FFF7D9FE04460F4800680068A04262
:10D9800000D903E00C4800680068251A0A480068BE
:10D99000406840190849096888600748006880683D
:10D9A00005490968C968884205D903480068C06804
:10D9B00001490968886070BDCC07002001480068F3
:10D9C00080687047CC070020002801D0024A106010
:10D9D000024A116070470000CC070020D0070020E9
:10D9E0000549002005E00A1D135C044A1354421C3B
:10D9F000D0B22028F7DB704700065000C82E002068
:10DA000001461048026814204843101882680D48E7
:10DA10000368142048431818C06882420BD909488B
:10DA20000268142048431018C2680648036814208E
:10DA300048431818826003480268142048431018AD
:10DA400080687047142F002010B5002100220020AC
:10DA500005E01B4B1C5C1B4B1C54431CD8B2062816
:10DA6000F7DB1221002006E0174B1C5C154B9B1DB9
:10DA70001C54431CD8B28842F6DB002006E0134B4E
:10DA80001C5C104B18331C54431CD8B20628F6DB20
:10DA9000002006E00E4B1C5C0A4B1E331C54431C3A
:10DAA000D8B20628F6DB0422002005E00024054B4E
:10DAB00024331C54431CD8B29042F7DB10BD000045
:10DAC000390700209C2E00203F070020330700204C
:10DAD0002D07002038B50446002000900094012254
:10DAE0006946052000F06AFC38BD000008B500203A
:10DAF000009001226946062000F020FC684600786C
:10DB00000F4908736846407848730846007B0D4902
:10DB100048730B48407B88730948807BC87308486A
:10DB2000C07B087400200873074908600749086033
:10DB300007490860074908600749087008BD0000E8
:10DB40004C280020C80900207C0000208000002014
:10DB500084000020880000208C00002008B50020F0
:10DB6000009001226946062000F0E8FB6846007834
:10DB700012490873684640784873002010490860CD
:10DB800048600872487288720C48007B48730B48E2
:10DB9000407B88730948807BC8730848C07B087441
:10DBA00000200873074908600749086007490860B2
:10DBB000074908600749087008BD00004C2800208C
:10DBC000C80900207C000020800000208400002084
:10DBD000880000208C00002038B50024002500209B
:10DBE00000900121FA48FDF797FA55280AD002F073
:10DBF00077FFF849487302F087FFF64988730120E0
:10DC0000087308E0F448007BF2494873F248407B0F
:10DC10008873002008730621ED48FDF77DFA55282A
:10DC200030D002F0A5FF002808D002F0A1FF401C70
:10DC3000002803D00120E749087502E00020E549EB
:10DC4000087502F077FF002808D002F073FF401C2F
:10DC5000002803D00120DF49C87402E00020DD491C
:10DC6000C87402F085FF002808D002F081FF401C34
:10DC7000002803D00120D749087507E00020D549C6
:10DC8000087503E00020D349C8740875D148407B6B
:10DC900000282BD1D1490860D1480068D149884279
:10DCA00008D8CF480068401CCD4908600020C94909
:10DCB00048736CE0C848007B022812D0C648007B3D
:10DCC00003280ED00121C248FDF726FA552803D0BB
:10DCD0000320C04948735AE0BF48007BBD494873E0
:10DCE00055E0BD48007BBB49487350E0B948407BD4
:10DCF00001282CD10020BA490860B8480068B94909
:10DD0000884208D8B5480068401CB4490860012022
:10DD1000B04948733BE0B048007B022812D0AE48BF
:10DD2000007B03280ED00121A948FDF7F5F95528FD
:10DD300003D00320A749487329E0A748007BA549E1
:10DD4000487324E0A448007BA24948731FE0A1481F
:10DD5000407B022805D10020A14908609F49086046
:10DD600015E09C48407B032808D100209C490860AE
:10DD70009A49086003209749487308E000209849B1
:10DD80000860964908609448007B9249487391481E
:10DD9000807B00282BD19449086094480068914901
:10DDA000884208D891480068401C904908600020CB
:10DDB000884988736CE08848407B022812D08648E6
:10DDC000407B03280ED001218148FDF7A5F9552895
:10DDD00003D003207F4988735AE07F48407B7D4908
:10DDE000887355E07C48407B7A49887350E07948D5
:10DDF000807B01282CD100207C4908607A4800688B
:10DE00007849884208D878480068401C76490860FC
:10DE10000120704988733BE06F48407B022812D094
:10DE20006D48407B03280ED001216948FDF774F945
:10DE3000552803D003206749887329E06648407B52
:10DE40006449887324E06448407B624988731FE01A
:10DE50006048807B022805D100206449086062493F
:10DE6000086015E05B48807B032808D100205F49EB
:10DE700008605D49086003205649887308E0002067
:10DE80005A490860584908605348007B51498873D3
:10DE90005048407B5049097B884205D14D48807BE2
:10DEA0004D49497B88424FD04A48407B4A49097BCB
:10DEB000884202D001204749C8734648807B4649C2
:10DEC000497B884202D00120424908744148407B86
:10DED000022803D03F48407B032816D13D48407BB1
:10DEE0003D49097B884210D03A48407B3A49087343
:10DEF0000846017B684601703748417B684641709F
:10DF000001226946062000F059FA3248807B022837
:10DF100003D03048807B032816D12E48807B2E49C1
:10DF2000497B884210D02B48807B2B494873084698
:10DF3000017B684601702848417B68464170012298
:10DF40006946062000F03AFA02F0D4FD044602F0D9
:10DF5000E7FD0546FEF768FD01287BD101211C483D
:10DF6000FDF7DAF8552807D100201A4908724872DF
:10DF7000086048608872BAE0FF2C01D0FF2D78D18C
:10DF8000FF2C3FD1FF2D3DD0002012490872012007
:10DF90004872174808601748684348604868662117
:10DFA000FAF7D4F80B49486008464068124988429D
:10DFB00002D908460749486003F0E8F8112803DB56
:10DFC00003F0E4F8192819DD0120024988728EE077
:10DFD00060080020C80900204C2800208000002094
:10DFE0007C000020701700008800002084000020C2
:10DFF000DE030000BE0A0000AC26000000205D49E0
:10E00000887274E0FF2C2BD0FF2D29D101205949B3
:10E0100008720020487258484860584860430860B9
:10E0200008686621FAF792F85249086008460068C5
:10E030005349884202D908464E49086002F0A2FFBF
:10E04000112803DB02F09EFF192805DD0120494954
:10E0500088724CE086E00CE000204649887246E079
:10E060004748444908604860002088720872487236
:10E070003DE001203F490872487240486043086013
:10E0800008686621FAF762F83A49086008460068AD
:10E090003B49884202D908463649086037486843F8
:10E0A0003449486048686621FAF750F831494860B9
:10E0B000084640683249884202D908462D494860DE
:10E0C00002F060FF11280BDB02F05CFF192807DC6F
:10E0D00003F05CF8112803DB03F058F8192803DD7E
:10E0E00001202449887202E00020224988722148D8
:10E0F000407B002802D11F49C87315E01D48407BB2
:10E10000012802D11B49C8730EE01A48407B02283F
:10E1100002D11849C87307E01648407B032803D191
:10E120001449C873164808601248807B002802D141
:10E13000104908741DE00F48807B012802D10D4969
:10E14000087416E00B48807B022802D10949087444
:10E150000FE00848807B03280BD106490874084863
:10E16000486006E000200349087248720860486071
:10E17000887238BDC8090020DE030000BE0A000016
:10E18000AC260000FFB583B006460D4617460024B6
:10E190000020029000BF1420784380190190002EC7
:10E1A00057D00198002854D02B4806602A49069879
:10E1B00048600846077200BF45E0FFF7B5FA0290D5
:10E1C000200129580298814204D820012858401C77
:10E1D000002806D1204902980A6814216143505052
:10E1E00006E0200129581C480268142060431150A1
:10E1F000200140194068401C002807D10021164822
:10E200000268142060431018416008E020014019A2
:10E2100041681148026814206043101841602001D1
:10E22000401981680C480268142060431018C160CE
:10E2300020014019017B084802681420604310182F
:10E240000161601CC4B20448007AA042B5DC00F051
:10E2500005F807B0F0BD0000142F002070B50024B1
:10E2600000250026FFF760FA054600BF4EE02A4869
:10E270000168142060430858A84239D8264801682C
:10E280001420604308582E1A234801681420604364
:10E29000081840688119204802681420604310184B
:10E2A00081601D48016814206043081881681A487D
:10E2B0000268142060431018C068814224D91648AF
:10E2C00001681420604308180069002803D0204624
:10E2D000FEF7D8FC18E010480168142060430818C5
:10E2E000C1680D48026814206043101881600BE07B
:10E2F00009480168142060430818406806490A6804
:10E300001421614351188860601CC4B20248007A2D
:10E31000A042ACDC70BD0000142F002010B500BF7F
:10E3200014244C432318002805D0002B03D0024CA2
:10E3300020606260217210BD142F0020F8B50546E0
:10E340000E4614462B0012F0BDFB0705131A31319F
:10E35000212931001748FAF707FC174908701548BA
:10E36000F9F7BCFF07466421F9F7F0FE30601EE0C4
:10E37000A004020C31462020FAF7F0FC17E0A004BC
:10E38000020C31466020FAF7E9FC10E0A004020C10
:10E390003146FF202130FAF7E1FC08E06004020C6E
:10E3A0003146FF204130FAF7D9FC00E000BF00BF42
:10E3B0000020F8BD3E280020D500002070B505469D
:10E3C0000E4614462B0012F07DFB07051D243A3A39
:10E3D0002B323A003068002802D1FAF763FA10E0D5
:10E3E00064223168514308461649F9F781FF00203D
:10E3F00015490870012264211248FAF71DFD1249DF
:10E4000008701DE0A004020C31462020FAF764FEDB
:10E4100016E0A004020C31466020FAF75DFE0FE022
:10E42000A2B23146FF202130FAF756FE08E0600420
:10E43000020C3146FF204130FAF74EFE00E000BFEB
:10E4400000BF70BD30280020D400002000B5AFB060
:10E4500050211BA8F9F72AFF00201A90142115A8B3
:10E46000F9F724FF0020129013901490119040218E
:10E4700001A8F9F71BFF002000904849086001221D
:10E480001BA9FFF75BFF1B98401C002801D11A90C5
:10E4900001E01B981A904248159042481690424855
:10E4A0001790002018904148199015AA1AA94048C1
:10E4B000FFF7ECF802221CA90120FFF73FFF1C9890
:10E4C000401C002801D1129001E01C9812901C9869
:10E4D000401C002801D1139001E01D98139035488D
:10E4E000149012A93448199AFFF718FA08221EA9A5
:10E4F0000220FFF723FF1E98401C002801D1019045
:10E5000001E01E9801901F9802902C480390012072
:10E5100069460874801E059029490791012101A8C8
:10E520000177881E099026490B91012109A80173E2
:10E53000881E0D9022490F9101210DA8017304221C
:10E5400001A92048199BFFF71DFE01221BA90520E8
:10E55000FFF7F4FE1B98401C002807D101201A4940
:10E560008860012208310520FFF728FF01221BA93E
:10E570000620FFF7E3FE1B98401C002808D100216D
:10E58000684601704170012269460620FFF716FFB8
:10E590000E48024908602FB000BD0000D8000020DE
:10E5A00029CA00001DCA000001CA0000BDE3000026
:10E5B000C427002076841E00D02700200F270000EB
:10E5C0009F860100E02700204C280020A33AA55A8E
:10E5D00000B585B014216846F9F768FE00200F49A0
:10E5E00008600F4800900F4801900F4802900020EB
:10E5F00003900E48049069460D48FFF71FF90D4837
:10E600000499FFF7E1F904210B48049AFFF786FE0D
:10E610000A480249086005B000BD0000D80000208B
:10E6200029CA00001DCA000001CA0000BDE30000A5
:10E63000C4270020D0270020E0270020A33AA55AB5
:10E6400000200C4908800C4908800C4908800120F2
:10E650000B49087000200B4908730B49088048805B
:10E660000120087100200749488008800749086098
:10E670007047000034000020360000203C000020DD
:10E680003E000020500800204000002038000020FC
:10E69000F8B502F0EBF9064602F0F2F90746FEF78C
:10E6A000C3F9012865D10521AB48FCF735FD552894
:10E6B00007D10020A9490870A9490880A949888084
:10E6C0005FE0012F07D10020A4490870A449088009
:10E6D000A449888055E0A1480078002808D101208D
:10E6E0009E49087035460A2068439D49088048E0E5
:10E6F0009C48007B42009B48801D8652801F047B03
:10E7000011E061009748801D455A601E4100954800
:10E71000801D415A62008152601E41009148801D57
:10E720004552601EC4B2002C0ADD61008D48801D78
:10E73000415A601E42008B48801D805A8142E0DBB6
:10E740008848007B401C874908730846007B0328E3
:10E7500007DB00200873084605890A2068438049C2
:10E7600008807F4800887F49888001207B490870A5
:10E7700007E00020794908707949088079490873D1
:10E7800088807748008878490860744800780028B5
:10E7900015D0084600686C2148437349086064211D
:10E7A00071480068F9F7D2FC6F49086008460068B4
:10E7B0006E49884206D908466B49086002E000208D
:10E7C000694908606848006869490988884203D235
:10E7D000654800680F2804D26348008864490880AF
:10E7E0000AE06348008860490968401A0F2803D38B
:10E7F0005D4800885E4908805A480088401C594995
:10E800000880084600880A282CDB00200880594828
:10E81000008857490988884203DA0120564908715F
:10E8200008E05448008852490988884202DD0220E5
:10E830005149087150480079012840D14C4800885E
:10E840004C49098888420DDB4948018849480088BD
:10E85000FF309130814206DD46480088FF3073303A
:10E860004449088077E04248018842480088963051
:10E87000814205DD3F48008878303E4908806AE0E3
:10E880003B4801883B4800883230814205DD3948E9
:10E8900000881E30374908805DE0354801883548DA
:10E8A00000880A30814205DD324800880A3031494B
:10E8B000088050E02E4800882E4908804BE02E4802
:10E8C0000079022847D12A4800882A4909888842C5
:10E8D00039DA27480088FF30913026490988884274
:10E8E00006DA24480088FF387338224908802AE075
:10E8F0001F48008896301F490988884205DA1D485C
:10E90000008878381B4908801DE01948008832309B
:10E9100018490988884205DA164800881E381549C2
:10E92000088010E0124800880A301249098888429D
:10E9300005DA104800880A380E49088003E00C48C0
:10E9400000880C4908800B4800880849884202DB8F
:10E95000084608490880F8BD600800203E000020F5
:10E96000340000205008002038000020C6070000B6
:10E970003C00002036000020400000200020084914
:10E9800008800849088008490880488001200871EB
:10E99000002006494880088005490860704700004B
:10E9A000360000203C0000204000002050080020DD
:10E9B0003800002000200449087004490870002134
:10E9C00003480176704700008D0000208E00002073
:10E9D000400A002070B500250024FEF725F8012824
:10E9E00063D103213448FCF797FB552808D1002058
:10E9F000324908703249087000213248017659E0E6
:10EA00002F480078002807D102F0D0F82B49087071
:10EA100001202B4908704DE001202949087002F0BF
:10EA2000C5F82849097E8900264A603A5050254891
:10EA3000047E10E0A000234960390D5C601E800058
:10EA40000858A1001F4A603A5050601E80001146CD
:10EA50000D50601EC4B2002C0ADDA00019496039B7
:10EA60000958601E8000174A603A10588142E1D36D
:10EA70001448007E401CC1B212480176007E1E2858
:10EA800018DB00210F48017601466039896B024688
:10EA9000603AD26B89180246603A126C88180321DA
:10EAA000F9F754FB0549087004E000200349087099
:10EAB0000349087070BD0000600800208D00002030
:10EAC0008E000020400A0020F0B5A9B004460E4692
:10EAD0000025002700202890A0216846F9F7E6FBD2
:10EAE000FEF722FE26490A6814216143505024484B
:10EAF0000168142060430818C068B0420CD2204856
:10EB00000168142060430818C1681D480268142079
:10EB100060431018416005E0194801681420604303
:10EB20000818466016484068002826D0002517E0DF
:10EB30006806070E282F00D316E01148016814203C
:10EB400068430858B9006A4650500D4801681420BF
:10EB5000684308184168781C80001150681CC5B2D1
:10EB60000748007AA842E3DC00BF6A00044869460F
:10EB700043680220984701202890289829B0F0BDCA
:10EB8000142F002010B500F0F9FD00F0D7F810F0B8
:10EB9000B9FE00F00DFB00F001F810BD70B5414862
:10EBA0000078912800D070BD00F0BEF8012876D121
:10EBB0003D4800883D49088008468078F021884318
:10EBC00020303A49887008468078000900013549AC
:10EBD000097A0907090F0843344988703148807A57
:10EBE000401E3049887208460089401C088108464A
:10EBF0000089C988884216DA08202C4988720024C6
:10EC00000EE0284841882848001D415C2748C01C68
:10EC1000015524484088401C22494880601CC4B2E9
:10EC2000072CEEDB2DE01F4800891E49C988884269
:10EC30001CD11C4800791B498978401AC5B2681C50
:10EC40001A49887200240EE0164841881648001DB3
:10EC5000415C1648C01C015512484088401C1149AF
:10EC60004880601CC4B2AC42EEDB0AE000F012FD4A
:10EC700000200C4908700C490888092100F0B8F9F7
:10EC800091E7012000F0C8FC084A917A1088921C94
:10EC900000F070F905490888002100F0C1F800BFB4
:10ECA00081E700004C2C0020E82B0020782B00206E
:10ECB0001B49097E002932D01949897E0C22514313
:10ECC000174A515A174A118000200CE01449897ED6
:10ECD0000C225143124A8918891C0A5C1149891C6B
:10ECE0000A54411CC8B20828F0DB0D49897E0C2269
:10ECF00051430B4A8918897A0A4A91720121D172CB
:10ED00000749097E491E064A11761146897E491C2B
:10ED100091761146897E022901DB002191767047A8
:10ED2000442B00206C2B00200349487B012802D192
:10ED30000021014A517370475C2C002010B5334804
:10ED40004068002861D13148007B030011F0BAFE11
:10ED500007590512212E3D4A59002D4800780028F8
:10ED600007D000202A4908702A490888012100F0AC
:10ED70003FF947E026480078002809D000202449C0
:10ED8000087025494A8808880123091D00F040F9C8
:10ED900038E01F480078002807D000201C49087080
:10EDA0001C490888022100F023F92BE0184800785C
:10EDB000002809D000201649087017494A88088899
:10EDC0000923091D00F024F91CE0114800780028EF
:10EDD00007D000200E4908700E490888092100F06C
:10EDE00007F90FE00A480078002809D000200849F8
:10EDF000087009494A8808880323091D00F008F9AA
:10EE000000E000BF00BF00F045FC10BD5C2C0020FE
:10EE10004C2C0020E82B0020842B002070470000A1
:10EE200070B504460D4634480088A04263D1002DD9
:10EE300061D13248007822284ED004DC20283DD011
:10EE4000212856D141E0902802D0912851D115E0D7
:10EE50002A48C08801280AD100202849087000F0FB
:10EE600019FC27490888002100F0C2F805E00320BA
:10EE700000F0D2FBA020214908703BE01F48008928
:10EE80001E49C98888420AD100201C49087000F038
:10EE900001FC1B490888002100F0AAF80DE0174882
:10EEA000807A002806D000F0F5FB1449087B00F0BA
:10EEB00095FB02E0032000F0AFFB1BE0062000F012
:10EEC000ABFB11200D49087014E0062000F0A4FBF4
:10EED00011200A4908700DE000200849087000F070
:10EEE000D9FB08494A8808880923091D00F090F8D1
:10EEF00000E000BF00BF70BD602B00204C2C002044
:10EF0000E82B0020842B002070B50346184C247E8B
:10EF1000022C00DB70BD164C647E0C256C43144D36
:10EF20002B5300200AE0155C114C647E0C267443C0
:10EF30000F4EA419A41C2554441CE0B28842F2D3FD
:10EF40000B4C647E0C267443094EA419A1723446FE
:10EF5000247E641C35462C762C46647E641C6C76BC
:10EF60002C46647E022C01DB00246C7600BFD1E7C6
:10EF7000442B0020F0B585B007460D4616461A48CA
:10EF80000780002406E031781748801C0155761C64
:10EF9000601CC4B2AC42F6DB2C4605E0AA21124844
:10EFA000801C0155601CC4B2082CF7DB0E48008899
:10EFB000019008216846C1720021417201720170FE
:10EFC000002406E00848801C015D03A80155601C70
:10EFD000C4B2082CF6DB69460448FCF7AEF9012000
:10EFE0000149887205B0F0BD602B002090550440A7
:10EFF00070B504460D462946204610F0A5FB70BDAD
:10F0000070B504460D462946204610F0ABFB70BD96
:10F01000F8B504460D4616461F463B46324629467D
:10F02000204610F0A0FBF8BDF8B507460E46154681
:10F030005C480078002804D009213846FFF7D8FF43
:10F04000F8BD002D01D0602D04DD09213846FFF701
:10F05000CFFFF5E7544807804580002406E031786B
:10F060005148001D0155761C601CC4B2AC42F6DB51
:10F0700000204C49487008468580FF2088727F2018
:10F0800008730846808808282EDA0120C8800846C0
:10F0900080884880012008814348008843490880CF
:10F0A00008468078F0218843404988700846807877
:10F0B000000900013B4909790907090F08433B4949
:10F0C000887038480079401C8872002407E0364870
:10F0D000001D015D3548C01C0155601CC4B231489B
:10F0E0008088A042F3DC4AE00721681CF9F744F865
:10F0F000002907D0072128460830F9F73DF82949AB
:10F10000C88005E00721681CF9F736F82549C88052
:10F11000062024494880012008812348008823498B
:10F12000088008468078F021884310301F49887095
:10F1300008468078000900011A4989880905090FE5
:10F1400008431A49887008464088FF21090288430D
:10F15000144989880902FF22120211400843134909
:10F16000488008208872002407E00F48001D015DD8
:10F170000E48001D0155601CC4B2062CF5DB0120B1
:10F1800000F04AFA094A917A1088921CFFF7F2FEC1
:10F19000902004490870054908880021FFF740FEC7
:10F1A00000BF4DE74C2C0020E82B0020782B0020DE
:10F1B00010B5FFF77DFD1448C07A002822D0124810
:10F1C00080780009002806D0012807D002280AD03C
:10F1D000032810D10CE000F0A7F90FE000F09EF832
:10F1E00000F066FA0AE000F011F800F061FA05E0BC
:10F1F00000F000F902E0FFF711FE00BF00BF0020A1
:10F200000149C87210BD00006C2B002010B53F48AA
:10F210000078112800D010BD3D4800883D49884243
:10F2200000D0F8E73A4880780007000F3749097A9C
:10F230000907090F88420CD000203449087000F0FB
:10F2400029FA35494A8808880423091DFFF7E0FE9A
:10F25000E1E72E480089401C2C4908810846807A45
:10F26000401E887208460089C98888421BDA2848EF
:10F27000807A082800D0CEE700240EE02448C01C85
:10F28000015D224842882448001D81541F4840885F
:10F29000401C1E494880601CC4B2072CEEDB0620CF
:10F2A00000F0BAF930E01948808818494988401AB6
:10F2B0001749897A884203DA1548807A082800D0ED
:10F2C000A9E700240EE01248C01C015D0F484288E7
:10F2D0001148001D8154601CC4B20C484088401C79
:10F2E0000A49488009484088084989888842EADBF9
:10F2F00000200649087000F0CDF907494A880888BF
:10F300000023091DFFF784FE00BF84E74C2C00207A
:10F310006C2B002014070000842B002070B53148AE
:10F32000007880210840802800D170BD2E480088D8
:10F330002E49884200D0F8E72B48807A082800D070
:10F34000F3E72948807805072D0F2D0226484088CD
:10F35000000A0543082D00DAE7E70020214948703C
:10F360000620488008468580012008810820887290
:10F370000020C8728988481C0721F8F7FDFE002983
:10F3800009D018498988084608300721F8F7F4FEA3
:10F390001449C88007E013498988481C0721F8F7F9
:10F3A000EBFE1049C88010480088114908800846C3
:10F3B0004580002407E00C48001D015D0C48001D3D
:10F3C0000155601CC4B2062CF5DB042000F024F9C2
:10F3D000102004490870064A51881088FFF710FE73
:10F3E00000BFA2E74C2C00206C2B0020140700006B
:10F3F000842B002010B548480078A02808D0464843
:10F400000078912804D044480078A12800D010BD8D
:10F4100042480088424988420AD042490888092166
:10F42000FFF7E6FD00F036F900203B490870EEE7F3
:10F430003A48807A08280AD03A4908880921FFF713
:10F44000D7FD00F027F9002033490870DFE7334883
:10F4500080780007000F002804D001282DD0022852
:10F460004BD136E02C484078002800D050E02B48A3
:10F47000C078002803D101202749487003E02748BD
:10F48000C078254988722448007891280BD02348F9
:10F490000079002803D101201F49087303E01F48A9
:10F4A00000791D49087391201B49087000F0F2F89B
:10F4B0001949087B00F092F82AE0174840780028A4
:10F4C00000D025E0A12014490870032000F0A4F822
:10F4D0001EE011484078002800D019E00E4800785E
:10F4E000A02809D10F4908880821FFF781FD00F005
:10F4F000D1F80020084908700AE00A490888052167
:10F50000FFF776FD00F0C6F800200349087000BF41
:10F5100000BF00BF7BE700004C2C00206C2B0020BC
:10F5200014070000E82B002010B52848007880213F
:10F530000840802800D110BD24480078002805D05C
:10F54000234800882349884200D0F4E72048807A85
:10F550001F4989780907090F884203DD1C48807A12
:10F56000082800D0E7E71A4880780007000F002835
:10F5700005D0174880780007000F072800DDDAE77C
:10F580001348008814490880114880780007000F4C
:10F590004880002407E00E48C01C015D0E48001D95
:10F5A0000155601CC4B20C484088A042F3DC002026
:10F5B0000649087000F06EF807494A880888002359
:10F5C000091DFFF725FD00BFB5E700004C2C00200A
:10F5D0006C2B002014070000842B00207F2805DC02
:10F5E0007D21C90041430A4A91600DE0F12808DB02
:10F5F000F92806DC0107090F64225143044A91608F
:10F6000002E00449024A91600221014A51737047A5
:10F610005C2C002018F0010000B5030011F052FA34
:10F620000729050B11171D2329000121144A117305
:10F630001449516022E00221114A117311495160AD
:10F640001CE003210E4A11730F49516016E004219A
:10F650000B4A11730D49516010E00521084A1173DE
:10F66000002151600AE00621054A117308495160E2
:10F6700004E00021024A1173516000BF00BF00BDC9
:10F680005C2C0020A8610000F82401002823000061
:10F69000F049020000200149087370475C2C0020EB
:10F6A000024909880918014A118070475C2C002022
:10F6B00010B52E480078102818D12D4840886028B1
:10F6C0000ADD2C48807800090001801C29498870D7
:10F6D00022202649087025E026488078000900018C
:10F6E000244988702020214908701BE01F480078B9
:10F6F000112816D11D48807A002800D010BD1B4863
:10F700004078002800D0F9E7082018498872194885
:10F71000807800090001174988702020134908707B
:10F7200000E0EBE714481349088008468078F02190
:10F73000884330300F4988700846C0780020C87070
:10F740000846007914200871032088720220FFF710
:10F7500063FF084A917A1088921CFFF70BFC054959
:10F7600008880021FFF75CFB00BFC7E74C2C002096
:10F77000842B0020782B002094070000244A118855
:10F7800052888A4242D0224A52888A4204DA204A67
:10F7900052888A1A90B207E01D4A52880023DB4340
:10F7A0009A1A521C521890B2194A5180127B002AA0
:10F7B00010D0174A5268002A0CD0154A526882426B
:10F7C00005D9134A5268121A114B5A6002E00022FE
:10F7D0000F4B5A600E4A527B022A17D10C4A92688C
:10F7E000002A0CD00A4A9268824205D9084A9268D7
:10F7F000121A074B9A6002E00022054B9A60044AF5
:10F800009268002A02D10122014B5A73704700000E
:10F810005C2C002010B506F03BF910BD00BF70470E
:10F8200010B5044621460320400206F057F810BDEB
:10F8300010B580210320400205F0E4FF10BD000058
:10F8400010B50224024806F02DF80446204610BDEB
:10F850000106000010B50021014805F0D3FF10BDDE
:10F860000106000010B504462146024806F036F8AD
:10F8700010BD00000106000010B58021014805F010
:10F88000C1FF10BD0106000030B503460C46002143
:10F8900001250D48834201D0002B01D1022030BD4B
:10F8A000012A01D10120FAE7002108E0C800205810
:10F8B000984202D100252846F1E7481C81B29142C6
:10F8C000F4DB2846EBE70000FFFF0000002000BF4C
:10F8D00014E00021C200134B9950C200D21891804D
:10F8E000C200114B9950C200D2189180C2000F4B38
:10F8F0009950C200D2189180411C88B24828E8DB98
:10F900000B490C4A11600C495160002191600B4970
:10F9100011610B49D16000210A4A11800A4A117015
:10F9200070470000901F0020D021002010240020EC
:10F93000FD0D01007C1F0020990E0100430F010006
:10F94000350F0100B6000020BA000020F0B585B0E8
:10F950000646674F38460390029000250024002099
:10F960000190009063480068002803D0614908684E
:10F97000804707465F484068002803D05D494868D3
:10F98000804703905B488068002803D05949886805
:10F990008047029057480069002803D055490869FC
:10F9A000804700905348C068002803D05149C86878
:10F9B00080470546482D00DD48250098002876D070
:10F9C000002D74DD4C480088A8420BDA2B463A46DD
:10F9D00049494A48FAF788FE2B4647494748039A5F
:10F9E000FAF782FE44480088002833DD4248008848
:10F9F000A84202D1002040490880002415E0E00020
:10FA00003F490858E1003D4A515888420BD0E00078
:10FA100011460858E1003A4A5050E0001146085893
:10FA2000E100384A5050601C84B2AC42E7DB012050
:10FA3000354908702C460BE00020E100314A505057
:10FA4000E1002F4A5050E1002C4A5050601C84B213
:10FA5000482CF1DB2B4800682549884246D02948CC
:10FA600080882A49884205DA2648808880192549F5
:10FA700088803BE000202349888008460068019088
:10FA8000012D33DD002408E0601CC0001D4908582A
:10FA9000E1001C4A5050601C84B2681EA042F3DC96
:10FAA000691EC900174A019850501FE0FFE7002067
:10FAB00015490870002414E00020E100114A50505C
:10FAC000E10089188880E1000C4A5050E100891853
:10FAD0008880E1000A4A5050E10089188880601C43
:10FAE00084B2482CE8DB00200349088005B0F0BD53
:10FAF000FFFF00007C1F0020B6000020D021002066
:10FB000010240020901F0020BA000020881300005D
:10FB10002E480078401C2D4908702D480078401C64
:10FB20002B4908702B480078401C2A4908702A4845
:10FB30000068401C2849086008460068FF21913190
:10FB4000884202D900202449086020480078C8284B
:10FB500002D900201D4908701D480078842802D968
:10FB600000201B4908701B480078502802D900204B
:10FB700018490870194818490968405C1849087004
:10FB8000184812490978405C17490870174810490D
:10FB90000978405C1649087016480E490978405C9F
:10FBA00015490870154809490978405C14490870DE
:10FBB000144806490978405C134908701348034902
:10FBC0000978405C12490870704700006307002004
:10FBD000640700206507002068070020432002001A
:10FBE0005C070020D32102005D0700209B22020059
:10FBF0005E070020E7230200600700201F230200A9
:10FC00005F0700203724020061070020FF24020064
:10FC10006207002010B58200054BD218525C012A01
:10FC200004D100228300024C1B195A5410BD00005D
:10FC3000C82A002010B50446204600F055FA204698
:10FC400000F002F810BD000010B50446B34800787B
:10FC500000287DD1B2480088B249884278DAB2489B
:10FC6000007800284FD0B1480078002803D0AC4875
:10FC70000088AF490880AF480078002818D1A8480C
:10FC80000188AB4800880A30814206D30120A94987
:10FC90000870A3480088A6490880A1480088A449A4
:10FCA000098888421CDA9E480088A149088017E02C
:10FCB0009F4801889A4800880A30814206D3002074
:10FCC0009C490870964800889949088094480088A3
:10FCD00097490988884203DD914800889449088043
:10FCE00094480078002858D193480078042803D01D
:10FCF0008E480078002807D089480088822803DAD7
:10FD000005208D490870A3E08B480078032803D0B4
:10FD100086480078002809D081480088FF211931E1
:10FD2000884203DA04208449087091E08248007810
:10FD3000022803D07D48007800280AD0784800883F
:10FD4000FF21AF31884204DA03207B4908707FE04D
:10FD5000E2E079480078012803D074480078002850
:10FD600009D06F480088AF218900884203DA022059
:10FD7000714908706CE070480078002803D06B4827
:10FD80000078002864D066480088E1218900884214
:10FD90005EDA0120684908705AE066480078012858
:10FDA00056D165480078012803D0604800780028C3
:10FDB00009D05B480088E1218900884203DB0020EC
:10FDC0005D49087044E05C480078022803D0574839
:10FDD0000078002809D052480088AF218900884265
:10FDE00003DB01205449087032E0534800780328AF
:10FDF00003D04E480078002809D049480088FF21E8
:10FE0000AF31884203DB02204B49087020E04A48AA
:10FE10000078042803D045480078002809D04048DD
:10FE20000088FF211931884203DB03204249087012
:10FE30000EE041480078052803D03C4800780028AF
:10FE400006D037480088822802DB04203A4908702F
:10FE5000FCF7D0FD3349643988425DD337480068E8
:10FE600000193649086031480078002808D0002081
:10FE70002E490870314908602F48007830490870D1
:10FE800000F0A8FD00281FD12C4800682D498842A9
:10FE900039D3002029490860294800782649097883
:10FEA000884205DA26480078401C254908702AE077
:10FEB0002348007820490978884224DD20480078CA
:10FEC000401E1F4908701EE01C4800681E498842F9
:10FED00019D3002019490860194800781649097893
:10FEE000884205DA16480078401C154908700AE077
:10FEF0001348007810490978884204DD10480078DA
:10FF0000401E0F4908700E4800780B490978884256
:10FF100002D100200949086010BD00000B0000203C
:10FF2000020000201C0C000012000020080000202D
:10FF3000040000200A000020060000201800002015
:10FF400007000020C05D0000407E050000200B4936
:10FF500008700B49087001200A4908700A490870A6
:10FF600000200A4908700A4908700A4908800A49AD
:10FF700008800A4908800A49087070470600002076
:10FF80000700002008000020090000200A000020CF
:10FF90000B0000200C0000200E00002010000020AC
:10FFA0001200002000200B4908700B490870012046
:10FFB0000A4908700A49087000200A4908700A496D
:10FFC00008700A4908800A4908800A4908800A49D5
:10FFD000087070470600002007000020080000207D
:10FFE000090000200A0000200B0000200C00002067
:10FFF0000E0000201000002012000020F8B5064678
:020000040001F9
:1000000000270024002500200090314800780028B7
:1000100009D00320F9F7A8FA002804D00320F9F743
:1000200097FA2C4908802C4800880A284AD30020D7
:100030002949088029480078282829D20320F9F77F
:1000400087FA0746002407E060002549085AB842AD
:1000500000DD05E0601CC4B2204800788442F3DB78
:1000600000BF1E48057808E0681E40001C49085A79
:1000700069001B4A5052681EC5B2A542F4DC6000FC
:1000800017490F5215480078401C1449087019E0B0
:10009000002000900F2407E060001149095A0098E1
:1000A00008180090601CC4B2192CF5D30A210098DE
:1000B000F8F74CF80749088000200849087001202B
:1000C0000849087004480088801903490880F8BD71
:1000D000090000200200002016000020000000207F
:1000E000F407002012000020394909881E2928DA67
:1000F0000021384A1180384A118038490988384A25
:10010000914207DC37490978002914D0334909881E
:10011000914210DC0121344A11700021334A1170E0
:10012000334A11702F4A11700121324A1170002197
:10013000314A11704BE0294909880918274A118072
:1001400045E023490988264A643291422ADB00218E
:10015000224A1180204A11801E490988204A914272
:1001600007DC20490978002916D01A4909889142EC
:1001700012DC02211C4A117000211C4A1170052159
:100180001B4A11700021174A11700121194A117080
:100190000021194A11701AE00E49098809180D4A00
:1001A000118014E000210D4A11800A4A11800A4989
:1001B00009880B4A914205DD00210B4A1170094A5A
:1001C000117004E0044909880918034A1180704736
:1001D00002000020100000200C0000200E00002073
:1001E000B80B0000090000200B00002006000020D2
:1001F00007000020080000200A00002001480078C5
:1002000070470000502600200148407A70470000E7
:100210005026002010B5642102480068F7F796FFC9
:1002200080B210BDC40000200148807870470000F3
:1002300050260020F8B50023002500950024002258
:1002400000BF94E001259D40ACB20D88254000958B
:10025000009DA5426FD11A468D79012D0DD1464DD5
:1002600003263602AD192D5C012696403543424ED9
:1002700003273F02F61935540CE03F4D03263602A2
:10028000AD192D5C01269640B5433B4E03273F0236
:10029000F6193554CD78002D4ED1374D60352D5C93
:1002A000CE78002E01D1012600E000269640B5430D
:1002B000314E603635548D78002D2ED12E4D1926B5
:1002C0007601AD192D5C8E78002E01D1012600E05B
:1002D00000269640B543284E19277F01F61935545C
:1002E0000D79002D0ED1244D50352D5C0E79002E48
:1002F00001D1012600E000269640B5431E4E50363F
:10030000355423E01C4D50352D5C0E799640354315
:10031000EEB2194D50352E5418E0174D19267601BE
:10032000AD192D5C8E7896403543134E19277F0109
:10033000F61935540AE018E00F4D60352D5CCE7883
:1003400096403543EEB20C4D60352E544D79012D5B
:100350000AD1094D30352D5C012696403543EEB269
:10036000054D30352E5400E000BF5D1CABB2082BAC
:1003700000DA67E7F8BD000000000440FFB507465B
:1003800015461E4600243846019900F01FF8002843
:1003900002D0012004B0F0BD00240CE00A2060432C
:1003A0000949085CB04204D12946204600F05EF8B5
:1003B00007E0601C84B20A2060430349085C0028FF
:1003C000ECD100BF0020E5E7B80100200246002A7A
:1003D00003D1402901DD01207047032A03D10229FE
:1003E00001DD0120F8E7042A03D1202901DD0120E5
:1003F000F2E7052A03D1202901DD0120ECE70C2AD0
:1004000003D1102901DD0120E6E70D2A05D10129DC
:1004100003DD402901DA0120DEE70E2A03D120297D
:1004200001D10120D8E70020D6E7000010B5064A28
:1004300003231B02D218125C8A43034B03242402B9
:100440001B191A5410BD00000000044010B5064AE4
:1004500003231B02D218125C0A43034B0324240219
:100460001B191A5410BD00000000044070B502466C
:100470000020B1E00A2353435A4C1B195B1C440073
:1004800004191B199B788B427DD10A235343554C89
:100490001B195B1C440004191B195B78082B33D112
:1004A0000A2353434F4C1B195B1C440004191B5770
:1004B0004D4C4E4D6419E35C012423430A245443FC
:1004C000484D6419641C450045196457464D474E14
:1004D000AD192B550A235343424C1B195B1C440096
:1004E00004191B57404C35466419E35C022423432E
:1004F0000A2454433B4D6419641C45004519645754
:10050000394DAD192B5564E00A235343354C1B1963
:100510005B1C440004191B195B78092B34D10A2396
:100520005343304C1B195B1C440004191B572E4CC1
:100530002E4D6419E35C402423430A245443294D7F
:100540006419641C450045196457274D274EAD19A1
:100550002B550A235343234C1B195B1C44000419DD
:100560001B57214C35466419E35C8024A3430A24BD
:1005700054431C4D6419641C4500451964571A4DB9
:10058000AD192B5525E025E00A235343154C1B19C3
:100590005B1C440004191B57134C144D6419E35C95
:1005A0000A2454430F4D6419641C4500451964190D
:1005B00065780124AC402343DCB20A235343094D40
:1005C0005B195B1C450045195B57074D074EAD197C
:1005D000EC5404E0431CD8B2032800DA4AE700BF19
:1005E00070BD0000B8010020000004407508000044
:1005F000F8B50024FCF718FA012861D100F0A6FB39
:100600000446FF220721002003F0BCF8012C21D171
:1006100000F09AFC00280ED000F0AAFB054600F07E
:100620009BFB0646012003460246294600903046C1
:1006300005F068FC50E000F09BFB054600F08CFBE9
:10064000064601200023024629460090304605F068
:1006500059FC41E0022C21D100F076FC00280ED09C
:1006600000F086FB054600F077FB064601200346B6
:10067000024629460090304605F044FC2CE000F08C
:1006800077FB054600F068FB0646002001231A466A
:1006900029460090304605F035FC1DE000F054FC82
:1006A000054600F065FB064600F056FB07460120B4
:1006B00003462A4631460090384605F023FC0BE0FD
:1006C0000020034602460146009005F01BFC002274
:1006D0000721104603F056F8F8BD0000FEB50024CF
:1006E00081480078012827D1FCF79EF9012815D10F
:1006F000FBF77CFF00BF0EE0182C0AD0152C08D0A9
:100700000D2C06D01A2C04D0FF222146002003F025
:1007100039F8601CC4B2242CEEDBE4E0FCF7B2F83C
:10072000002406E000222146104603F02BF8601C4E
:10073000C4B2242CF6DBD6E0FCF776F901287BD195
:10074000FCF758F96949884278D300F00BFB06465C
:1007500000F022FB07460A21F7F7F8FC054632466F
:10076000294601200BF08AF900F060FD064600F0F2
:10077000E1FC0A210290F7F7E9FC054600F0F2FAE5
:1007800007463246294609F007F9FFF731FF00F026
:10079000CBFA05462946012007F044FC00F0F6FAA2
:1007A0000646FF21F531F7F7E7FCC5B229460120DF
:1007B00006F064FBFFF722FD0546FFF72BFD06461A
:1007C000FFF732FD07462B4632463946012005F039
:1007D00073FE00F005F90546294601200BF0F4FBF5
:1007E00000F0CEFC054600F0C7FB064600F0CEFC4C
:1007F000074600F0C7FB00233A46014600960195E4
:10080000029001200AF056FEFF220321002002F090
:10081000B9FFFF220421002002F0B4FF00F07EFCAB
:10082000054600F075FC064600F07EFC07462A46A9
:10083000314607F02BFE56E00DE0FFE7FF220321D3
:10084000002002F09FFFFF220421002002F09AFF07
:10085000FBF746FF47E0FCF715F80022032110469E
:1008600002F090FF00220421104602F08BFF0022CC
:100870002321104602F086FF00222221104602F0BA
:1008800081FF00220721104602F07CFF0022082190
:10089000104602F077FF00220921104602F072FF95
:1008A00000220A21104602F06DFF0022132110469B
:1008B00002F068FF00221121104602F063FF0022BF
:1008C0001221104602F05EFF00220E21104602F0B7
:1008D00059FF00220F21104602F054FF0022102180
:1008E000104602F04FFFFEBDF1000020B80B0000E3
:1008F0000149086070470000900700200248006826
:10090000401C0149086070478C070020F3B581B096
:10091000064600200E49086000F01EF8044600F06C
:100920001BF805462F1B3046029903F03DFF00904F
:100930000AE000F011F805462F1B06480068002861
:1009400002D004480068804700988742F1D3FEBD7A
:100950008C070020900700200148006870470000C5
:100960008C0700200B490978012901D101200FE0F3
:1009700008490978022901D1022009E005490978CE
:10098000032901D1042003E00121024A1170012052
:10099000704700001D07002010B5094B1B8899B255
:1009A0000A12C8B2D3433133064C2370C3432333F6
:1009B000637013465633A37003467133E37010BD62
:1009C00054070020230700200148008870470000DA
:1009D0001C000020014800887047000034000020FF
:1009E00001480078704700008D0000200148007821
:1009F000704700008E00002010B500220521064837
:100A0000FAF778FB0402012205210348FAF772FB8A
:100A1000201880B210BD00006008002010B506222A
:100A200005210348FAF766FBC006C00F10BD0000A1
:100A30006008002010B5042205210648FAF75AFB89
:100A40000402052211460348FAF754FB201880B22D
:100A500010BD00006008002010B5062205210248E4
:100A6000FAF748FBC01110BD6008002010B5022243
:100A700005210248FAF73EFB10BD00006008002087
:100A800010B5062205210348FAF734FB8006C00F93
:100A900010BD00006008002010B5042202210348A8
:100AA000FAF728FBC007C00F10BD00006008002047
:100AB00010B5052202210348FAF71CFBC007C00F3E
:100AC00010BD00006008002010B50022042103487A
:100AD000FAF710FB4006400F10BD00006008002030
:100AE00010B5042201210248FAF704FB801110BD61
:100AF0006008002010B5002201210248FAF7FAFA36
:100B000010BD00006008002010B505220121034837
:100B1000FAF7F0FA8007800F10BD0000600800208F
:100B200010B5012211460248FAF7E4FA10BD0000A0
:100B30006008002010B5002206210C48FAF7DAFA06
:100B40000402012206210948FAF7D4FA2018040207
:100B5000022206210548FAF7CDFA201804020322E2
:100B600006210248FAF7C6FA201810BD60080020D6
:100B700010B5042206210C48FAF7BCFA040205223B
:100B800006210948FAF7B6FA20180402062211468F
:100B90000548FAF7AFFA2018040207220621024896
:100BA000FAF7A8FA201810BD6008002010B502223C
:100BB00003210248FAF79EFA10BD000060080020E9
:100BC00010B5032200210248FAF794FA10BD000084
:100BD0006008002010B5002211460248FAF78AFA90
:100BE00010BD00006008002010B50422002102485A
:100BF000FAF780FA10BD00006008002010B501224D
:100C000000210248FAF776FA10BD000060080020C3
:100C100010B5052200210248FAF76CFA10BD000059
:100C2000600800200146322915DA3E488078012804
:100C300003DD01203B4A507070E03A48807800287C
:100C400005DD2F296ADC0020364A507066E000205E
:100C5000344A507062E03E2917DA322915DB3148F8
:100C60008078022803DD02202E4A507056E02D487D
:100C70008078012805DD3B2950DC0120294A50708D
:100C80004CE00120274A507048E0502917DA3E29ED
:100C900015DB24488078032803DD0320214A5070A7
:100CA0003CE020488078022805DD4D2936DC022012
:100CB0001C4A507032E002201A4A50702EE062291D
:100CC00017DA502915DB17488078042803DD042043
:100CD000144A507022E013488078032805DD5F290C
:100CE0001CDC03200F4A507018E003200D4A50709E
:100CF00014E073290FDA62290DDB0A488078042892
:100D000005DD70290ADC0420064A507006E0042044
:100D1000044A507002E00520024A507001484078B1
:100D200070470000502600200148007870470000FE
:100D3000070000200148006870470000901F002055
:100D40000148007870470000E50000200148007865
:100D500070470000E4000020014800787047000060
:100D6000E900002001480079704700004C2800206D
:100D70000148407870470000E90000200148007AEF
:100D8000704700004C280020002070470148008870
:100D9000704700001E00002010B50024FFF7E2FF9E
:100DA00000280AD10A4800880A49884202DB08461E
:100DB000074908800648048808E005480088FCF7D1
:100DC000E9FB84B20448844200DB0446204610BD9F
:100DD00036000020C6070000CE04000000200549B0
:100DE0000988054A914202DB1146024A11800149F5
:100DF0000888704736000020C6070000F8B50027B5
:100E0000002500260024FFF7E5FE0546FFF7F6FE65
:100E10000646F020284000110A2805DBF020284073
:100E20000011C01C044303E0F020284000110443DB
:100E300024022807000F0A2804DB2807000FC01C23
:100E4000044302E02807000F04432402F02030404E
:100E500000110A2805DBF02030400011C01C0443BB
:100E600003E0F02030400011044324023007000F5B
:100E70000A2804DB3007000FC01C044302E03007DF
:100E8000000F0443002C01D10248F8BD2746384624
:100E9000FBE70000FFFF0000F8B500270025002653
:100EA0000024FFF7A1FE0546FFF7B2FE0646F0203C
:100EB000284000110A2805DBF02028400011C01C42
:100EC000044303E0F02028400011044324022807D3
:100ED000000F0A2804DB2807000FC01C044302E0AF
:100EE0002807000F04432402F020304000110A2894
:100EF00005DBF02030400011C01C044303E0F0206B
:100F000030400011044324023007000F0A2804DB9C
:100F10003007000FC01C044302E03007000F0443F9
:100F2000002C01D10248F8BD27463846FBE70000F7
:100F3000FFFF000010B50024FFF742FE04462046E4
:100F400010BD012070470000014800787047000084
:100F50005D07002001480078704700005F0700200F
:100F60000148C07B70470000C80900200148C07CD0
:100F700070470000C80900200148007A704700004F
:100F8000C809002010B5002405480088323084B21A
:100F900064212046F7F7F0F884B2204610BD000027
:100FA000C809002070B5002407490868FBF75CFEFB
:100FB00005466421F7F7CAF884B20448844200DD8C
:100FC0000446204670BD0000C8090020DE03000072
:100FD00010B5002400F014F8012800D10CE000F056
:100FE0000FF8022802D1FF24373405E00A21034814
:100FF0000088F7F7C1F884B2204610BD0200002037
:1010000001480078704700000B00002000200549CF
:101010000968002903D003490968086800E002480C
:1010200070470000700100203075000010B50024EA
:10103000044804F037FC002801D0012400E000241B
:10104000204610BD0407000010B50024044804F039
:1010500029FC002801D0012400E00024204610BD16
:101060000507000010B50024044804F01BFC00280C
:1010700001D0012400E00024204610BD0707000035
:1010800010B50024062004F00DFC002801D0012436
:1010900000E00024204610BD10B50024052004F017
:1010A00001FC002801D0012400E00024204610BDEE
:1010B00010B50024044804F0F5FB002801D00124F9
:1010C00000E00024204610BD0607000010B50024F3
:1010D000044804F0E7FB002801D0012400E00024CC
:1010E000204610BD0305000010B50024044804F09C
:1010F000D9FB002801D0012400E00024204610BDC7
:10110000040500000148807A70470000C8090020EB
:101110000148807870470000600A0020014840685C
:1011200070470000600A00200148407870470000C6
:10113000600A002070B50024FFF714FE002803D1D8
:10114000FCF73CFC04460DE0FFF70CFE012806D13D
:10115000FCF734FC0546FCF71DFA044602E0FCF7F8
:101160002DFC0446204670BD0148007C70470000FD
:10117000C80900200148007D70470000C809002010
:101180000148407A70470000C809002010B50024CB
:1011900005488088323084B264212046F6F7ECFF9F
:1011A00084B2204610BD0000C809002070B500249C
:1011B00007494868FBF758FD05466421F6F7C6FF66
:1011C00084B20448844200DD0446204670BD00001D
:1011D000C8090020DE03000070B50BF003FA0546D5
:1011E0000BF000FA04490860002D01D1012400E051
:1011F0000024204670BD00007C0100200148007BD7
:1012000070470000C80900200148407B704700007B
:10121000C80900200148807B70470000C8090020F1
:101220000148007870470000E800002070B50024F5
:10123000FFF798FD002803D1FCF7E2FB04460FE01E
:10124000FFF790FD012807D10020FCF7D9FB0546E8
:10125000FCF7A0F9044603E00020FCF7D1FB0446AC
:10126000204670BD01480078704700003E00002015
:1012700070B505460024032D00D170BD002D01D0AE
:10128000012D1BD181210320800204F0BBFA8021B3
:10129000134804F0B7FA32211248FFF737FB002455
:1012A00009E0A200104BD2189178A200985A04F0DD
:1012B000A9FA601CC4B23B2CF3DB0FE0022D0DD168
:1012C000002409E0A200094BD2189178A200985A94
:1012D00004F098FA601CC4B23B2CF3DB00BFCCE7EF
:1012E00002060000A0860100601602004C170200F2
:1012F000F8B5002100240023002200BF0AE00125E8
:101300008D40ABB205881D402C469C4200D10A4658
:101310004D1CA9B21029F2DB0588FF2D1FDC284DDA
:101320006D7E0688B543264E757635462D7E068839
:10133000B543234E357635466D7E8678F607F60F33
:10134000964035431E4E757635462D7E86780227AB
:101350003E40760896403543194E357622E0184DCA
:10136000ED7E0688B543164EF5763546AD7E068889
:10137000B543134EB5768578ED07ED0F1646083E5A
:10138000B5400F4EF67E35430D4EF5768578022634
:1013900035406D081646083EB540094EB67E3543C9
:1013A000074EB5760025009505E000BF6D462D7807
:1013B0006D1CEEB200966D462D78012DF5D9F8BD65
:1013C000206B0440C107C90F002905D00021394A0C
:1013D0001171002238490A7102210140002905D00B
:1013E0000021344A1172002233490A72042101405B
:1013F000002905D000212F4A117300222E490A73BB
:1014000008210140002905D000212A4A1174002238
:1014100029490A7410210140002905D00021254ADC
:101420001175002224490A7520210140002905D0A8
:101430000021204A117600221F490A7640210140EE
:10144000002904D000221B494A711B494A7180219E
:101450000140002904D0002216494A7216494A72F6
:10146000FF2101310140002904D0002211494A73B3
:1014700011494A73012149020140002904D0002288
:101480000C494A740C494A7401218902014000291F
:1014900004D0002207494A7507494A750121C9024B
:1014A0000140002904D0002202494A7602494A76C6
:1014B000704700000060004000610040C107C90F94
:1014C000002905D001223C490A7100213B4A1171D3
:1014D00002210140002905D0012237490A7200216A
:1014E000364A117204210140002905D001223249F7
:1014F0000A730021314A117308210140002905D0E7
:1015000001222D490A7400212C4A11741021014036
:10151000002905D0012228490A750021274A1175A2
:1015200020210140002905D0012223490A7600210B
:10153000224A117640210140002905D001221E498E
:101540004A7100221D494A7180210140002905D0BD
:10155000012219494A72002218494A72FF210131B9
:101560000140002905D0012213494A730022134982
:101570004A73012149020140002905D001220E4988
:101580004A7400220D494A74012189020140002950
:1015900005D0012208494A75002208494A750121EF
:1015A000C9020140002905D0012203494A760022E0
:1015B00002494A7670470000006100400060004028
:1015C00010B50C480078002803D00B4A5068916889
:1015D000884708484078002803D0084A5068916836
:1015E000884704488078002803D0054A50689168ED
:1015F000884710BD006000400803002088040020D8
:101600000806002010B508480079002803D0074AD2
:1016100010695169884704484079002803D0044A7A
:1016200050689168884710BD0060004008030020A2
:101630009404002010B50848007A002803D0074A17
:10164000D069116A88470448407A002803D0044AC8
:1016500050689168884710BD006000400803002072
:10166000A004002010B50848007B002803D0074ADA
:10167000906AD16A88470448407B002803D0044A16
:1016800050689168884710BD006000400803002042
:10169000AC04002010B50848007C002803D0074A9D
:1016A000506B916B88470448407C002803D0044A63
:1016B00050689168884710BD006000400803002012
:1016C000B804002010B50848007D002803D0074A60
:1016D000106C516C88470448407D002803D0044AB0
:1016E00050689168884710BD0060004008030020E2
:1016F000C404002010B50848007E002803D0074A23
:10170000D06C116D88470448407E002803D0044AFD
:1017100050689168884710BD0060004008030020B1
:10172000D004002010B50848407F002803D0074AA5
:101730005068916888470448007F002803D0044A15
:10174000906DD16D884710BD00600040DC04002022
:101750000803002010B508484078002803D0074A45
:1017600050689168884704480078002803D0044AEC
:10177000506E916E884710BD20600040E804002044
:101780000803002010B509480079002803D0084A52
:10179000106F516F88470548001D4078002803D01E
:1017A000044A50689168884710BD000020600040DE
:1017B00008030020F404002010B5034AD06F7832EB
:1017C0009168884710BD00000803002010B5024A48
:1017D00050689168884710BD8C03002010B50948F7
:1017E000007C002803D0084A506891688847054863
:1017F00010304078002803D0044A50689168884728
:1018000010BD000020600040980300201805002053
:1018100010B5024A50689168884710BDA4030020A3
:1018200010B5024A50689168884710BDB003002087
:1018300010B50948007F002803D0084A5068916815
:10184000884705481C304078002803D0044A506877
:101850009168884710BD000020600040BC03002054
:101860003C05002010B50C480078002803D00B4A36
:1018700050689168884708484078002803D0084A93
:1018800050689168884704488078002803D0054A4A
:1018900050689168884710BD40600040C803002030
:1018A00048050020C806002010B50D480079002822
:1018B00003D00C4A5068916888470948001D407859
:1018C000002803D0084A5068916888470448001DE2
:1018D0008078002803D0054A50689168884710BD79
:1018E00040600040D403002054050020D4060020AE
:1018F00010B50D48007A002803D00C4A5068916852
:101900008847094808304078002803D0084A5068C2
:1019100091688847044808308078002803D0054A39
:1019200050689168884710BD40600040E003002087
:1019300060050020E006002010B50D48007B00285F
:1019400003D00C4A50689168884709480C304078A9
:10195000002803D0084A50689168884704480C3032
:101960008078002803D0054A50689168884710BDE8
:1019700040600040EC0300206C050020EC060020D5
:1019800010B50D48007C002803D00C4A50689168BF
:101990008847094810304078002803D0084A50682A
:1019A00091688847044810308078002803D0054AA1
:1019B00050689168884710BD40600040F8030020DF
:1019C00078050020F806002010B5024A506891689A
:1019D000884710BD0404002010B50948007E002887
:1019E00003D0084A50689168884705481830407805
:1019F000002803D0044A50689168884710BD000051
:101A000040600040100400209005002010B50948F7
:101A1000007F002803D0084A50689168884705482D
:101A20001C304078002803D0044A506891688847E9
:101A300010BD0000406000401C0400209C050020F8
:101A400010B508480078002803D0074A506891680C
:101A5000884704484078002803D0044A50689168B9
:101A6000884710BD6060004028040020A8050020C1
:101A700010B509480079002803D0084A50689168D9
:101A800088470548001D4078002803D0044A506864
:101A90009168884710BD0000606000403404002059
:101AA000B405002010B50948007A002803D0084A80
:101AB000506891688847054808304078002803D06E
:101AC000044A50689168884710BD0000606000407B
:101AD00040040020C005002010B5024A50689168FB
:101AE000884710BD4C04002010B5024A5068916828
:101AF000884710BD5804002010B50948007D002813
:101B000003D0084A506891688847054814304078E7
:101B1000002803D0044A50689168884710BD00002F
:101B20006060004064040020E405002010B509480E
:101B3000007E002803D0084A50689168884705480D
:101B400018304078002803D0044A506891688847CC
:101B500010BD00006060004070040020F00500200F
:101B600010B50948007F002803D0084A50689168E2
:101B7000884705481C304078002803D0044A506844
:101B80009168884710BD0000606000407C04002020
:101B9000FC05002010B5FE4800688079002806D0BA
:101BA00001286ED002286DD003286CD104E2F848D9
:101BB0000068407903000EF085FF0A0614BC2BBCB8
:101BC00047BC67BC9BBC0AF0D7FF0020F0490968FE
:101BD000C873EF4800684079401CED4909684871B6
:101BE000AEE0EC490969EA4A1268D27A885C0BF0E7
:101BF0003BF8E74800684079401CE54909684871AE
:101C0000E34800684079401CE1490968487197E061
:101C100001F020FF002810D10BF026F8DC48006806
:101C20004079401CDA4909684871D9480068407910
:101C3000401CD7490968487105E00AF0C7FF002039
:101C4000D349096848717BE001F004FF002811D1F5
:101C500001200BF009F8CE4800684079401CCC49BF
:101C600009684871CA4800684079401CC849096839
:101C7000487105E00AF0AAFF0020C54909684871CB
:101C80005EE05FE0FEE0A3E101F0E4FE002828D181
:101C9000BF490968C97A24225143BF4A126889188A
:101CA000BB4A1268D27B885C0AF0DEFFB848006845
:101CB000C07B401CB6490968C873B5480068C07B42
:101CC000242814D3B24800684079401CB049096800
:101CD0004871AF4800684079401CAD4909684871B7
:101CE00005E00AF073FF0020A9490968487127E060
:101CF00001F0B0FE002815D1A5480068C07A401C4C
:101D0000A3490968C872A2480068C07AA149097845
:101D1000884207DB00209E490968C87201209C495F
:101D2000096888710AF052FF0020994909684871D2
:101D300006E00AF04BFF002095490968487100BF92
:101D400000BF4FE192480068407903000EF0BAFEF0
:101D5000080513912A91479170910AF00DFF002018
:101D60008B490968C8738A4800684079401C8849D3
:101D70000968487184E087490969854A1268D27AFE
:101D8000885C0AF071FF824800684079401C8049F5
:101D9000096848717E4800684079401C7C490968A0
:101DA00048716DE001F056FE002811D126200AF09E
:101DB0005BFF774800684079401C754909684871A5
:101DC000734800684079401C71490968487105E012
:101DD0000AF0FCFE00206E490968487150E001F0ED
:101DE00039FE00281DD101200AF03EFF6848006836
:101DF000C07B401C66490968C87365480068C07BA1
:101E0000242814D3624800684079401C604909685E
:101E100048715F4800684079401C5D490968487115
:101E200005E00AF0D3FE002059490968487127E00F
:101E300001F010FE002815D155480068C07A401CFA
:101E400053490968C87252480068C07A51490978F4
:101E5000884207DB00204E490968C87202204C49BD
:101E6000096888710AF0B2FE002049490968487182
:101E700006E00AF0ABFE002045490968487100BF42
:101E800000BFAFE042480068407903000EF01AFE40
:101E90000805138B2A8B478B638B0AF06DFE00209D
:101EA0003B490968C8733A4800684079401C384982
:101EB000096848717EE037490969354A1268D27A63
:101EC000885C0AF0D1FE324800684079401C3049F5
:101ED000096848712E4800684079401C2C490968FF
:101EE000487167E001F0B6FD002811D125200AF005
:101EF000BBFE274800684079401C254909684871A5
:101F0000234800684079401C21490968487105E070
:101F10000AF05CFE00201E49096848714AE001F0A1
:101F200099FD002810D10AF09FFE194800684079F9
:101F3000401C174909684871154800684079401CE1
:101F400013490968487105E00AF040FE0020104975
:101F5000096848712EE001F07DFD002815D10C487C
:101F60000068C07A401C0A490968C87208480068BD
:101F7000C07A08490978884207DB002004490968CB
:101F8000C87203200249096888710AF01FFE05E043
:101F9000E00700204C2F0020DC0700200020124921
:101FA0000968487106E00AF011FE00200E49096830
:101FB000487100BF00BF15E000200B490968887117
:101FC000094909684871062007490968C87009E08D
:101FD0000AF0FCFD002004490968487102490968BB
:101FE000887100BF00BF10BDE007002010B56A482F
:101FF0000068407903000EF065FD090610C627C68B
:1020000044C6608EC6000AF0B7FD63480068407998
:10201000401C614909684871BCE0604909695E4A31
:102020001268D27A885C0AF01FFE5B48006840792B
:10203000401C594909684871574800684079401C5C
:10204000554909684871A5E001F004FD002811D147
:102050004F200AF009FE504800684079401C4E4964
:10206000096848714C4800684079401C4A49096831
:10207000487105E00AF0AAFD002047490968487147
:1020800088E001F0E7FC002810D10AF0EDFD42489D
:1020900000684079401C4049096848713E48006822
:1020A0004079401C3C490968487105E00AF08EFD02
:1020B00000203949096848716CE001F0CBFC002828
:1020C00022D135480068C07A401C33490968C8727B
:1020D00031480068C07A3149097888420FDB002016
:1020E0002D490968C8722C4800684079401C2A496B
:1020F00009684871002028490968486208E0002002
:1021000025490968487103E000202349096848719E
:102110000AF05CFD3EE020480068407C002816D0B4
:102120001E48C068002803D01C48C1681920884791
:102130000020194909684862174909684871164919
:1021400009688871052014490968C8701AE01248A6
:102150000068406A282807D20F480068406A401C7F
:102160000D49096848620DE000200B490968486282
:1021700009490968487108490968887105200649B4
:102180000968C87006E00AF021FD002002490968CC
:10219000487100BF00BF10BDE00700204C2F002099
:1021A00010B50024F7480068807A01287ED1F548F0
:1021B0000068C07900287AD0F24800688079002849
:1021C00004D0012874D0022873D191E1ED48006851
:1021D000007B24286ED2EB480068C07901287AD1B0
:1021E000002475E0E7480068C07A24214843E649A6
:1021F00009684018E3490968097B415CE1480068C7
:10220000C07A24225043E14A12688018DD4A1268DD
:10221000127B805C814229D0DA480068C07A242190
:102220004843DA4909684018D6490968097B415C86
:10223000D4480068C07A24225043D34A12688018D8
:10224000D04A1268127B8154CE480068407B242813
:1022500005D3CC480068007BCA4909684873C9485F
:102260000068007BC7490968887308E0C5480068B2
:10227000407B242803D20120C24909688871C148E3
:102280000068007B401CBF4909680873BD480068AE
:10229000007B242808D3BB480068407B242803D255
:1022A0000120B84909688871B64805E0D3E1CDE15D
:1022B00069E0BAE138E00EE00068007B242804D22F
:1022C000B04800688079012800D103E0601CC4B2E6
:1022D000242C87D356E0002413E0AA480068C07A73
:1022E00024214843A94909684018015DA5480068B0
:1022F000C07A24225043A44A126880180155601CF9
:10230000C4B2242CE9D300209E49096848732320D5
:102310009C490968887301209A49096888712420BA
:102320009849096808732DE00020964909680873E8
:1023300094480068C07A401C92490968C872914864
:102340000068C07A92490978884217DB8D48006896
:10235000007C012804D102208A490968887106E0BE
:10236000002088490968887186490968C871002079
:1023700084490968C8728349096808740020814942
:102380000968487161E17F480068407903000EF0F8
:1023900099FB080513A62AA651A68EA60120794905
:1023A000096808740AF0E8FB764800684079401C28
:1023B00074490968487199E075490969714A126858
:1023C000D27A885C0AF050FC6E4800684079401C64
:1023D0006C49096848716B4800684079401C69493C
:1023E0000968487182E001F035FB00281BD165497E
:1023F0000968497B491CC8B20AF036FC614800688C
:10240000407B60490968C8735E4800684079401C99
:102410005C49096848715B4800684079401C59492B
:102420000968487105E00AF0D1FB002055490968A8
:1024300048715BE001F00EFB00282BD1514909687F
:10244000C97A24225143504A126889184D4A1268A9
:10245000D27B885C0AF008FC4A480068C07B401CBC
:1024600048490968C87347480068C07B45490968FE
:10247000897B88421ADD434800684079401C414905
:10248000096848713F4800684079401C3D49096827
:1024900048710BE00AF09AFB3A480068407B3949E2
:1024A0000968C87300203749096848711EE001F0C7
:1024B000D1FA00280CD133490968887124203149A8
:1024C0000968C8732F49096848732E4909688873D9
:1024D0000AF07CFB00202B490968487106E00AF0ED
:1024E00075FB002027490968487100BF00BFACE0B8
:1024F00024480068407903000EF0E4FA08050F8EC6
:10250000268E4C8E688E0AF037FB1E480068407994
:10251000401C1C490968487185E01D490969194A30
:102520001268D27A885C0AF09FFB164800684079EE
:10253000401C144909684871124800684079401CE1
:102540001049096848716EE001F084FA002811D141
:1025500025200AF089FB0B4800684079401C094996
:1025600009684871074800684079401C05490968B6
:10257000487105E00AF02AFB002002490968487109
:1025800051E00000E0070020DC070020D807002011
:102590004C2F002001F05EFA002810D10AF064FBF5
:1025A000644800684079401C624909684871614884
:1025B00000684079401C5F490968487105E00AF0ED
:1025C00005FB00205B49096848712CE001F042FAE4
:1025D00000281AD157480068C07A401C554909683C
:1025E000C87254480068C07A5349097888420CDBA5
:1025F000002050490968C8724E49096888714D49E0
:10260000096848714B490968C8710AF0DFFA00206F
:1026100048490968487106E00AF0D8FA002045499F
:102620000968487100BF00BF0FE00AF0CFFA002030
:102630004049096848713F49096888713D490968FE
:1026400008733C490968C87200BF71E0002039492D
:10265000096888726CE037480068807A022867D180
:1026600034480068007A00285ED03248006840791B
:10267000002804D001280CD0032846D11BE00AF022
:102680007BFA2C4800684079401C2A490968487147
:1026900049E000200AF0E8FA264800684079401C2A
:1026A000244909684871234800684079401C214941
:1026B0000968487137E00AF029FA002812D11D484C
:1026C00000684078401C1B49096848701948006838
:1026D0004078032812D301F05DFA002015490968FB
:1026E00048700BE00020134909680872AA201149BC
:1026F0000968887000200F49096848700AF066FA76
:1027000000200C49096848710DE00AF05FFA0020CA
:10271000084909684871074909684870AA200549AD
:102720000968887000BF03E00020024909688872C8
:1027300010BD0000E00700204C2F0020F8B5044633
:102740000D4600260C2060431D49085C002801D07E
:102750000120F8BD0C2060431949401885600C2009
:10276000604340188068002801D10120F1E7012171
:102770000C206043124A115400222046E317DB0E5E
:102780001B185B115B01E31A9B000E4FDB19E71767
:10279000FF0E3F197F11DA550EF0C6F900222046D0
:1027A000E317DB0E1B185B115B01E31A9F00064B5E
:1027B000FB18E717FF0E3F197F11DA553046C8E7BF
:1027C00008030020006000400061004000BFFEE7F9
:1027D00009480088401C08490880084600880749C5
:1027E000884208DD06480078002804D008460249DF
:1027F0000880012088707047E0000020DC050000A0
:10280000E400002010B515488078012824D1144830
:10281000007801280CD113480078012808D1002045
:1028200011498870084602F00BFE00200D4908701F
:102830000B48007802280CD10C480078012808D1F8
:10284000002009498870084602F0FAFD0020074977
:10285000087000200249087010BD0000E000002050
:10286000E4000020E6000020E9000020E70000204E
:102870007047000010B500F05DFE012803D1002074
:1028800001490880887010BDE0000020F0B50546C1
:102890000E46174600243A463146284600F058FEB8
:1028A00000BF42E000202101394A12685052210144
:1028B000374A12688918488000212001344A12687A
:1028C000801881802001324A12688018C18020015E
:1028D0002F4A12688018017220012D4A1268801850
:1028E000417220012A4A1268801881722001284A08
:1028F00012688018C17200202101254A12688918C7
:10290000087300212001224A1268801841730020B8
:1029100021011F4A126889188873002120011C4A6E
:1029200012688018C173601CC4B21A484078A04273
:10293000B8DC64201849096808807D20C000164969
:102940000968488015481449096888807D2000017D
:1029500011490968C88010490968088110480E4962
:10296000096848810F480C490968888140000A4974
:102970000968C8813220084909680882FF20F530BB
:10298000054909684882044909688882F0BD000049
:10299000A0070020940700209C0700204C040000A2
:1029A000102700003075000038B5002404E0002036
:1029B00013490855601C84B2282CF8D301216846BD
:1029C000417001706A460F490D48FFF75FFF7D2196
:1029D000C900322000F0ACF90B490C4800F0C6F9F0
:1029E0000948643000F058F90748C83000F064F92D
:1029F000074800F077F9074800F08AF938BD000071
:102A00005C280020341C020028230000B80B0000C2
:102A1000542400001027000010B524480078002836
:102A200003D10120214908703EE0204800780128A8
:102A300010D11F480078012808D100201D49887056
:102A4000084602F0FDFC00201949087002201749D1
:102A5000087029E015480078022810D1164800783F
:102A6000012808D1002013498870084602F0E8FCCC
:102A700000201149087003200C49087014E00B482D
:102A80000078032803D10520084908700CE00748A6
:102A90000078052803D005480078062804D10020D6
:102AA000024908700549087010BD0000E4000020CC
:102AB000E6000020E9000020E7000020E8000020F8
:102AC000F8B50024002500263548007800281ED1DE
:102AD00034480078002803D101203249087016E0FC
:102AE00030480078012803D102202E4908700EE0FA
:102AF0002C480078022803D103202A49087006E0F8
:102B000028480078032802D100202649087024486C
:102B1000007801280ED10124172500262248012320
:102B2000324629460090204601F09CFE01201F49B4
:102B3000087034E01A48007802280FD101243B25A0
:102B400000261948401C01233246294600902046A1
:102B500001F088FE01201649087020E01048007836
:102B600003280DD1FEF7FEF8002803D101201149FA
:102B7000087102E000200F4908710DF075FF0EE0AA
:102B800007480078052803D106200549087006E0AB
:102B900003480078062802D1052001490870F8BDD5
:102BA000E4000020E5000020E9000020E60000200D
:102BB000E70000204C28002010B5044623000DF04B
:102BC00081FF095B060E16171819595A5E00F9F7AE
:102BD00011FF2C49884201D3FFF772FF50E0F9F74B
:102BE00009FF2849884201D3FFF716FF48E047E074
:102BF00046E045E0F9F7FEFE2249884239D301F06C
:102C0000E1FD21480078032814D1204800780028ED
:102C100010D1FEF7B3F8002806D101201C498860C6
:102C20008868FAF757FF05E000201949886088682E
:102C3000FAF750FF14480078012805D113480078AE
:102C4000002801D1FAF768F810480078052803D168
:102C50000120104908700AE00C480078062803D1CA
:102C600002200C49087002E000200A4908700BF0AD
:102C70009BFC05E004E003E0FFF7AAFD00E000BFD5
:102C800000BF10BDB80B0000E5000020E4000020EC
:102C90004C280020E800002001460020054A126868
:102CA00052898A4201DC012002E0024A1268118145
:102CB000704700009C07002001460020084A126867
:102CC00012898A4201DB012009E0054A12689289D3
:102CD0008A4201DC012002E0014A126851817047FA
:102CE0009C07002001460020084A126852898A4247
:102CF00001DB012009E0054A1268D2898A4201DC21
:102D0000012002E0014A1268918170479C0700206F
:102D100001460020054A126892898A4201DB01209F
:102D200002E0024A1268D181704700009C0700202F
:102D3000024600200C4B1B681B8A934201DD0120D8
:102D400010E08A4201DB01200CE0074B1B689B88E6
:102D50008B4201DC012005E0034B1B681A80024B0B
:102D60001B685980704700009C0700200246002025
:102D70000C4B1B681B8A934201DD012010E08A4244
:102D800001DB01200CE0074B1B685B88934201DBF1
:102D9000012005E0034B1B689A80024B1B68D98019
:102DA000704700009C07002070B5044600250C20E9
:102DB0006043FE49096840184068002807D00C218C
:102DC0006143FA4A126889184868804705460C2012
:102DD0006043F6490968085C002873D10C20604301
:102DE000F249096840188068002874D02001F04931
:102DF00009684018C07A02280AD1032D08D10C2096
:102E00006043EA4A1268801881680120884762E0BE
:102E10002001E74909684018C07A02280AD1042D28
:102E200008D10C206043E14A1268801881680220B2
:102E3000884750E02001DE4909684018C07A02281E
:102E40000AD1052D08D10C206043D84A1268801899
:102E50008168032088473EE02001D5490968401871
:102E6000C07A02280AD1062D08D10C206043CF4A2F
:102E7000126880188168042088472CE02001CC4922
:102E800009684018C07A02280AD1072D08D10C2001
:102E90006043C64A126880188168052088471AE096
:102EA0002001C34909684018C07A02280BD1082DB7
:102EB00009D10C206043BD4A126880188168062041
:102EC000884708E00DE00C206043B84A126880187B
:102ED0008168002088472001B54909684018C572FB
:102EE0000CE30C206043B1490968085C012873D1E8
:102EF0000C206043AD49096840188068002874D0F0
:102F00002001AB4909684018C07A03280AD1022D74
:102F100008D10C206043A54A1268801881680120FE
:102F2000884762E02001A24909684018C07A042855
:102F30000AD1022D08D10C2060439C4A12688018E7
:102F400081680220884750E02001994909684018AB
:102F5000C07A05280AD1022D08D10C206043934A7B
:102F6000126880188168032088473EE0200190495C
:102F700009684018C07A06280AD1022D08D10C2011
:102F800060438A4A126880188168042088472CE0D0
:102F90002001874909684018C07A07280AD1022D04
:102FA00008D10C206043814A12688018816805208E
:102FB00088471AE020017E4909684018C07A08282D
:102FC0000BD1022D09D10C206043784A1268801879
:102FD00081680620884708E00DE00C206043734AB2
:102FE00012688018816800208847200170490968AC
:102FF0004018C57282E20C2060436C490968085C85
:103000000228F7D1002D7DD1200169490968085AAD
:1030100068490968098A884275DA200164490968A3
:10302000085A0A3081B22001614A12681152200107
:103030005F490968085A5F490968098A884231DB93
:1030400020015B490968401840885A490968098885
:10305000884227DB200156490968401840885549B5
:103060000968498888421DDC00202101504A126805
:103070008918488020014E4909684018807A002844
:10308000B8D10C206043494909684018806800287D
:10309000B0D00C206043454A126880188168012036
:1030A00088472BE2200142490968085A41490968CA
:1030B000098A88429EDB20013D4909684018408802
:1030C0003C4909688988884294DB200138490968AD
:1030D0004018408837490968C98888428ADC00203E
:1030E0002101334A12688918488020013049096853
:1030F0004018807A0028D4D10C2060432B490968FD
:10310000401801E063E00BE080680028C9D00C2083
:103110006043264A12688018816802208847EDE1E2
:1031200000202101224A1268891848802101204A82
:1031300012688918C872002120011D4A126880187F
:10314000C18020011A4A1268801841722001184A71
:10315000126880188172184801782001144A126898
:103160008018017200202101114A12688918888094
:1031700021010F4A12688918087321010C4A12684C
:103180008918487321010A4A126889188873002136
:103190002001074A12688018C1730C20604303495C
:1031A0000968401880680028B9D007E09807002017
:1031B000A00700209C070020940700200C206043FB
:1031C000CF4A1268801881680020884796E1012D57
:1031D000A5D12001CB4909684018C07AA84225D062
:1031E00000212001C74A1268801841800020210177
:1031F000C44A12688918C8802001C2490968401869
:10320000C572C14800782101BE4A12688918487207
:1032100000202101BB4A126889188880BA480178C9
:103220002001B84A12688018017267E12001B5498F
:1032300009684018007AB4490978884220D0B24819
:1032400000782101AF4A1268891808722001AD493F
:1032500009684018407AAC490978884209D02001B1
:10326000A8490968401880882101A64A126889186F
:10327000C88000212001A34A12688018818012E0D2
:103280002001A049096840188088A04988420AD2D4
:1032900020019C490968401880880A302101994A18
:1032A000126889188880200196490968401840886A
:1032B000964988420AD220019249096840184088FC
:1032C0000A3021018F4A12688918488020018D49EF
:1032D00009684018407A8C490978884205D0012055
:1032E0002101884A12688918887220018549096875
:1032F00040184088864909680988884204DB002113
:103300002001804A1268115220017E490968401844
:10331000807A00287ED10C206043794909684018E2
:103320008068002877D020017649096840184088D5
:10333000774909680989884214DB200171490968C5
:103340004018007B00280DD10C2060436C4A1268A5
:10335000801881680320884701202101694A12688A
:10336000891808732001674909684018408868492E
:1033700009684989884214DB2001624909684018BC
:10338000407B00280DD10C2060435D4A12688018F4
:10339000816804208847012021015A4A126889184F
:1033A00048732001574909684018408858490968FE
:1033B0008989884214DB2001524909684018807BC2
:1033C00000280DD10C2060434D4A12688018816896
:1033D00005208847012021014A4A1268891888730C
:1033E0002001484909684018408849490968C98945
:1033F000884210DB2001434909684018C07B00283F
:103400007CD10C2060433E4A1268801881680620F7
:10341000884701E007E03BE001202101394A1268BA
:103420008918C8736AE02001364909684018407A53
:1034300001282ED13448007802282AD120013149B0
:1034400009684018C08832490968498A884255DBB2
:1034500020012C490968401880882D490968898A0B
:1034600088424BDB0C20604325490968401880687E
:10347000002843D00C206043214A126880188168DC
:1034800007208847002021011E4A126889184872C7
:1034900034E020011B4909684018407A02282DD1E8
:1034A00019480078012829D12001164909684018D7
:1034B000C08817490968898A88421FDB20011149A1
:1034C00009684018808812490968498A884215DBD2
:1034D0000C2060430A4909684018806800280DD014
:1034E0000C206043064A12688018816808208847CB
:1034F00000202101034A12688918487270BD00003B
:1035000098070020A007002094070020F0FF00008B
:103510009C07002010B5002400BF04E02046FFF700
:1035200043FC601CC4B202484078A042F6DC10BDE7
:103530009407002010B50024044802F0B3F90028D5
:1035400000D000E00124204610BD0000030400006C
:1035500010B5074B14781C7054785C70054B1960DB
:10356000054B186003461833044C236010BD00005F
:1035700094070020980700209C070020A007002047
:1035800010B50446012C09D1FF220C21002000F0C7
:10359000F9F80121022004F0B3FE08E000220C211A
:1035A000104600F0EFF80021022004F0A9FE10BD43
:1035B00010B5002404210848F7F7AEFD552801D1C5
:1035C000012407E0042001F06FF8002801D0002456
:1035D00000E00124204610BD6008002010B504461C
:1035E000012C09D1FF221C21002000F0CBF8012181
:1035F000062004F085FE08E000221C21104600F0A1
:10360000C1F80021062004F07BFE10BD10B5002497
:10361000062001F049F8002801D0012400E0002430
:10362000204610BD10B50446012C09D1FF221721F8
:10363000002000F0A7F80121042004F061FE08E05A
:1036400000221721104600F09DF80021042004F00C
:1036500057FE10BD00200449097A002901D001203D
:1036600000E0002070470000600A002010B504460A
:10367000022C1CD100220D21104600F083F8FDF72A
:1036800063FC002809D0FF220B21002000F07AF80B
:1036900001210D2004F034FE58E000220B211046D9
:1036A00000F070F800210D2004F02AFE4EE0032CFB
:1036B0001CD100220B21104600F064F8FDF744FCF9
:1036C000002809D0FF220D21002000F05BF8012125
:1036D0000D2004F015FE39E000220D21104600F007
:1036E00051F800210D2004F00BFE2FE0042C0ED128
:1036F000FF220D21002000F045F800220B2110468A
:1037000000F040F801210D2004F0FAFD1EE0012C2C
:103710000ED100220D21104600F034F8FF220B21BB
:10372000002000F02FF801210D2004F0E9FD0DE04C
:1037300000220D21104600F025F800220B21104632
:1037400000F020F800210D2004F0DAFD10BD00008B
:1037500010B500240A480078012801D101240CE0AA
:10376000FCF752FD012801D1032406E0FCF74CFDD3
:10377000022801D1022400E00424204610BD0000EC
:10378000F100002010B5064B1B78834207DD242989
:1037900005D224234343034C24681B195A5410BDFB
:1037A0004C2F0020D807002010B5744800684079DD
:1037B00003000DF087F90B0711D325D35A6D77D38A
:1037C0008DA8D30009F0D8F96C4800684079401CF6
:1037D0006A4909684871CFE069494969087809F080
:1037E00043FA664800684079401C6449096848719A
:1037F000624800684079401C604909684871BBE034
:1038000000F028F9002811D17F2009F02DFA5B483B
:1038100000684079401C5949096848715748006858
:103820004079401C5549096848711DE053480068BB
:103830004078401C514909684870504800684078F9
:1038400003280BD300204D4909684870AA204B4932
:1038500009688870032049490968C87009F0B6F9F9
:10386000002046490968487186E000F0F3F8002816
:1038700007D1424800684079401C404909684871B6
:1038800003E000203D490968487109F09FF973E0A1
:1038900009F072F9394800684079401C37490968D5
:1038A000487169E0364949690978491CC8B209F08C
:1038B000DBF9324800684079401C3049096848719A
:1038C0002E4800684079401C2C490968487153E033
:1038D00000F0C0F800280FD109F020F92749096845
:1038E0008870012009F094F9244800684079401C50
:1038F00022490968487105E009F068F900201F496C
:103900000968487138E01D480068807818280CD193
:1039100002201A490968087000201849096848708F
:10392000042016490968C87011E0144800684078FE
:10393000401C124909684870104800684078032804
:1039400005D300F027F900200C490968487009F0F8
:103950003DF900200949096848710DE009F036F980
:103960000020064909684871044909684870AA207E
:1039700002490968887000BF00BF10BDE007002041
:103980004C2F002010B5314800684079002804D041
:1039900001280CD0032848D11DE009F0EDF82B4890
:1039A00000684079401C2949096848714BE0284962
:1039B0000969087809F058F9244800684079401CE2
:1039C000224909684871214800684079401C1F4914
:1039D0000968487137E000F03DF800280CD101205B
:1039E0001A490968087000201849096848700420BD
:1039F00016490968C87011E0144800684078401CF6
:103A0000124909684870114800684078032805D3B6
:103A100000F0C0F800200D490968487009F0D6F898
:103A200000200A49096848710DE009F0CFF800202C
:103A3000064909684871054909684870AA20034980
:103A40000968887000BF00BF10BD0000E0070020BB
:103A50004C2F002010B509F059F804461F480068A3
:103A60000078002838D01D480068C078042833D377
:103A7000002C09D1002119480068C07A820017483B
:103A800000681430815027E014480068C07A810033
:103A900012480068143040581149884211D20F482A
:103AA0000068C07A81000D48006814304058401CFE
:103AB0000A490968C97A8A00084909681431885096
:103AC0000AE000F067F8002104480068C07A82002C
:103AD0000248006814308150204610BDE0070020E5
:103AE000B80B000000B587B001206946087108488E
:103AF0000290084803900848049008480590084838
:103B0000069001A9074800F00FF807B000BD0000BB
:103B10004D3E0100915A0100510C0200A11C02000F
:103B2000A01C0200C4280020F8B506460F46002459
:103B300000253946304600F0EFF900BF14E00025BB
:103B40000EE00021242060430B4A12688018415582
:103B500024206043094A126880184155681CC5B288
:103B6000242DEED3601CC4B205480078A042E6DCE8
:103B700000F010F8F8BD0000D8070020DC07002096
:103B80004C2F00200120024909680871704700008D
:103B9000E007002010B500F073F900200349096820
:103BA000087002490968C87010BD0000E0070020D5
:103BB00007480068C078062808D105480068C07921
:103BC000002803D1012002490968C871704700002C
:103BD000E007002010B555480068C07803000CF0DD
:103BE00071FF08671D1A1714110E056650484068CA
:103BF000002803D04E4841680020884793E000F039
:103C0000E5F890E000F0C6F88DE000F0D1F88AE029
:103C1000FFF7B8FE87E0FFF7C7FD84E0444840683F
:103C2000002803D042484168012088473F48006887
:103C3000407C00281AD03E48C068002803D03C4889
:103C4000C168C82088470020384909684862374859
:103C500000680078002804D0042034490968C8703E
:103C600024E0022031490968C8701FE02F4800682D
:103C7000406A401C2D49096848622C480068406A27
:103C80007D21C900884211D3002028490968486273
:103C9000264800680078002804D0042023490968D9
:103CA000C87003E0022021490968C8703BE000BFEA
:103CB0001F484068002803D01D48416800208847FD
:103CC0001A480068407C002813D01948C0680028B2
:103CD00003D01748C168C8208847002013490968E5
:103CE000486212480068C078401C10490968C870D2
:103CF00018E00E480068406A401C0C490968486298
:103D00000A480068406A7D21C90088420AD3002021
:103D100006490968486205480068C078401C0349A4
:103D20000968C87000BF00BF10BD0000E007002098
:103D30004C2F002010B515480068C078072824D003
:103D4000012012490968487408E011488068002879
:103D500002D00F4988688047FFF73CFF0B48006896
:103D6000C0780628F1D109480068007A0028ECD113
:103D700006480068C0790028E7D104480068807AC6
:103D80000028E2D101490968487410BDE00700200D
:103D90004C2F002010B5054800680078012802D19A
:103DA000FDF7F8FE01E0F5F7A9FC10BDE0070020E3
:103DB00010B5054800680078012802D1FEF716F911
:103DC00001E0F6F779F810BDE007002010B51D48B6
:103DD0000068807A002829D11A480068007A0028F3
:103DE00003D0022017490968887216480068C07914
:103DF000002803D00120134909688872114800681F
:103E00000079012812D100200E49096808710D4976
:103E10000968887207200B490968C8700A48406819
:103E2000002803D0084841680020884705480068FA
:103E30000078012802D1FEF7B3F901E0F6F716F990
:103E400010BD0000E00700204C2F002010B50446F4
:103E50002146084801F042FD07480078002805D1B6
:103E6000002C03D032210548FCF750FD02480470B5
:103E700010BD000001030000F200002050C300004C
:103E80000020244909684870AA20224909688870DE
:103E900000202049096848621E49096808711D49C7
:103EA000096848711B49096888711A490968C8710D
:103EB000184909680872174909688872154909681C
:103EC000C8721449096808732420124909684873A4
:103ED0001049096888730F490968C87300200D49A3
:103EE000096808740B49096848740A4909688874A4
:103EF00008490968C87407490968486100210548EC
:103F00000068816103480068C1610248006801627D
:103F100070470000E007002010B50A780D4B1860CC
:103F2000034628330C4C236024235343044628348F
:103F30001B190A4C23600A4C4B6863608B68A360B2
:103F4000CB68E3604B6963610B6923610B78237075
:103F500010BD0000E0070020D8070020DC0700208B
:103F60004C2F002007480068C078062808D1054873
:103F70000068007A002803D101200249096808720C
:103F800070470000E007002010B50446012C09D15D
:103F9000FF2220210020FFF7F5FB0121084604F055
:103FA000AFF908E0002220211046FFF7EBFB0021CB
:103FB000012004F0A5F910BD10B50024032000F085
:103FC00073FB002801D0012400E00024204610BD2E
:103FD00010B50446032C0ED1FF2215210020FFF757
:103FE000D1FB002214211046FFF7CCFB01210E204B
:103FF00004F086F939E0022C1CD1FCF7A5FF00285B
:1040000009D0FF2214210020FFF7BCFB01210E2064
:1040100004F076F908E0002214211046FFF7B2FB05
:1040200000210E2004F06CF9002215211046FFF744
:10403000A9FB1AE0012C0ED1FF2214210020FFF76A
:10404000A1FB01210E2004F05BF90022152110468E
:10405000FFF798FB09E0002215211046FFF792FBBD
:10406000002214211046FFF78DFB10BD10B500246F
:10407000F8F7C0FC094988420DD3FCF7C1FF0028BE
:1040800007D1FCF751FE012801DD032404E00224DE
:1040900002E0022400E00124204610BDB80B00001D
:1040A00010B50446012C09D1FF221D210020FFF785
:1040B00069FB0121002004F023F908E000221D2102
:1040C0001046FFF75FFB0021084604F019F910BD08
:1040D00010B50024022000F0E7FA002801D00124E6
:1040E00000E00024204610BD10B50446012C09D183
:1040F000FF221E210020FFF745FB0121092004F0CB
:10410000FFF808E000221E211046FFF73BFB0021CC
:10411000092004F0F5F810BD70B500240025002634
:10412000FCF7BAFC0546FCF7C3FC0646022108482A
:10413000F6F7F2FF552800D108E0012E01D1002446
:1041400004E0012D01D1012400E00024204670BDCF
:104150006008002010B50446012C09D1FF221F2160
:104160000020FFF70FFB0121082004F0C9F808E048
:1041700000221F211046FFF705FB0021082004F054
:10418000BFF810BD70B500240025FCF70FFD0546F3
:1041900003211A48F6F7C0FF552806D10120184917
:1041A000088000201749088023E01648008801286D
:1041B00011D114490880FCF713FC762803DA01209A
:1041C0000F49088015E0FCF70BFC782811DB002074
:1041D0000B4908800DE001200A490880FCF700FC2B
:1041E000762803DA01200649088002E0002004490D
:1041F000088003480488204670BD00006008002045
:104200000E0100201001002010B50446012C09D138
:10421000FF2221210020FFF7B5FA0121072004F039
:104220006FF808E0002221211046FFF7ABFA0021C9
:10423000072004F065F810BD10B50024FCF7CCFF92
:10424000012801D1012400E00024204610BD10B552
:104250000446012C09D1FF2216210020FFF792FA13
:104260000121032004F04CF808E00022162110463A
:10427000FFF788FA0021032004F042F810BD10B5C2
:104280000024052000F010FA002801D0012400E0ED
:104290000024204610BD10B50446012C09D1FF2290
:1042A00019210020FFF76EFA0121052004F028F8FB
:1042B0003CE0022C17D1FCF747FE002809D0FF2272
:1042C00019210020FFF75EFA0121052004F018F8FB
:1042D0002CE0002219211046FFF754FA0021052096
:1042E00004F00EF822E0032C17D1FCF733FE00286F
:1042F00009D0FF2219210020FFF744FA01210520EF
:1043000003F0FEFF12E0002219211046FFF73AFAEF
:104310000021052003F0F4FF08E0002219211046D7
:10432000FFF730FA0021052003F0EAFF10BD00007E
:1043300010B50024FCF722FD012839D104214048A2
:10434000F6F7EAFE552803D101203E49087032E015
:10435000FCF7BAFB01280BD0FCF7B6FB022807D00C
:10436000FCF7B2FB032803D0FCF7AEFB052803D112
:104370000120344908701EE0FCF7A6FB042803D195
:1043800002203049087016E0FCF79EFB062803D196
:1043900003202C4908700EE0FCF796FB002803D0A0
:1043A000FCF792FB072806D100202649087002E09E
:1043B00000202449087024480078022813D123489B
:1043C0000078002807D1FCF7BFFD002803D01D4866
:1043D00000781D490870FCF7B7FD1C490870FCF710
:1043E000B3FD044616E018480078032812D1174898
:1043F0000078002807D1FCF7ADFD002803D0114854
:10440000007811490870FCF7A5FD10490870FCF709
:10441000A1FD04460C48007802280ED00A48007816
:1044200003280AD007480078074908700846007832
:10443000002801D0012400E00024204610BD000027
:104440006008002012010020130100201401002048
:1044500010B50446012C0ED1FF221B210020FFF7CE
:1044600091F900221A211046FFF78CF901210A2048
:1044700003F046FF1EE0022C0ED1FF221A2100207D
:10448000FFF780F900221B211046FFF77BF901217D
:104490000A2003F035FF0DE000221A211046FFF735
:1044A00071F900221B211046FFF76CF900210A2048
:1044B00003F026FF10BD000010B50024104800785E
:1044C000012801D1012418E0FCF74AFD022803D09D
:1044D000FCF74AFE02280FD1FCF714FE012809D18F
:1044E000FCF744FD012803D0FCF744FE012801D16C
:1044F000012402E0022400E00224204610BD000056
:10450000F100002010B5F8F78FFA0446204610BDE0
:1045100010B5034B08220349034800F013F910BDFE
:1045200005450100401C02008428002070B50646A5
:104530005C488068002804D05A498868804705464E
:1045400000E000250024A6E0564841680C206043A6
:1045500008184088A84207D0524841680C206043A0
:104560000818408802287DD14E4841680C206043DD
:104570000818806800280CD04A494A680C21614319
:1045800051188868804747490968E20089184870CF
:1045900009E0444841680C206043095C41480068D8
:1045A000E200801841703F480068E1004018407800
:1045B0003C490968E200895C88420FD039480068AC
:1045C000E1004018417837480068E200815400203B
:1045D00034490968E200891848605AE031480068A7
:1045E000E100401841782F4842680C2060431018C1
:1045F000407881421FD12B480068E1004018416893
:10460000284842680C2060431018808881420BD8EB
:1046100024480068E1004018406880192149096871
:10462000E2008918486034E001201E490968E20070
:10463000891848802DE01B480068E1004018416857
:10464000184842680C2060431018C08881420DD879
:1046500014480068E100401840688119114800685A
:10466000E20000E009E08018416012E000200D49FE
:104670000968E200891848800BE0002009490968B0
:10468000E20089184880002106480068E20080188E
:104690004160601C84B203488089A04200DD53E77A
:1046A00070BD0000042F00200146064A92898A420C
:1046B00005DD044A1268CB00D218508800E00020C3
:1046C00070470000042F0020002000BF14E00D49B7
:1046D0004A680C2141435118498801290AD1002117
:1046E000084A1268C300D2185180064A1268C300F3
:1046F000D2185160411C88B2024989898142E6DCA6
:1047000070470000042F0020002000BF13E00C4978
:104710004A680C21414351184988002909D1084AA7
:104720001268C300D2185180054A1268C300D2181B
:104730005160411C88B2024989898142E7DC704797
:10474000042F0020F0B504460020164DAB606960D0
:104750002C60AA8100BF1FE0124D6E680C254543F6
:10476000755D104E3668C700F61975700D4D6E6890
:104770000C254543755D0B4E3668C700F555002581
:10478000084E3668C700F6197580064E3668C700B1
:10479000F6197560451CA8B2024DAD898542DBDC77
:1047A000F0BD0000042F002070B505460E46002E17
:1047B00005D031462846F3F7C9FC044600E02C46F4
:1047C000204670BD10B5FCF707FD012817D10C4835
:1047D0000078012813D00A48007803280FD0094830
:1047E000007800280BD1FCF711FC0749884202D160
:1047F00008F075F803E07D20000108F077F810BD9F
:10480000E5000020E40000208813000008B5002027
:104810000090012269460520F9F790FD05490098AE
:104820008860002004490870044908700449087031
:1048300008BD00004C280020E4000020E600002015
:10484000E700002008B500200090012269460520FD
:10485000F9F774FD0020024908710098886008BDCE
:104860004C28002070B5049C2578914216DD012863
:104870000AD18D4206DAFF26F61AAE420ED3EE18A2
:10488000F5B20BE0154609E0022807D1954204DD98
:104890009D4203DBEE1AF5B200E00D46257070BDB7
:1048A0000D4A4168516081699161C168D160416A76
:1048B0005162016A11620168116041695161816848
:1048C0009160C169D16101691161816A91620021C0
:1048D000024A117070470000202F0020D4070020EA
:1048E00010B5FFF7F1FEF7F7E5FE00210148F6F7F6
:1048F0001DFD10BD6C08002010B5F7F7DBFEFFF7BB
:1049000003FF0AF0C5F80AF061F9FBF71FFBFAF79D
:1049100051F8FFF77BFFF8F7E9FBF6F703FBF9F730
:10492000E5F855210548F6F701FDF8F735F9F9F7EF
:1049300057F8FAF7CBFFF6F7EFFC10BD6C08002034
:104940001CB500203249087008F0C6F80020FCF7BA
:104950008FFC0CF0DFFBF7F773F8F9F7FFF8F6F7C9
:10496000DBFC55212B48F6F7E1FCF8F715F9F9F7D0
:1049700037F8F5F7E5FEF6F763F9E12040020CF0B1
:104980000BF800F071FAF6F7CDFA08F085FAF7F7B0
:1049900091FEF9F755FEF8F739FCF8F7B3FBFFF78E
:1049A000B7FDFEF701F8FFF79DF8FFF7C3F9F9F738
:1049B0004DFDFBF7F7FAF9F7FDFF174A17490120FC
:1049C0000AF0CAF90022114601200AF009F907F09D
:1049D000F1FF0AF043F80AF0F9F8FFF733FF00207F
:1049E0000F4988714871087101208870487014203F
:1049F000087007226846F3F740FC0199009800F020
:104A0000BDFF0221012000F095FEFAF75FFF1CBDFB
:104A1000F10000206C0800200090D003EC0400009E
:104A2000020100207047000010B50446552C03D148
:104A300005494869804702E003490868804700202B
:104A40000249087010BD0000202F0020D40700206C
:104A500010B54648007803000CF034F80A06111B24
:104A600026303B465051738141484068002802D0AF
:104A70003F494868804701203C49087000BF3C48D6
:104A80008068002804D03A49886880473749087010
:104A900069E03748C068002802D03549C8688047B7
:104AA00003203249087000BF31480069002804D053
:104AB0002F49086980472D49087054E02C48406907
:104AC000002802D02A4948698047002027490870F9
:104AD00049E027488069002802D025498869804735
:104AE00006202249087000BF2148C069002804D070
:104AF0001F49C86980471D49087034E000BF1B4842
:104B0000007807280AD11A48006A002802D01849FC
:104B1000086A804709201549087011E01348007899
:104B200008280AD11248406A002802D01049486A71
:104B3000804709200D49087002E000200B490870E9
:104B400000BF0A480078002808D00948806A002879
:104B500004D00749886A80470449087003E00020B0
:104B60000249087000BF00BF10BD0000D40700203C
:104B7000202F00207047000010B500200CF086FBAD
:104B800009F064F809F0B8F809F0CEF800F0C6FCB6
:104B9000F6F7ECF80220FCF76BFB002007490870E1
:104BA000FFF7C8F8FEF7EEFFFFF714F8F5F738FF48
:104BB00010200AF0E7FC00F0B1FD10BDA8010020B4
:104BC00010B5012408F010FC012801D1052407E0EC
:104BD000F7F70AFF0349884201D2012400E00224CA
:104BE000204610BD204E000010B5062408F0FCFB46
:104BF000002800D1002408F0FDFB012803D008F0B4
:104C0000F9FB072800D90924204610BD10B5F6F796
:104C1000ADF80022114601200AF014F900213C48A9
:104C2000F6F784FB00203B490880002400BF00F019
:104C30002FFF32217D200001FBF768FE002036495E
:104C400008700AE00022344801781046FEF79AFD09
:104C500031480078401C304908702F4800782428DB
:104C6000F0DB00202D49087009E000212B48007876
:104C700009F0FCFC29480078401C284908702748A6
:104C800000780D28F1DBFEF7A5FFF5F79FFD08F092
:104C9000FDFA23480078401C214908700846007836
:104CA000052812D300200870FEF782FF1D48007807
:104CB0000A2805D300201B490870FFF753F904E0C8
:104CC00018480078401C1749087008F093FB012829
:104CD000ADD908F08FFB0728A9D200200F49087032
:104CE00008E00E48007809F0DBFC0C480078401C16
:104CF0000A490870094800780D28F2DBF5F7A0FF93
:104D000055210348F6F712FBF7F744FE204610BD85
:104D10006C0800207A0000200B010020090100200F
:104D20000A0100200C01002010B5032408E000F067
:104D3000AFFE012000F0B6FD002801D0042400E001
:104D4000F5E700BF204610BD10B5002029490860D6
:104D500007F0C2FE0120FCF78BFAF6F771FE552131
:104D60002548F6F7E3FAF7F717FFF8F739FE0CF0E6
:104D7000D1F9F5F7E5FCF9F72BFCF5F761FF08F041
:104D800095FAF9F75DFCF9F7F9FDF8F73FFAFFF747
:104D9000BFFBFDF709FEFFF7B7FCFFF737FDFEF796
:104DA000A1FEFEF7C7FF00F05FF8E12040020BF024
:104DB000F3FDF6F7B7F8FBF7F5F8F9F7FBFD0F4A47
:104DC0000F49012009F0C8FF00221146012009F017
:104DD00007FF09F043FE09F0F9FEF8F787FE02210C
:104DE000012000F0A7FCFAF771FD07F005FEF6F7C9
:104DF00093FA10BD4C0000206C0800200090D003F6
:104E0000EC04000070B506460D4614460E480660D8
:104E10000E4805600E49206808600E496068086009
:104E20000D49A06808600D49206908600C49E068D8
:104E300008600C496069086005480068002802D0D5
:104E400003480068804770BDA8000020B000002023
:104E50009000002094000020980000209C0000207A
:104E6000A0000020A400002000B587B00C480190ED
:104E70000C4802900C4803900020049005900B48C9
:104E8000069000200A49086048600A4908604860A6
:104E900001AA0121C9020848FFF7B4FF07B000BD0D
:104EA000BD4E010061520100E951010015510100A0
:104EB000741200206C0A00207C170020012070472B
:104EC000F3B5C3B00446449E0020009057E002E0D2
:104ED000641C761E00BF022E05D32078EB28F7D184
:104EE00060789028F4D1072E00D24AE0A778FD1C04
:104EF000B54200D945E0A81E205C0002691E615C35
:104F000008434290042D38D9291FA01C0CF01CF92D
:104F10004299884226D11D480068002804D0B91E55
:104F2000E01C1A4A1268904719480068002824D0EB
:104F3000E1786846017120798111684641712079D4
:104F40008106890E68468171381FC1B26846C171F9
:104F5000C279611D02A8F3F790F901A80C4909680C
:104F600088470AE00020009002E00098401C009072
:104F70000098A842F9D3002000906419761B072EF0
:104F8000A5D200BF4498801B45B0F0BD9C00002016
:104F9000A4000020F7B5C0B0154600260027E81D84
:104FA000FF210131884202DD002043B0F0BDEB213A
:104FB0006846017090214170281DC1B26846817019
:104FC0000021C1704098C1B26846017105240026D5
:104FD00005E04198805D69460855641C761CAE4228
:104FE000F7DBA11E00A802300CF0AEF8074638121D
:104FF00069460855641C0F55641C06480068002863
:1050000005D021466846034A12689047CDE7002044
:10501000CBE700009400002070B500240025002696
:105020001B4840681A490968884200D170BD184879
:10503000406817490968884205D9154840681449ED
:105040000968451A07E01248006811494968401A82
:10505000012189020D1AFF2D01D9FF2600E02E46FD
:1050600000240DE00A4801680830405C09490855F1
:1050700007480088401C8005800D05490860641CB5
:10508000B442EFD3B1B203480BF0E2FC00BFCDE76E
:10509000741200207C16002070B500251A480068A4
:1050A000002830D0194A1288FF230133991A184A70
:1050B0001268164B1B88D018134A12689047054691
:1050C000002D20D01148008840191049088008465A
:1050D00001880F480068FFF7F3FE0446002C0DDD41
:1050E0000A480088844209DA08480088021B0848F8
:1050F0000068011906480068F3F7BFF80348008804
:10510000001B0249088070BD98000020AC00002000
:10511000A800002038B5044600200090A078102890
:105120000CD120792D49087008460078012853D108
:10513000002211462020FFF72DFF4DE0A078122815
:1051400003D120792549087246E0A078052803D1CB
:105150002079224988723FE0A07802281DD1207969
:105160001E4948720846407A012806D10090012263
:1051700069460420FFF70EFF2EE01848407A022807
:105180002AD100BFBFF34F8F15481649C860BFF33F
:105190004F8F00BF00BF00BFFDE7A07801281BD1E3
:1051A0002079332803D101200C49487005E020798B
:1051B000352802D100200949487060790749887074
:1051C000607A0006217A09040843E179090208435C
:1051D000A17908430149486038BD0000600A0020F9
:1051E0000400FA0500ED00E070B50346002200243B
:1051F00000251A484068194E3668B04201D1002097
:1052000070BD16484068154E3668B04205D913483F
:105210004068124E3668841B07E0104800680F4E45
:105220007668801B0126F602341AA14201D9254670
:1052300000E00D4600220CE0084806680830805D5A
:10524000985406480088401C4005400D034E3060CD
:10525000521CAA42F0D32846D2E700006C0A002074
:1052600070B503460022002415484068144D2D688F
:10527000A84208D312484068114D2D68401B0125F3
:10528000AD022C1A04E00E4800680D4D6D68441BF9
:10529000A14201D9012070BD00220CE09D5C0848AC
:1052A00046680830855508388088401C8005800D88
:1052B000034D6860521C8A42F0D30020EBE70000E7
:1052C0007412002010B50248FFF7EAFA10BD000082
:1052D000281D02000021014A1175704740600040FE
:1052E000014600BFF020084000110A23584302463F
:1052F0000807000F8018C0B270470146002204E082
:10530000501CC2B208460A38C1B20A29F8DA10079E
:10531000000E08437047000010B5044601218020AC
:10532000F6F78EF8607A012805D14248C07810213E
:1053300008434049C870607AA22805D13E48007FE2
:10534000802108433C490877607A3B490877002070
:105350003A4948770846407F2178084337494877DB
:10536000E07B002805D00846407F202108433349D0
:1053700048773248407FC008C000A17A08432F49CF
:1053800048770846807FF72108402C498877E078E5
:10539000FFF7B3FF29498874A078FFF7AEFF2749CC
:1053A000C8746078FFF7A9FF2449087520780028A1
:1053B00005D10846007D2179084320490875E07928
:1053C000FFF79BFF1D4988756079FFF796FF1B4922
:1053D0004875A079FFF791FF1849C875207AFFF743
:1053E0008CFF164908760846807F4006400E887775
:1053F000E07A002806D00846807F402108430F4904
:10540000887703E00D48807F0C498877A07BFFF701
:1054100074FF0A498876607BFFF76FFF0749C876FB
:10542000207B08770846807F1021884303498877CE
:1054300010BD00002004024060040440404F0440BE
:1054400010B504461B48807F01210843194988771D
:105450002078FFF752FF174908756078FFF74DFF76
:105460001449C874A078FFF748FF1249887420785F
:105470000C2806DD0846407F082108430D4948777F
:1054800009E00C48407F0B4948770846007DE178E9
:105490000843084908750748807F400840000549CF
:1054A000887700BF0348807F022108400028F9D197
:1054B00010BD0000404F044010B50020144908768C
:1054C00016200BF025FB0021124801761248407F80
:1054D00080210843104948770846807F012108430E
:1054E0000D49887700BF0C48807F022108400028C2
:1054F000F9D00948807F400840000749887700BFFD
:105500000548807F022108400028F9D110BD000025
:105510004060004040610040404F044010B5002012
:105520000749087000212020F5F78AFF012105486E
:10553000017500200449087515200BF0D1FA10BD43
:1055400000500440406100404060004070B5044697
:105550000D46002C14D0002D12D0042D10D800F0D0
:1055600013F800280CD1002608E00649885D224681
:105570000121F3F701FFA41C701CC6B2AE42F4DB9C
:1055800070BD0000A41C020000200549897DC907E8
:10559000C90F002901D0012000E000207047000061
:1055A0000050044030B585B005460C4600200390FD
:1055B0000490009001900290072C0BDC0120A04089
:1055C00081B2684681810121C17303A90220FAF7E3
:1055D00031FE3EE0082C01D0092C0BD10120A04067
:1055E00081B2684681810121C17303A90120FAF7C4
:1055F00021FE2EE00A2C03D00B2C01D00D2C0BD158
:105600000120A04081B2684681810121C17303A9B4
:105610000020FAF70FFE1CE00C2C01D00F2C0BD150
:105620000120A04081B2684681810121C17303A994
:105630000E20FAF7FFFD0CE00E2C0AD10120A0404D
:1056400081B2684681810121C17303A90C20FAF758
:10565000F1FD002168460170C17041700121817027
:1056600000210171C1720D218172FF21017200219F
:105670004172F3F7E1FE03491520FDF75FF805B02D
:1056800030BD0000D552010010B50020104908754A
:1056900015200BF025FA00210E4801751520002871
:1056A00009DB00BF00BFC206D20E012191400A4AA9
:1056B000116000BF00BF00BF084880798011032837
:1056C00005D006480078802108430449087010BDC1
:1056D000406000404061004000E100E000500440B4
:1056E00010B5F3F7A3FF10BD10B501231A46002132
:1056F0001846F5F759FE012211461046F5F7C0FE8F
:10570000F2F7E0FC03480BF0F7FC0248024908609E
:1057100010BD00000090D0035807002000BF0448CF
:105720000069042108430249086130BF00BF704787
:1057300000ED00E0F3B585B0054600240027002603
:10574000002003900490EEB22804070E0F2F54DAC5
:10575000082E52DA002009E00C214143284A515A10
:10576000A94201D1044603E0411CC8B21728F3D373
:1057700000BF0120B04086B20C2060432049401891
:10578000C3780C20604340188278F8B2314601900B
:10579000FAF7F4FD68468681012181730021C17307
:1057A00002214174F8B203A9FAF744FD0C216143C8
:1057B000134A8918C888FBF781FE0C206043104902
:1057C0004018C1886846018169460698887202A817
:1057D000FBF78EFD0C226243094BD21891680C2214
:1057E0006243D21804201056FCF7A8FF0C21614335
:1057F000034A8918C888FBF7E5FD07B0F0BD000033
:10580000C01E0200FEB505460C460020C0430290B3
:10581000EFB22804060E0F2E42DA082F40DA0120DC
:10582000B8406946088080202040002816D1012019
:105830008870A007800F022801D1487109E0A007F5
:10584000800F012802D16946487102E000206946B4
:105850004871F0B26946FAF7EDFC1FE00020694696
:1058600088700E202040002800D000BF102020406B
:10587000002802D16946087102E0012069460871DA
:10588000E007C00F002802D16946887102E00120BC
:1058900069468871F0B26946FAF7CCFC00200290A4
:1058A0000298FEBD30B50146CAB20C04230E00209A
:1058B0000F2B0FDA082A0DDA01249440A2B2064C0D
:1058C00003252D026419E45C1440002C01D0012052
:1058D00000E0002030BD000000000440F8B50446A0
:1058E0000F460020C0430090E6B22004050E0F2DA5
:1058F00011DA082E0FDA0120B04086B2002F04D151
:10590000E8B23146FAF792FD03E0E8B23146FAF721
:105910009DFD002000900098F8BD00001649897F89
:1059200001221143144A917700BF1349897F022253
:1059300011400029F9D01049897C81700E49C97C39
:1059400041700D49097D01700B498A7D8271497D45
:1059500001710949CA7D42710A7EC271897F490875
:105960004900054A917700BF0349897F022211400F
:105970000029F9D170470000404F044003B585B0BD
:10598000002001900290039004900021684641732A
:10599000817E01A8C1706846417E01A88170684679
:1059A000017E4171002101A8017108216846017141
:1059B000817D01A8C1716846C17D4172417D01A808
:1059C00081716846017D01A80172002168468173DA
:1059D000C17301A881730C21417341216846017490
:1059E0000021C17401A8FFF797FC1D20044988829B
:1059F00004491620FCF7A2FE00F006F807B000BD2F
:105A0000204F04404512020010B5FFF755FD10BDB0
:105A100070B504460D46601E0D49884200D9012428
:105A2000002C00D1012440200A4908700846007863
:105A30006043094948610321081F0BF081F80020E9
:105A400005498861072008610448056070BD0000B1
:105A5000FFFFFF008401002000E000E08001002043
:105A60000020C043002809DBC206D20E012191406C
:105A7000054A1160BFF34F8FBFF36F8F00BF002047
:105A8000024908618861704780E100E000E000E0C1
:105A900010B50AF0FBFF10BD1A20084908722B2030
:105AA00048723C2088724D20C8727F2004490968E2
:105AB0000860AC20034948707047000000040240B1
:105AC000880100200010024010B51C480078012811
:105AD00012D11B480078642809DB0220194948715B
:105AE00008710020164908701449087004E0144831
:105AF0000078401C124908701348007801281CD116
:105B000012480078012804D100201049087010497B
:105B100008700F48007832280ADBF7F785F8002173
:105B20000C48F5F7B3FB55210B48F5F7FFFB04E0F4
:105B300007480078401C0649087010BD2107002066
:105B400020070020100700201A0700201C07002053
:105B50001B070020600800206C080020F8B50446F0
:105B60000D46002700200090032000032040001372
:105B70000090102C04D0122C02D01148844217D16E
:105B800022202840222806D127073F0F39460098B7
:105B9000F4F7C2FD06461220284012280ED1200735
:105BA000000F471C39460098F4F7B6FD064605E09D
:105BB0002107090F0098F4F7AFFD06463046F8BDFF
:105BC00010100000F8B504460D46002600270120FD
:105BD000000320400713102C04D0122C02D00F48D1
:105BE000844215D122202840222805D12607360FCD
:105BF00031463846FAF70EF81220284012280CD108
:105C00002007000F461C31463846FAF703F804E037
:105C10002107090F3846F9F7FDFFF8BD1010000005
:105C2000FFB58BB01C4600200790069005903848C1
:105C3000049010210B980840002801D0022707E0AB
:105C400040210B980840002801D0012700E00027E0
:105C5000002C04D0149804700120089001E010205A
:105C60000890002548E0002C08D025466000294A0D
:105C7000115A0C98F2F76AFA079006E06800254A74
:105C8000115A0C98F2F762FA07903E4630E0711C08
:105C90000798F2F75BFA400806900D98F2F7ACFB14
:105CA00003900D9A0699881AF2F7A6FB18490190FD
:105CB000F2F727FB02900399F2F760FB0590059835
:105CC000F2F7A1FB49004908039102900498F2F70A
:105CD0009AFB4900490801910090039B029AF2F750
:105CE000A7FB03D20A95099605980490701CC6B2CA
:105CF0007F2ECCDD681CC5B208988542B3DB1499B1
:105D00000A98087014990998487004980FB0F0BD6B
:105D10000000C842D41F02000246412A2ED010DCE7
:105D2000212A2AD006DC102A45D0122A4BD0202A5C
:105D300059D11CE0222A26D0232A2AD0402A52D127
:105D400016E081235B01D01A9A4228D008DC422A4F
:105D50001AD0432A1ED025481018002843D13AE013
:105D6000012822D020281BD021283CD11EE000BFD2
:105D70001F4803890B43038136E000BF1C48438959
:105D80000B43438130E000BF194883890B43838173
:105D90002AE000BF1648C3890B43C38124E000BF3B
:105DA000144883880B4383801EE000BF1148C388DA
:105DB0000B43C38018E00E4843890B43438103899A
:105DC0000B43038110E00A48C3890B43C3818389D5
:105DD0000B43838108E00748C3880B43C380838853
:105DE0000B43838000E000BF00BF7047F0EFFFFF70
:105DF0000011044000140440F0B505460E46412D44
:105E000030D010DC212D2CD006DC102D51D0122DDD
:105E100056D0202D62D11CE0222D2AD0232D30D047
:105E2000402D5BD116E081214901681A8D4230D0A6
:105E300008DC422D1ED0432D24D02A4828180028E3
:105E40004CD144E001282CD0202823D0212845D152
:105E500028E000BF244F3888314600F049F8044656
:105E60003DE000BF204F7888314600F041F80446FD
:105E700035E000BF1C4FB888314600F039F80446C1
:105E80002DE000BF184FF888314600F031F8044685
:105E900025E000BF154F3888314600F029F8044648
:105EA0001DE000BF114F7888314600F021F804460C
:105EB00015E00D4F7888314600F01AF804460EE0E0
:105EC000094FF888314600F013F8044607E0074F01
:105ED0007888314600F00CF8044600E000BF00BFAF
:105EE0002046F0BDF0EFFFFF001104400014044015
:105EF0000246002013460B40002B01D0012000E099
:105F000000207047FFB581B00E461746012F07D11C
:105F1000F748407D00090001C01DF549487505E0BE
:105F2000F348407D00090001F149487504980128B3
:105F30007ED10A210198F2F709F90546ED48445D42
:105F4000E007C00F002807D0E948007C00090001E5
:105F5000C01DE749087405E0E548007C0009000120
:105F6000E349087402202040002807D0E048C07BA5
:105F7000F02188437030DE49C87305E0DC48C07BFF
:105F8000F0218843DA49C87304202040002807D054
:105F9000D748807C00090001C01DD549887405E000
:105FA000D348807C00090001D14988740820204032
:105FB000002807D0CE48407CF02188437030CC497F
:105FC000487405E0CA48407CF0218843C8494874B9
:105FD00010202040002807D0C548407C000900015F
:105FE000C01DC349487405E0C148407C0009000158
:105FF000BF49487420202040002807D0BC48007CBE
:10600000F02188437030BA49087405E0B848007C34
:10601000F0218843B649087440202040002808D069
:10602000B348807CF02188437030B149887406E021
:106030008BE0AF48807CF0218843AD4988740A2109
:106040000198F2F783F80D46AA48445DE007C00FB7
:10605000002807D0A648807BF02188437030A449EF
:10606000887305E0A248807BF0218843A0498873AB
:1060700002202040002807D09D48807B00090001B5
:10608000C01D9B49887305E09948807B0009000189
:106090009749887304202040002807D09448007D49
:1060A000F021884370309249087505E09048007DE2
:1060B000F02188438E49087508202040002807D029
:1060C0008B48007D00090001C01D8949087505E065
:1060D0008748007D0009000185490875102020408F
:1060E000002807D08248C07CF02188437030804966
:1060F000C87405E07E48C07CF02188437C49C874A0
:1061000020202040002807D07948C07B00090001EA
:10611000C01D7749C87305E07548C07B00090001C0
:106120007349C87340202040002807D07048C07CC5
:1061300000090001C01D6E49C87454E06C48C07C61
:10614000000900016A49C8744DE06948007C0009F3
:106150000001674908740846C07BF0218843644900
:10616000C8730846807C0009000188740846407C9A
:10617000F02188435E4948740846407C00090001CC
:1061800048740846007CF021884359490874084641
:10619000807CF0218843564988740846807BF02132
:1061A0008843534988730846807B0009000188733F
:1061B0000846007DF02188434D4908750846007D5A
:1061C0000009000108750846C07CF0218843484951
:1061D000C8740846C07B00090001C8730846C07C2B
:1061E00000090001C8740A9801287DD10A213046AF
:1061F000F1F7ACFF05463F48445DE007C00F0028BB
:1062000007D03B48407B00090001C01D3849487356
:1062100005E03748407B00090001354948730220FA
:106220002040002807D03248007BF021884370309E
:106230002F49087305E02E48007BF02188432C4944
:10624000087304202040002807D02948807DF021D1
:10625000884370302649887505E02548807DF02107
:1062600088432349887508202040002807D020480B
:10627000807D00090001C01D1D49887505E01C488E
:10628000807D000900011A498875102020400028EF
:1062900007D01748407DF021884370301449487575
:1062A00005E01348407DF0218843114948752020BE
:1062B0002040002807D00E48407BF02188437030F2
:1062C0000B49487305E00A48407BF02188430849A0
:1062D00048734020204000280ED00548C07D0009AA
:1062E0000001C01D024900E092E0C8750AE000000C
:1062F0005C260020F81902006D48C07D00090001ED
:106300006B49C8750A213046F1F720FF0D466948F0
:10631000445DE007C00F002807D06548C07AF0212F
:10632000884370306249C87205E06148C07AF02144
:1063300088435F49C87202202040002807D05C488B
:10634000C07A00090001C01D5949C87205E05848CB
:10635000C07A000900015649C87204202040002874
:1063600007D05348407E00090001C01D50494876BF
:1063700005E04F48407E000900014D49487608205D
:106380002040002807D04A48007EF0218843703022
:106390004749087605E04648007EF0218843444995
:1063A000087610202040002807D04148007E0009D0
:1063B0000001C01D3E49087605E03D48007E000909
:1063C00000013B49087620202040002807D03848AB
:1063D000007B00090001C01D3549087305E0344801
:1063E000007B00090001324908734020204000284A
:1063F00007D02F48C07DF021884370302C49C875E4
:1064000054E02B48C07DF02188432949C8754DE0F0
:106410002748407B00090001254948730846007B56
:10642000F0218843224908730846807DF021884383
:106430001F4988750846807D000900018875084657
:10644000407DF02188431A4948750846407BF02179
:106450008843174948730846C07D00090001C87584
:106460000846C07AF02188431149C8720846C07AAC
:1064700000090001C8720846407E00090001487604
:106480000846007EF0218843094908760846007EC8
:106490000009000108760846007B00090001087326
:1064A0000846C07DF02188430149C87505B0F0BD9C
:1064B0005C260020F8190200FFB581B00E46174691
:1064C000019801287ED10498002826D1FA48007846
:1064D000012822D0F6F78EFAF84988421DD3FAF740
:1064E00033FD00280DD0F648807DF02188437030C0
:1064F000F34988750846C07C00090001C01DC874B6
:1065000018E0EF48807DF0218843ED498875084602
:10651000C07C00090001C8740CE0E948807DF021CE
:1065200088437030E64988750846C07C0009000140
:10653000C01DC874E248C07CF02188437030E04937
:10654000C8740846007EF02188437030DC49087624
:106550000846807D00090001401C88750846407D82
:10656000F02188431030D64948750846407D00091F
:106570000001401C48750846007DF021884310301A
:10658000CF4908750846007D00090001401C0875C8
:1065900033000AF097FA062E261E140C042FC84862
:1065A000007D00090001C01DC549087500BFC44831
:1065B000007DF02188437030C149087500BFC04894
:1065C000407D00E0ADE100090001C01DBC494875F7
:1065D00000BFBB48407DF02188437030B849487502
:1065E00000BFB748807D00090001C01DB44988750F
:1065F00000BF00E000BF00BF049800285ED1AE4895
:10660000007801285AD0F6F7F5F9AC49884255D3FD
:10661000AB48C07FF0218843A949C8770846807FEE
:106620000009000188770846407FF0218843A4498B
:1066300048770846007FF0218843A149087708463B
:10664000C07DF02188439E49C8750846C07F000977
:106650000001C8770846807FF021884398498877F1
:106660000846407F00090001C01D48770846807E2B
:10667000F0218843924988760846807E000900010F
:1066800088760846407E0009000148760846007E6C
:106690000009000108760846007F0009000108771C
:1066A0000846C07EF02188438549C8760846407E6A
:1066B000F0218843703082494876B8E16421384639
:1066C000F1F744FD0546012D07D17D48C07FF0213B
:1066D000884370307A49C87705E07948C07FF02157
:1066E00088437749C8770A213846F1F72FFD0A21F8
:1066F0000090F1F72BFD0D46642F02D37148445DE5
:1067000001E07148445DE007C00F002807D06C48E5
:10671000807F00090001C01D6949887705E068484D
:10672000807F000900016649887702202040002808
:1067300007D06348407FF021884370306049487734
:1067400005E05F48407FF02188435D494877042099
:106750002040002807D05A48007FF021884370303D
:106760005749087705E05648007FF021884354498F
:10677000087708202040002807D05148C07DF0212C
:10678000884370304E49C87505E04D48C07DF02102
:1067900088434B49C87510202040002807D048483E
:1067A000C07F00090001C01D4549C87705E0444885
:1067B000C07F000900014249C877202020400028FE
:1067C00007D03F48807FF021884370303C4988776C
:1067D00005E03B48807FF021884339498877402095
:1067E0002040002807D03648407F00090001C01D26
:1067F0003349487705E03248407F000900013049BD
:1068000048770A213846F1F7A1FC0D462D48445D32
:10681000E007C00F002807D02948807EF021884378
:1068200070302749887605E02548807EF02188432E
:106830002349887602202040002807D02048807E07
:1068400000090001C01D1E49887605E01C48807EB5
:10685000000900011A49887604202040002807D04A
:106860001748407E00090001C01D1549487605E023
:106870001348407E00090001114948760820204055
:10688000002807D00E48007E00090001C01D0C49F9
:10689000087605E00A48007E0009000108490876EC
:1068A00010202040002811D00548007F0009000179
:1068B000C01D034908770FE0F1000020B80B00006D
:1068C00030270020F81902000B1A02005948007FF7
:1068D000000900015749087720202040002807D0F0
:1068E0005448C07EF021884370305249C87605E094
:1068F0005048C07EF02188434E49C8764020204051
:10690000002807D04B48407EF02188437030494929
:1069100048768CE04748407EF021884345494876D8
:1069200085E04448807D0009000142498875084699
:10693000407DF02188433F4948750846407D000965
:10694000000148750846007DF021884339490875E3
:106950000846007D0009000108750846C07C000952
:106960000001C8740846807DF0218843314988754C
:106970000846C07CF02188432E49C8740846007E32
:10698000F02188432B4908760846C07FF0218843D0
:106990002849C8770846807F0009000188770846A3
:1069A000407FF0218843234948770846007FF02143
:1069B0008843204908770846C07DF02188431D4957
:1069C000C8750846C07F00090001C8770846807F67
:1069D000F0218843174988770846407F0009000165
:1069E00048770846807EF021884312498876084619
:1069F000807E0009000188760846407E000900017B
:106A000048760846007E0009000108760846007FA7
:106A10000009000108770846C07EF0218843054937
:106A2000C8760846407EF02188430249487605B082
:106A3000F0BD00003027002010B5014600220020E4
:106A40000A0EFE4B985CC307DB0F002B07D0FC4BF4
:106A5000DB7FF024A3437033F94CE37705E0F84B78
:106A6000DB7FF024A343F64CE37702230340002BA3
:106A700007D0F34BDB7F1B091B01DB1DF04CE377D9
:106A800005E0EF4BDB7F1B091B01ED4CE377042393
:106A90000340002B07D0EA4B9B7F1B091B01DB1D2A
:106AA000E74CA37705E0E64B9B7F1B091B01E44CF9
:106AB000A37708230340002B09D0E14B20335B78F8
:106AC0001B091B01DB1DDE4C2034637007E0DC4B2F
:106AD00020335B781B091B01D94C203463701023D1
:106AE0000340002B09D0D64B20331B78F024A3435E
:106AF0007033D34C2034237007E0D14B20331B7804
:106B0000F024A343CE4C2034237020230340002BD9
:106B100009D0CB4B20331B781B091B01DB1DC84C54
:106B20002034237007E0C64B20331B781B091B0160
:106B3000C34C2034237040230340002B07D0C04BAC
:106B40009B7FF024A3437033BD4CA37705E0BC4B7F
:106B50009B7FF024A343BA4CA377FF231B040B4075
:106B60001A0CB64B985CC307DB0F002B07D0B44B55
:106B70001B7F1B091B01DB1DB14C237705E0B04BCC
:106B80001B7F1B091B01AE4C237702230340002B04
:106B900007D0AB4BDB7EF024A3437033A84CE376E5
:106BA00005E0A74BDB7EF024A343A54CE37604234A
:106BB0000340002B07D0A24B9B7EF024A3437033ED
:106BC0009F4CA37605E09E4B9B7EF024A3439C4CF8
:106BD000A37608230340002B07D0994B5B7FF0245A
:106BE000A3437033964C637705E0954B5B7FF024AD
:106BF000A343934C637710230340002B07D0904BA3
:106C00005B7F1B091B01DB1D8D4C637705E08C4B03
:106C10005B7F1B091B018A4C637720230340002BF9
:106C200007D0874B1B7FF024A3437033844C23771A
:106C300005E0834B1B7FF024A343814C2377402343
:106C40000340002B07D07E4BDB7E1B091B01DB1DA5
:106C50007B4CE37605E07A4BDB7E1B091B01784C0D
:106C6000E376FF231B020B401A0A744B985CC307A0
:106C7000DB0F002B07D0724B1B7EF024A343703335
:106C80006F4C237605E06E4B1B7EF024A3436C4CC7
:106C9000237602230340002B07D0694B1B7E1B0980
:106CA0001B01DB1D664C237605E0654B1B7E1B0933
:106CB0001B01634C237604230340002B07D0604B59
:106CC000DB7D1B091B01DB1D5D4CE37505E05C4BA7
:106CD000DB7D1B091B015A4CE37508230340002B85
:106CE00007D0574B9B7E1B091B01DB1D544CA37621
:106CF00005E0534B9B7E1B091B01514CA3761023CF
:106D00000340002B07D04E4B5B7EF024A34370332F
:106D10004B4C637605E04A4B5B7EF024A343484C22
:106D2000637620230340002B07D0454B5B7E1B0975
:106D30001B01DB1D424C637605E0414B5B7E1B096A
:106D40001B013F4C637640230340002B07D03C4B94
:106D5000DB7DF024A3437033394CE37505E0384BF9
:106D6000DB7DF024A343364CE375CAB2334B985C09
:106D7000C307DB0F002B07D0314B1B7DF024A3434F
:106D800070332F4C237505E02D4B1B7DF024A3435E
:106D90002B4C237502230340002B07D0284B1B7D6F
:106DA0001B091B01DB1D264C237505E0244B1B7DB5
:106DB0001B091B01224C237504230340002B07D021
:106DC0001F4BDB7C1B091B01DB1D1D4CE37405E025
:106DD0001B4BDB7C1B091B01194CE374082303408C
:106DE000002B07D0164B9B7CF024A3437033144C2C
:106DF000A37405E0124B9B7CF024A343104CA374B6
:106E000010230340002B07D00D4B5B7DF024A343E0
:106E100070330B4C637505E0094B5B7DF024A34395
:106E2000074C637520230340002B0BD0044B5B7D84
:106E30001B091B01DB1D024C637509E0F8190200F8
:106E4000102700200C4B5B7D1B091B010A4C63754E
:106E500040230340002B07D0074BDB7CF024A343E7
:106E60007033054CE37405E0034BDB7CF024A34353
:106E7000014CE37410BD00001027002000B501286C
:106E80007ED1FE4AD278F0239A437032FB4BDA70FF
:106E90001A46127912091201D21D1A711A46127974
:106EA000F0239A437032F54B1A711A46527912093F
:106EB0001201D21D5A711A465279F0239A43703248
:106EC000EE4B5A711A46D27912091201D21DDA71AB
:106ED0001A46D279F0239A437032E84BDA711A4697
:106EE000527A12091201D21D5A721A46527AF023AE
:106EF0009A437032E14B5A721A46927AF0239A43BF
:106F00007032DE4B9A721A469278F0239A437032AE
:106F1000DA4B9A701A46D27A12091201D21DDA722D
:106F20001A46527812091201D21D5A701A46D27AA4
:106F3000F0239A437032D14BDA721A46203AD27F4C
:106F4000F0239A437032CD4B203BDA77CB4A127B49
:106F500012091201D21D20331A731A46203A927F69
:106F600012091201D21D203B9A77C44A127BF023EA
:106F70009A437032C14B1A731A46203A127F00E0CE
:106F8000F2E1F0239A437032BC4B203B1A77BB4AA4
:106F9000527B12091201D21D20335A731A46203A2D
:106FA000D27E12091201D21D203BDA76B44AD27881
:106FB000F0239A437032B24BDA701A46127B1209F0
:106FC0001201D21D1A731A46127912091201D21D2A
:106FD0001A711A46927AF0239A437032A84B9A7229
:106FE0001A461279F0239A437032A54B1A711A4649
:106FF000527912091201D21D5A711A469279120958
:107000001201D21D9A711A46127A12091201D21D6A
:107010001A721A46127AF0239A437032984B1A72F7
:107020001A46527A12091201D21D5A72934A927963
:1070300012091201521C914B9A711A469279F0234F
:107040009A4310328D4B9A711A46127A1209120124
:10705000521C1A721A46127AF0239A431032874B46
:107060001A721A46927A12091201521C9A721A4620
:10707000D27812091201521CDA701A46927812095B
:107080001201521C9A701A465278F0239A43103219
:107090007A4B5A701A461278F0239A431032774B83
:1070A0001A701A46127812091201521C1A701A46E6
:1070B000203AD27F12091201521C203BDA771A467D
:1070C000927FF0239A4310326C4B203B9A771A46FA
:1070D000527FF0239A431032684B203B5A771A466E
:1070E000527F12091201521C5A771A46127F120956
:1070F0001201521C1A771A46D27EF0239A4310329C
:107100005E4B203BDA761A46927EF0239A43103289
:107110005A4B203B9A765A4A127BF0239A431032FC
:10712000574B1A731A46D27AF0239A431032544BB3
:10713000DA721A46D27A12091201521CDA721A460F
:10714000927A12091201521C9A721A46527AF0234C
:107150009A4310324A4B5A721A465279F0239A4394
:107160001032474B5A711A46D279F0239A431032A3
:10717000434BDA710B0009F0A5FC19F3E9DFD5CB1D
:10718000C1B7ADA3998F87786E645A50463E362EAC
:10719000261E160EF5003A4AD279F0239A43703231
:1071A000374BDA7100BF364A5279F0239A43703276
:1071B000334B5A7100BF324A527AF0239A437032ED
:1071C0002F4B5A7200BF2E4A927A12091201D21D19
:1071D0002B4B9A7200BF2A4AD27A12091201D21D91
:1071E000274BDA7200BF264AD27AF0239A437032D4
:1071F000234BDA7200BF224A127BF0239A4370328B
:107200001F4B1A7300BF1D4A203A927EF0239A4307
:1072100070321A4B203B9A7600BF184A203AD27E31
:10722000F0239A437032154B203BDA7600BF134AA5
:10723000203A127F12091201D21D104B203B1A77FF
:1072400000BF0E4A203A527F12091201D21D0B4B89
:10725000203B5A7700BF094A203A527FF0239A43D5
:107260007032064B203B5A7700BF044A203A927F87
:10727000F0239A437032014B203B03E07C26002030
:10728000502700209A7700BFDC4AD27F12091201F2
:10729000D21DDA4BDA7700BFD84A203212781209B1
:1072A0001201D21DD54B20331A7000BFD34A2032B1
:1072B0001278F0239A437032D04B20331A7000BFFB
:1072C000CE4A20325278F0239A437032CB4B20338F
:1072D0005A7000BFC94A2032927812091201D21D99
:1072E000C64B20339A7000BFC44A2032D2781209AC
:1072F0001201D21DC14B2033DA7000BFBF4A2032C9
:10730000927A12091201D21DBC4B20339A7200BF2F
:10731000BA4A2032127AF0239A437032B74B2033A4
:107320001A7200BFB54A2032127A12091201D21D18
:10733000B24B20331A7200BFB04A20329279F02348
:107340009A437032AD4B20339A7100BFAB4A203262
:10735000927912091201D21DA84B20339A7100BFF5
:1073600001E0FFE700BF47E1A44A2032D278F023D2
:107370009A43A24B2033DA701A461279120912018D
:107380001A711A461279F0239A439C4B20331A71D2
:107390001A465279120912015A711A465279F0238B
:1073A0009A43964B20335A711A46D2791209120128
:1073B000DA711A46D279F0239A43904B2033DA716E
:1073C0001A46527A120912015A721A46527AF02358
:1073D0009A438A4B20335A721A46927AF0239A4380
:1073E000864B20339A721A469278F0239A43834B45
:1073F00020339A701A46D27A12091201DA721A46AA
:107400005278120912015A701A46D27AF0239A431E
:107410007A4B2033DA72794AD27FF0239A43774B42
:10742000DA771A462032127B1209120120331A73BE
:10743000724A927F12091201203B9A771A46203233
:10744000127BF0239A436D4B20331A736B4A127FE1
:10745000F0239A43694B1A771A462032527B12095D
:10746000120120335A73654AD27E12091201203B61
:10747000DA76634AD278F0239A43614BDA701A467F
:10748000127B120912011A731A461279120912019B
:107490001A711A46927AF0239A43594B9A721A46F5
:1074A0001279F0239A43564B1A711A4652791209EF
:1074B00012015A711A469279120912019A711A46EA
:1074C000127A120912011A721A46127AF0239A439A
:1074D0004B4B1A721A46527A120912015A72474AD3
:1074E0002032927912091201444B20339A711A46C4
:1074F0009279F0239A43414B20339A711A46127ABB
:10750000120912011A721A46127AF0239A433B4B5F
:1075100020331A721A46927A120912019A721A4686
:10752000D27812091201DA701A4692781209120101
:107530009A701A465278F0239A43304B20335A708F
:107540001A461278F0239A432C4B20331A701A46AD
:107550001278120912011A70284AD27F12091201F8
:10756000203BDA771A46927FF0239A43234B9A778F
:107570001A46527FF0239A43204B5A771A46527F7D
:10758000120912015A771A46127F120912011A774C
:107590001A46D27EF0239A43184BDA761A46927E28
:1075A000F0239A43154B9A76154A127BF0239A439F
:1075B000134B1A731A46D27AF0239A43104BDA729D
:1075C0001A46D27A12091201DA721A46927A12090E
:1075D00012019A721A46527AF0239A43084B5A7251
:1075E0001A465279F0239A43054B5A711A46D279BA
:1075F000F0239A43024BDA7100BD00005C260020A4
:1076000050270020F7B582B0064617460025002017
:107610000190002E7ED1F9F799FB05285FD1F9F78B
:1076200093FC00280DD0FA484079F021884370304F
:10763000F74948710846807800090001C01D88702C
:107640000AE0F3484079F0218843F149487108463F
:107650008078000900018870ED48C07900090001B8
:10766000EB49C87108468079000900018871084615
:1076700040790009000148710846007AF0218843EA
:10768000E34908720846007A0009000108720846BA
:10769000C079F0218843DE49C8710846C0780009E6
:1076A0000001C87008468078F0218843D849887066
:1076B00008464078F0218843D5494870084640780C
:1076C00000090001487008460079000900010871AE
:1076D0000846C078F0218843CD49C87029E2CC48DB
:1076E0004079F02188437030C94948710846807854
:1076F00000090001C01D88700846C079000900011A
:10770000C8710846807900090001887108464079EF
:10771000000900E034E0000148710846007AF021D9
:107720008843BB4908720846007A000900010872C4
:107730000846C079F0218843B549C8710846C07829
:1077400000090001C87008468078F0218843B049DC
:10775000887008464078F0218843AD494870084653
:1077600040780009000148700846007900090001CE
:1077700008710846C078F0218843A549C870ADE774
:10778000012E5FD1F9F7E0FB00280DD0A048407929
:10779000F021884370309E4948710846807800097E
:1077A0000001C01D88700AE099484079F0218843A3
:1077B000974948710846807800090001887094480C
:1077C000C079000900019249C87108468079000912
:1077D0000001887108464079000900014871084697
:1077E000007AF02188438A4908720846007A000925
:1077F000000108720846C079F02188438449C871A5
:107800000846C07800090001C87008468078F02159
:1078100088437F49887008464078F02188437C4936
:107820004870084640780009000148700846007911
:107830000009000108710846C078F02188437449A6
:10784000C870EAE3022E7DD1F9F780FA05287AD1D3
:10785000F9F77AFB002877D0012F76D10A21039817
:10786000F0F774FC0546F9F78FFA002802D1694851
:10787000445D01E06848445DE007C00F002807D080
:107880006348C07900090001C01D6149C87105E065
:107890005F48C079000900015D49C871022020409D
:1078A000002807D05A48807900090001C01D5849B6
:1078B000887105E0564880790009000154498871B3
:1078C00004202040002807D05148407900090001D9
:1078D000C01D4F49487105E04D484079000900013D
:1078E0004B49487108202040002807D04848007ABA
:1078F000F021884370304649087205E04448007A18
:10790000F02188434249087210202040002807D007
:107910003F48007A00090001C01D3D49087205E09A
:107920003B48007A000900013949087220202040B4
:1079300000280BD03648C079F02188437030344994
:10794000C87109E0AEE242E1F4E0A4E03048C07959
:10795000F02188432E49C87140202040002807D0DC
:107960002B484079F021884370302949487105E05F
:1079700027484079F0218843254948710A21039816
:10798000F0F7E4FB0D462348445DE007C00F0028F4
:1079900007D01F48C07800090001C01D1C49C870ED
:1079A00005E01B48C078000900011949C870022091
:1079B0002040002807D016488078F0218843703096
:1079C0001349887005E012488078F02188431049F7
:1079D000887004202040002807D00D484078F0210E
:1079E000884370300A49487005E009484078F02122
:1079F0008843074948700820204000280ED00448DA
:107A0000407800090001C01D014948700CE00000E9
:107A10009C260020F81902000B1A0200FE4840784C
:107A200000090001FC49487010202040002807D0C0
:107A3000F948007900090001C01DF749087105E007
:107A4000F548007900090001F34908712020204021
:107A5000002807D0F048C078F02188437030EE4904
:107A6000C87005E0EC48C078F0218843EA49C87046
:107A700040202040002807D0E74880780009000116
:107A8000C01DE5498870C8E2E3488078000900011C
:107A9000E1498870C1E2E0484079F02188437030C4
:107AA000DD4948710846807800090001C01D8870D2
:107AB0000846C07900090001C871084680790009AC
:107AC00000018871084640790009000148710846A4
:107AD000007AF0218843D04908720846007A0009EC
:107AE000000108720846C079F0218843CA49C8716C
:107AF0000846C07800090001C87008468078F02167
:107B00008843C549887008464078F0218843C249B7
:107B1000487008464078000900014870084600791E
:107B20000009000108710846C078F0218843BA496D
:107B3000C87072E2B8484079F0218843B64948716C
:107B4000084680780009000188700846C07900095D
:107B50000001C87108468079000900018871084653
:107B600040790009000148710846007AF0218843F5
:107B7000A94908720846007A0009000108720846FF
:107B8000C079F0218843A449C8710846C07800092B
:107B90000001C87008468078F02188439E498870AB
:107BA00008464078F02188439B4948700846407851
:107BB00000090001487008460079000900010871B9
:107BC0000846C078F02188439349C87025E2012F08
:107BD00073D10A210398F0F7B9FA0546F9F7D4F8FA
:107BE000002802D18D48445D01E08D48445DE007E6
:107BF000C00F002807D08848C07900090001C01DC7
:107C00008549C87105E08448C079000900018249AE
:107C1000C87102202040002807D07F4880790009E1
:107C20000001C01D7C49887105E07B48807900090E
:107C300000017949887104202040002807D0764847
:107C4000407900090001C01D7349487105E0724880
:107C5000407900090001704948710820204000283F
:107C600007D06D48007AF021884370306A49087265
:107C700005E06948007AF0218843674908721020BE
:107C80002040002807D06448007A00090001C01D88
:107C90006149087205E06048007A000900015E4908
:107CA000087220202040002808D05B48C079F021CD
:107CB000884370305849C87106E09DE05648C07945
:107CC000F02188435449C87140202040002807D043
:107CD00051484079F021884370304F49487105E0A0
:107CE0004D484079F02188434B4948710A21039857
:107CF000F0F72CFA0D464948445DE007C00F002814
:107D000007D04548C07800090001C01D4249C8702D
:107D100005E04148C078000900013F49C8700220D1
:107D20002040002807D03C488078F02188437030FC
:107D30003949887005E038488078F0218843364911
:107D4000887004202040002807D033484078F02174
:107D5000884370303049487005E02F484078F02162
:107D600088432D49487008202040002807D02A4821
:107D7000407800090001C01D2749487005E02648E9
:107D80004078000900012449487010202040002854
:107D900007D02148007900090001C01D1E49087163
:107DA00005E01D480079000900011B4908712020E9
:107DB0002040002807D01848C078F0218843703050
:107DC0001549C87005E01448C078F021884312496D
:107DD000C87040202040002807D00F488078000954
:107DE0000001C01D0C49887017E10B48807800091C
:107DF00000010949887010E107484079F021884363
:107E00007030054948710846807800090001C01D9E
:107E100088700846C07905E09C260020F819020009
:107E20000B1A020000090001C87108468079000998
:107E30000001887108464079000900014871084630
:107E4000007AF0218843764908720846007A0009D2
:107E5000000108720846C079F02188437049C87152
:107E60000846C07800090001C87008468078F021F3
:107E700088436B49887008464078F02188436849F8
:107E800048700846407800090001487008460079AB
:107E90000009000108710846C078F0218843604954
:107EA000C870BAE0032E9FD1F8F750FF05285FD1C4
:107EB000F9F74AF800280DD059484079F021884355
:107EC0007030574948710846807800090001C01D8C
:107ED00088700AE052484079F0218843504948713F
:107EE000084680780009000188704D48C079000973
:107EF00000014B49C871084680790009000188716A
:107F0000084640790009000148710846007AF021CE
:107F10008843434908720846007A00090001087244
:107F20000846C079F02188433D49C8710846C078A9
:107F300000090001C87008468078F021884338495C
:107F4000887008464078F0218843354948700846D3
:107F500040780009000148700846007900090001D6
:107F600008710846C078F02188432D49C87054E054
:107F70002B480079F0218843703029490871084660
:107F80004079F0218843703025494871084680784F
:107F900000090001C01D88700846C0790009000171
:107FA000C871084680790009000188710846407947
:107FB0000009000148710846007AF02188431849F9
:107FC00008720846007A0009000108720846C07964
:107FD000F02188431249C8710846C07800090001A1
:107FE000C87008468078F02188430D49887008469B
:107FF0004078F02188430A494870084640780009D3
:10800000000148700846007900090001087108461F
:10801000C078F02188430249C87005B0F0BD000067
:108020009C26002070B505460C46012D7ED1B14836
:10803000407D00090001C01DAE4948750846007D1D
:10804000F02188431030AB4908750846007D0009CF
:108050000001401C08750846C07CF02188431030A0
:10806000A449C8740846807CF02188431030A14997
:1080700088740846807C00090001401C8874F8F769
:10808000BFFF022803D0F8F7BBFF01286CD19A4844
:108090000078012868D0F4F7ADFC9849884263D392
:1080A000F8F752FF00282FD09248007DF021884336
:1080B0007030904908750846007D00090001C01D18
:1080C00008750846C07CF021884370308949C8741F
:1080D0000846807CF02188437030864988740846C1
:1080E000807C00090001C01D88740846407DF02195
:1080F000884370307F4948750846407CF0218843AA
:1081000070307C494874F4E07A48007DF02188435F
:108110001030784908750846007D00090001401CB0
:1081200008750846C07CF021884300E0B4E01030B8
:108130007049C8740846807CF021884310306D492E
:1081400088740846807C00090001401C8874084639
:10815000407DF0218843674948750846407CF021FE
:10816000884364494874C4E0F8F7DEFD002824D150
:10817000F4F740FC614988421FD3F8F7E5FE002878
:108180000ED05C48407DF0218843703059494875D5
:108190000846407CF02188437030564948741AE004
:1081A0005448407DF0218843524948750846407C38
:1081B000F02188434F4948740DE04E48407DF0213E
:1081C000884370304B4948750846407CF02188430D
:1081D000703048494874F8F7A7FD01282AD146486D
:1081E0000078012826D0F4F705FC4449884221D3C1
:1081F0004048407DF021884370303E49487508462C
:10820000407CF021884370303A494874F8F79CFE6E
:10821000002807D03748007DF02188437030354969
:10822000087566E03348007DF021884310303149FD
:1082300008755EE0230008F045FC062C241C140C95
:10824000042D2C48807C00090001C01D2949887438
:1082500000BF2848807CF02188437030254988740D
:1082600000BF2448C07CF021884370302149C87485
:1082700000BF2048007D00090001C01D1D49087590
:1082800000BF1C48007DF0218843703019490875F3
:1082900000BF00E000BF2CE01648407DF02188437D
:1082A000144948750846007DF02188431149087536
:1082B0000846007D0009000108750846C07CF021D1
:1082C00088430C49C8740846807CF02188430949DA
:1082D00088740846807C0009000188740846407D47
:1082E0000009000148750846407CF0218843014997
:1082F000487470BD7C260020F1000020B80B0000FF
:1083000030B50246002901D1002000E0072013000B
:1083100008F0D8FB0F09141F2B3743505D67727CA0
:1083200088929FA9B500574B5B7EF024A3430401BC
:10833000F0252C402343534C6376A1E0524B9B79AC
:10834000F024A3430401F0252C4023434E4CA37199
:1083500096E04D4B2033DB791B091B010407240FEA
:108360002343494C2034E3718AE0464B2033DB7CC5
:108370001B091B010407240F2343424C2034E374E0
:108380007EE0404B40331B781B091B010407240F80
:1083900023433C4C4034237072E03A4B2033DB7F64
:1083A000F024A3430401F0252C402343354C203412
:1083B000E37765E0334B20335B7BF024A343040178
:1083C000F0252C4023432F4C2034637358E02E4B70
:1083D0009B791B091B010407240F23432A4CA3711B
:1083E0004EE0294B9B7CF024A3430401F0252C4054
:1083F0002343254CA37443E0234BDB7E1B091B0165
:108400000407240F2343204CE37639E01D4B20332F
:10841000DB7F1B091B010407240F2343194C203465
:10842000E3772DE0174B9B7E1B091B010407240FEC
:108430002343144CA37623E0134B20339B79F02481
:10844000A3430401F0252C4023430F4C2034A37197
:1084500016E00D4BDB7D1B091B010407240F234392
:10846000094CE3750CE0074B20335B7C1B091B01B7
:108470000407240F2343034C2034637400E000BF3F
:1084800000BF30BD5C26002030270020F7B582B049
:108490000746154600260024FE480078012804D02F
:1084A000F4F7A8FAFC49884279D2FC48407CF021D4
:1084B00088437030F94948740846807C00090001FF
:1084C000C01D88740846007D00090001C01D0875A4
:1084D0000846007DF02188437030F0490875084651
:1084E000807CF02188437030EC4988740846C07C59
:1084F00000090001C01DC8740846C07CF0218843F3
:108500007030E649C8740846407C00090001C01D6F
:1085100048740846407D00090001C01D48750846A2
:10852000407DF02188437030DC4948750846007C66
:10853000F02188437030D94908740846007C00094E
:108540000001C01D08740846C07BF02188437030CC
:10855000D249C873FF220A210020FBF713F9FF223A
:1085600013210020FBF70EF9FF2211210020FBF759
:1085700009F9FF2212210020FBF704F9FF220E2146
:108580000020FBF7FFF8FF220F210020FBF7FAF88D
:10859000FF2210210020FBF7F5F8F4E3FFE7039832
:1085A00036283DD019DC08287ED007DC801E030069
:1085B00008F088FA0635A8FCFBFAF97E102874D07A
:1085C00006DC092872D00D2871D00E2870D1FDE389
:1085D00033286ED03428F9D170E13F286AD00FDCFF
:1085E0003738082864D243007B449B885B009F4453
:1085F0008A009702FF025F005F006503CB0318004B
:108600004E287BD006DC402879D0412878D04D28F0
:10861000DCD1BBE14F2874D05028D7D14FE100BF47
:1086200000BF9E48407CF02188439C49487408461E
:10863000807C0009000188740846007D0009000163
:10864000C01D08750846007DF021884370309349AD
:1086500008750846807CF021884390498874084654
:10866000C07C00090001C01DC8740846C07CF02110
:1086700088438A49C8740846407C00090001487450
:108680000846407D0009000148750846407DF021FC
:108690008843824948750846007CF02188437F4919
:1086A00008740846007C06E0A1E2FDE337E2D2E36D
:1086B000FBE394E028E00009000108740846C07B51
:1086C000F02188437549C873FF220A210020FBF777
:1086D00059F8FF2213210020FBF754F800220E2145
:1086E0001046FBF74FF800220F211046FBF74AF81F
:1086F000002210211046FBF745F877E2ABE110E2CB
:10870000DDE26DE000BF00BF6448407CF02188439B
:10871000624948740846807C000900018874084654
:10872000007D00090001C01D08750846007DF0218C
:1087300088437030594908750846807CF021884389
:10874000564988740846C07C00090001C874084670
:10875000C07CF02188435149C8740846407C000918
:10876000000148740846407D00090001C01D48759D
:108770000846407DF0218843484948750846007CFA
:10878000F0218843454908740846007C000900012F
:1087900008740846C07BF02188434049C873FF2213
:1087A0000A21002003E055E1EFE086E016E0FAF749
:1087B000E9FFFF2213210020FAF7E4FF00220E2137
:1087C0001046FAF7DFFF00220F211046FAF7DAFF12
:1087D000002210211046FAF7D5FF8EE700BF00BF38
:1087E0002E48407CF02188432C4948740846807C00
:1087F00000090001C01D88740846007D00090001C1
:10880000C01D08750846007DF0218843703023495B
:1088100008750846807CF021884370301F498874B1
:108820000846C07C00090001C8740846C07CF021DD
:1088300088431A49C8740846407C000900014874FE
:108840000846407D0009000148750846407DF0213A
:108850008843124948750846007CF02188430F4937
:1088600008740846007C0009000108740846C07BB3
:10887000F02188430949C873FF220A210020FAF732
:1088800081FFFF2213210020FAF77CFF00220E2136
:10889000104605E0F1000020B80B00009C260020E7
:1088A000FAF770FF00220F211046FAF76BFF002243
:1088B00010211046FAF766FF1FE700BF00BFFE4811
:1088C000407CF0218843FC4948740846807C0009BC
:1088D0000001C01D88740846007D00090001C01D0C
:1088E00008750846007DF02188437030F24908750C
:1088F0000846807CF0218843EF4988740846C07C94
:1089000000090001C8740846C07CF0218843EA4988
:10891000C8740846407C00090001C01D4874084620
:10892000407D0009000148750846407DF0218843DC
:10893000E14948750846007CF0218843DE49087407
:108940000846007C0009000108740846C07BF0213D
:108950008843D949C873FF220A210020FAF712FF81
:10896000FF2213210020FAF70DFF00220E211046EE
:10897000FAF708FF00220F211046FAF703FF002242
:1089800010211046FAF7FEFEF6E300BFCA48407C0D
:10899000F0218843C84948740846807C00090001DA
:1089A00088740846007D0009000108750846007DAE
:1089B000F02188437030C04908750846807CF0215A
:1089C0008843BD4988740846C07C00090001C8740A
:1089D0000846C07CF02188437030B749C874084607
:1089E000407C0009000148740846407D00090001F0
:1089F00048750846407DF0218843AF4948750846D0
:108A0000007CF0218843AC4908740846007C0009CA
:108A1000000108740846C07BF0218843A649C8734A
:108A2000FF220A210020FAF7ADFEFF2213210020C9
:108A3000FAF7A8FE00220E211046FAF7A3FE002244
:108A40000F211046FAF79EFE002210211046FAF779
:108A500099FE91E300BF9848407CF02188439649F5
:108A600048740846807C0009000188740846007D2F
:108A70000009000108750846007DF0218843703028
:108A80008D4908750846807CF02188438A4988749E
:108A90000846C07C00090001C8740846C07CF0216B
:108AA00088438549C8740846407C00090001487421
:108AB0000846407D0009000148750846407DF021C8
:108AC000884370307C4948750846007CF021884313
:108AD000794908740846007C0009000108740846BA
:108AE000C07BF02188437449C873FF220A2100200B
:108AF000FAF748FEFF2213210020FAF743FE002276
:108B00000E211046FAF73EFE00220F211046FAF71A
:108B100039FE002210211046FAF734FE2CE300BF84
:108B200000BF6548407CF02188437030624948743A
:108B30000846807C00090001C01D88740846007D3D
:108B400000090001C01D08750846007DF02188431A
:108B50007030594908750846807CF0218843564991
:108B600088740846C07C00090001C8740846C07CAF
:108B7000F02188435049C8740846407C0009000130
:108B800048740846407D0009000148750846407D4C
:108B9000F0218843484948750846007CF021884305
:108BA000454908740846007C00090001087408461D
:108BB000C07BF02188434049C873FF220A2100206E
:108BC000FAF7E0FDFF2213210020FAF7DBFD002277
:108BD0000E211046FAF7D6FD00220F211046FAF7B3
:108BE000D1FD002210211046FAF7CCFDC4E200BFEF
:108BF0003148407CF02188432F4948740846807CE6
:108C00000009000188740846007D0009000108750C
:108C10000846007DF02188437030274908750846D2
:108C2000807CF0218843244988740846C07C000970
:108C30000001C8740846C07CF021884370301E498A
:108C4000C8740846407C0009000148740846407D0D
:108C50000009000148750846407DF0218843164907
:108C600048750846007CF02188431349087408467B
:108C7000007C0009000108740846C07BF02188438D
:108C80000D49C873FF220A210020FAF77BFDFF225D
:108C900013210020FAF776FD00220E211046FAF784
:108CA00071FD00220F211046FAF76CFD0022102101
:108CB0001046FAF767FD5FE29C26002000BFFC48E3
:108CC000407CF0218843FA4948740846807C0009BA
:108CD000000188740846007D0009000108750846F7
:108CE000007DF02188437030F14908750846807C8A
:108CF000F0218843EE4988740846C07C00090001D1
:108D0000C8740846C07CF0218843E949C874084605
:108D1000407C0009000148740846407D00090001BC
:108D200048750846407DF02188437030E049487519
:108D30000846007CF0218843DD4908740846007C21
:108D40000009000108740846C07BF0218843D84917
:108D5000C873FF220A210020FAF714FDFF22132115
:108D60000020FAF70FFD00220E211046FAF70AFD47
:108D700000220F211046FAF705FD002210211046AF
:108D8000FAF700FDF8E1F8E1C948407CF02188439A
:108D90007030C74948740846807C00090001C01D36
:108DA00088740846007D00090001C01D087508464A
:108DB000007DF0218843BE4908750846807CF0217B
:108DC0008843BB4988740846C07C00E0A9E00009DC
:108DD0000001C8740846C07CF0218843B449C874B7
:108DE0000846407C0009000148740846407D00099F
:108DF000000148750846407DF0218843AC4948751C
:108E00000846007CF0218843A94908740846007C84
:108E10000009000108740846C07BF0218843A4497A
:108E2000C873FF220A210020FAF7ACFCFF221321AD
:108E30000020FAF7A7FC00220E211046FAF7A2FC48
:108E400000220F211046FAF79DFC00221021104647
:108E5000FAF798FC90E19648407CF02188439449C9
:108E600048740846807C0009000188740846007D2B
:108E70000009000108750846007DF02188438C49EF
:108E800008750846807CF021884389498874084623
:108E9000C07C00090001C8740846C07CF0218843EA
:108EA0008349C874084601E09EE003E1407C000964
:108EB000000148740846407D0009000148750846D5
:108EC000407DF02188437A4948750846007CF021AE
:108ED0008843774908740846007C0009000108743B
:108EE0000846C07BF021884370307149C873002266
:108EF0000A211046FAF746FC002213211046FAF721
:108F000041FCFF220E210020FAF73CFC00220F2139
:108F10001046FAF737FC002210211046FAF732FC0F
:108F20002AE16348407CF02188436149487408463F
:108F3000807C0009000188740846007D000900015A
:108F400008750846007DF021884359490875084690
:108F5000807CF0218843564988740846C07C00090B
:108F60000001C8740846C07CF02188435049C87489
:108F70000846407C0009000148740846407D00090D
:108F8000000148750846407DF021884348494875EE
:108F90000846007CF0218843454908740846007C57
:108FA00000090001C01D08740846C07BF0218843F9
:108FB0003F49C87300220A211046FAF7E3FB00225A
:108FC00013211046FAF7DEFB00220E211046FAF7B5
:108FD000D9FBFF220F210020FAF7D4FB0022102139
:108FE0001046FAF7CFFBC7E03148407CF0218843B8
:108FF0002F4948740846807C00090001887408469F
:10900000007D0009000108750846007DF0218843B5
:10901000274908750846807CF021884324498874D4
:109020000846C07C00090001C8740846C07CF021D5
:1090300088431F49C8740846407C000900014874F1
:109040000846407D0009000148750846407DF02132
:109050008843174948750846007CF02188437030E2
:10906000134908740846007C00090001087408468A
:10907000C07BF02188430E49C87300220A211046A4
:10908000FAF780FB002213211046FAF77BFB00223F
:109090000E211046FAF776FB00220F211046FAF750
:1090A00071FBFF2210210020FAF76CFB64E0000046
:1090B0009C260020FD48407CF0218843FB494874F1
:1090C0000846807C0009000188740846007D00097C
:1090D000000108750846007DF0218843F3490875B2
:1090E0000846807CF0218843F04988740846C07C9B
:1090F00000090001C8740846C07CF0218843EB4990
:10910000C8740846407C0009000148740846407D48
:109110000009000148750846407DF0218843E34975
:1091200048750846007CF0218843E04908740846E9
:10913000007C0009000108740846C07BF0218843C8
:10914000DA49C87300220A211046FAF71BFB0022F5
:1091500013211046FAF716FB00220E211046FAF7EB
:1091600011FB00220F211046FAF70CFB0022102100
:109170001046FAF707FB00BF00BF002F03D0CC4812
:10918000007A002808D1F3F735FCCA49884203D396
:10919000C9480078012872D1FF2211210020FAF776
:1091A000F1FAFF2212210020FAF7ECFAC248007807
:1091B000012804D0F3F71EFCBE49884216D2BF48EE
:1091C000807BF02188437030BC498873084640306A
:1091D0000078F02188437030B84940310870084663
:1091E000007800090001C01D08702DE07D20C0003E
:1091F000854214D2B148807BF0218843AF498873FF
:10920000084640300078F02188437030AB49403147
:1092100008700846007800090001087014E0A748AB
:10922000807BF02188437030A44988730846403021
:109230000078F0218843A149403108700846007841
:1092400000090001C01D08707D20C000854205D2C4
:1092500001462846EEF77AFF064604E0984928467C
:10926000EEF774FF064694480078012804D0F3F71F
:10927000C1FB9049884203D29248845D02E0A0E29B
:109280009148845DE007C00F002809D08B4840302A
:10929000C07800090001C01D88494031C87007E04E
:1092A00086484030C0780009000184494031C870C8
:1092B00002202040002807D08048C0790009000122
:1092C000C01D7E49C87105E07C48C07900090001D5
:1092D0007A49C87104202040002807D07748807957
:1092E00000090001C01D7549887105E07348807947
:1092F000000900017149887108202040002807D02A
:109300006E484079F021884370306C49487105E01F
:109310006A484079F021884368494871102020400C
:10932000002807D06548407900090001C01D634945
:10933000487105E061484079000900015F494871C2
:1093400020202040002807D05C480079F021884385
:1093500070305A49087105E058480079F021884377
:109360005649087140202040002807D05348807992
:10937000F021884370305149887105E04F48807969
:10938000F02188434D4988717D20C000854213D269
:1093900064212846EEF7DAFE0646474800780128A1
:1093A00004D0F3F727FB4349884202D24548845D45
:1093B00023E04548845D20E0642128463230EEF702
:1093C000C5FE7D21C9000090EEF7C0FE0191642129
:1093D0000198EEF7BBFE06463C48854208D2364867
:1093E0000078012804D0F3F705FB3249884202D205
:1093F0003448845D01E03448845DE007C00F0028F4
:1094000009D02E4840308078F021884370302B49B5
:109410004031887007E0294840308078F021884347
:1094200026494031887002202040002807D0234878
:10943000807A00090001C01D2049887205E01F489C
:10944000807A000900011D4988720420204000280C
:1094500007D01A48407A00090001C01D1749487218
:1094600005E01648407A00090001144948720820B6
:109470002040002807D01148007AF021884370303E
:109480000E49087205E00D48007AF02188430B4927
:1094900008721020204000281AD00848007A0009DD
:1094A0000001C01D0549087218E000009C2600203C
:1094B000600A0020B80B0000F100002010270020F7
:1094C000A0860100F81902000B1A02001027000004
:1094D000FE48007A00090001FC4908722020204063
:1094E000002807D0F948C079F02188437030F74947
:1094F000C87105E0F548C079F0218843F349C87187
:1095000040202040002807D0F048407AF0218843CE
:109510007030EE49487205E0EC48407AF02188430B
:10952000EA4948727D20C000854219D20A212846A6
:10953000EEF70CFE0A210190EEF708FE0E460A2D0A
:1095400008D2E3480078012804D0F3F753FAE14940
:10955000884202D2E048845D12E0E048845D0FE07A
:10956000642128463230EEF7F1FD0A210090EEF733
:10957000EDFD0A210190EEF7E9FD0E46D6498C5D1E
:10958000E007C00F002809D0D0484030807800099B
:109590000001C01DCD494031887007E0CB48403004
:1095A000807800090001C9494031887002202040BC
:1095B000002807D0C548807B00090001C01DC349B1
:1095C000887305E0C148807B00090001BF498873AA
:1095D00004202040002807D0BC48407B000900013F
:1095E000C01DBA49487305E0B848407B0009000136
:1095F000B649487308202040002807D0B348007BB4
:10960000F02188437030B149087305E0AF48007B12
:10961000F0218843AD49087310202040002807D06E
:10962000AA48C07A00090001C01DA849C87205E017
:10963000A648C07A00090001A449C8722020204031
:10964000002807D0A148807AF021884370309F49D4
:10965000887205E09D48807AF02188439B49887292
:1096600040202040002807D09848407BF0218843C4
:1096700070309649487305E09448407BF021884358
:10968000924948737D20C000854207D20A212846AE
:10969000EEF75CFD0E469048845D0BE064212846A1
:1096A0003230EEF753FD0A210190EEF74FFD0E46E2
:1096B00089498C5DE007C00F002809D083484030FD
:1096C0004078F0218843703080494031487007E08D
:1096D0007E4840304078F02188437C4940314870D2
:1096E00002202040002809D0784840304078000906
:1096F0000001C01D75494031487007E07348403093
:109700004078000900017149403148700420204030
:10971000002807D06D48007CF021884370306B49E9
:10972000087405E06948007CF021884367490874A3
:1097300008202040002807D06448007C0009000170
:10974000C01D6249087405E06048007C0009000102
:109750005E49087410202040002807D05B48C07B79
:10976000F021884370305949C87305E05748C07BE1
:10977000F02188435549C87320202040002807D095
:109780005248C07B00090001C01D5049C87305E064
:109790004E48C07B000900014C49C873402020405E
:1097A000002807D04948407C00090001C01D4749F6
:1097B0004874ECE04548407C000900014349487486
:1097C000E5E000220A211046F9F7DCFF0022132110
:1097D0001046F9F7D7FF002211211046F9F7D2FF02
:1097E000002212211046F9F7CDFF00220E2110466B
:1097F000F9F7C8FF00220F211046F9F7C3FF002236
:1098000010211046F9F7BEFF30484030C0780009FB
:1098100000012E494031C8702C48C0790009000170
:109820004039C871084680790009000188710846EE
:109830004079F0218843254948710846407900095C
:109840000001487108460079F02188431F490871DA
:1098500008468079F02188431C49887108464030C9
:109860008078F02188431949403188701748807A00
:1098700000090001403988720846407A0009000159
:1098800048720846007AF021884310490872084659
:10989000007A0009000108720846C079F021884367
:1098A0000A49C8710846407AF0218843074948723E
:1098B0000846403080780009000140318870034834
:1098C000807B000900014039887309E010270020DF
:1098D000F1000020B80B0000F81902000B1A02007A
:1098E0000846407B0009000148730846007BF021D0
:1098F0008843284908730846C07A00090001C872E5
:109900000846807AF0218843224988720846407BC5
:10991000F02188431F494873084640304078F021C1
:1099200088431C49403148700846407800090001CE
:1099300048701848007CF02188431649087408468E
:10994000007C0009000108740846C07BF0218843B0
:109950001049C8730846C07B00090001C873084657
:10996000407C0009000148740846807BF021884350
:1099700008498873084640300078F021884305493B
:10998000403108700846007800090001087005B0F1
:10999000F0BD000010270020F7B582B007460E4644
:1099A0000121FF200830FBF799FF0121FC48FBF75C
:1099B00095FFFC48007801287ED0F3F71BF8FA49A0
:1099C000884279D3F7F7C2F9032843D1F7F7B8F9FA
:1099D000002803D0F7F7B4F901283BD1002F1CD1A0
:1099E000F7F7B2FA00280CD0F048407CF021884309
:1099F000EE4948740846807C00090001C01D887447
:109A0000EEE0EA48407CF0218843E8494874084683
:109A1000807C000900018874E2E0F7F795FA0028DD
:109A20000CD0E248407CF02188437030DF49487414
:109A30000846807C000900018874D1E0DB48407C46
:109A4000F0218843D94948740846807C0009000108
:109A50008874C5E0F7F774F9002803D0F7F770F9B8
:109A6000012865D1002F0CD1D048407CF0218843DB
:109A7000CE4948740846807C00090001C01D8874E6
:109A80000BE0CA48407CF02188437030C7494874D5
:109A90000846807C000900018874F7F751F9002816
:109AA00021D1C2482030C078F02188437030BF49AE
:109AB0002031C870BD4800E064E0807D00090001ED
:109AC000203988750846807DF0218843B74988751C
:109AD000FF2223210020F9F755FE00222221104603
:109AE000F9F750FE7CE0F7F72BF9012878D1AF4861
:109AF0002030C078F0218843AC492031C870AB4891
:109B0000807D00090001C01D203988750846807DD0
:109B1000F02188437030A549887500222321104622
:109B2000F9F730FEFF2222210020F9F72BFE57E043
:109B30009E48407CF02188439C4948740846807CBC
:109B400000090001887408462030C078F02188435D
:109B500096492031C8709548807D00090001203960
:109B600088750846807DF0218843904988750022D9
:109B700023211046F9F706FE002222211046F9F7AC
:109B800001FE2DE08948407CF021884370308749F0
